:1000000000800020BD010000B9E1000071E10000A6
:1000100071E1000071E1000071E1000071E1000098
:1000200071E1000071E1000071E10000B9E1000040
:10003000B9E1000071E10000FDFA000001FC0000E0
:10004000B9E10000B9E10000B9E10000B9E1000048
:10005000B9E10000B9E10000B9E10000B9E1000038
:10006000B9E10000B9E10000B9E10000B9E1000028
:10007000B9E10000B9E10000B9E10000B9E1000018
:10008000B9E10000B9E10000B9E10000B9E1000008
:10009000B9E10000B9E10000B9E10000B9E10000F8
:1000A000C5C20000D1C20000B9E10000B9E1000002
:1000B000B9E10000B9E10000B9E10000B9E10000D8
:1000C000B9E10000B9E10000B9E10000B9E10000C8
:1000D000B9E10000B9E10000B9E10000B9E10000B8
:1000E000B9E10000B9E10000B9E10000B9E10000A8
:1000F000B9E10000D9FF0000B9E1000005010100ED
:10010000B9E1000041EA0000B9E10000B9E10000F6
:10011000B9E10000B9E10000B9E10000B9E1000077
:10012000B9E10000B9E10000B9E10000B9E1000067
:10013000B9E10000B9E10000B9E10000B9E1000057
:10014000B9E10000B9E10000B9E10000B9E1000047
:10015000B9E10000B9E10000B9E10000B9E1000037
:10016000B9E1000019ED0000B9E10000B9E10000BB
:10017000B9E10000B9E10000B9E10000B9E1000017
:10018000B9E10000B9E10000B9E10000B9E1000007
:10019000B9E10000B9E10000B9E10000B9E10000F7
:1001A000B9E10000B9E10000B9E10000B9E10000E7
:1001B000B9E10000B9E10000B9E10000564B4CF292
:1001C000205210B51A804DF628121A8000BF00BFC9
:1001D0000DF0F6FF514B4FF010621A60504A9A60D2
:1001E000504ADA60504A136813F4807304D14F49BF
:1001F0000B604FF4A85313604D4B1A78110703D5C9
:100200001A7842F008021A704A4B4B492A221A7097
:100210004A4A4B4B8B4204D252F8040F43F8040B6A
:10022000F8E7484B484900228B4202D243F8042B9E
:10023000FAE74649464A002352F8230041F82300D2
:1002400001336F2BF8D1434B434A802103F8011B44
:100250009342FBD1414B3D4A1A60414B8A221A70AE
:10026000A3F5805324225A70A0221A709A7992071B
:10027000FCD59A79D406FCD43A4A937903F00C035E
:10028000082B384BF9D103221A7140225A719A79FE
:100290009006FCD5334A9179324B4906FBD5324A58
:1002A000324911600221516020221A709A7902F0BD
:1002B0000C020C2AFAD12E4B2E4A1A602E4B2F4AD2
:1002C0001A6000225A60072243F8042C2C4AC3F813
:1002D0000C2D62B60EF07CFA144B1B68DA0705D5BC
:1002E00028480EF0CBF8284B284A1A60284B1B7878
:1002F0005B0609D5244C254B22689A4204D121483B
:100300000EF0BCF80023236011F0E4F90DF05EFF5D
:100310000FF0C2FDFEE700BF0E2005403080044014
:10032000823F04000100002B10D0034014D0034092
:1003300002D0074000E007403C9DFF1F74300100E1
:100340004088FF1F3C9DFF1F04A2FF1F0082FF1F6C
:100350000000000000E400E05FE400E008ED00E0E1
:100360000050064000400640448004400000030165
:1003700004800440C010050014E000E0FF76010096
:1003800000002020A956265C1CE00340A5C3945A17
:1003900000F00740FFFFFFFFFFFFFFFFFFFFFFFF32
:1003A000FFFFFFFFFFFFFFFFFFFFFFFFFFFFFFFF5D
:1003B000FFFFFFFFFFFFFFFFFFFFFFFFFFFFFFFF4D
:1003C000FFFFFFFFFFFFFFFFFFFFFFFFFFFFFFFF3D
:1003D000FFFFFFFFFFFFFFFFFFFFFFFFFFFFFFFF2D
:1003E000FFFFFFFFFFFFFFFFFFFFFFFFFFFFFFFF1D
:1003F000FFFFFFFFFFFFFFFFFFFFFFFFFFFFFFFF0D
:10040000FFFFFFFFFFFFFFFFFFFFFFFFDEF9FFFF23
:1004100010B5054C237833B9044B13B10448AFF33E
:1004200000800123237010BD3C9DFF1F00000000D1
:1004300078300100084B10B51BB108490848AFF3EC
:1004400000800848036803B910BD074B002BFBD0A0
:10045000BDE81040184700BF00000000409DFF1F8E
:10046000783001003C9DFF1F0000000070B44C6814
:10047000A04220D901230133DBB21CB2A60051F8FF
:10048000244084421D46F6D3A04211D005F1804598
:10049000013D965951F8251052F82530401AF21AAC
:1004A00000FB02F0641AB0FBF4F4E01870BC704773
:1004B000905970BC704704260125E5E700280CDA46
:1004C000064A434282FB0320DA17C2EB600000EBCE
:1004D0004000A3EB8000C0F10C007047ABAAAA2A31
:1004E000684B1B880C2B12D8DFE803F01E29333D24
:1004F0001148525C66707A12070063490B68984293
:1005000078D90B6C9842C0F0A580604B186C70478E
:100510005D490B68984240F28E800B6C9842C0F0A7
:1005200096805B4B186C704757490B6898427FD98F
:100530000B6C9842C0F08880564B186C704752493B
:100540000B68984271D90B6C98427AD3524B186C55
:1005500070474D490B68984264D90B6C98426DD333
:100560004E4B186C704748490B68984257D90B6C32
:100570009842C0F084804A4B186C704742490B681F
:10058000984249D90B6C984276D3464B186C704709
:100590003D490B6898423CD90B6C984269D3424B59
:1005A000186C704738490B6898422FD90B6C9842E9
:1005B0005CD33E4B186C704733490B68984222D984
:1005C0000B6C98424FD33A4B186C70472E490B680E
:1005D000984215D90B6C984242D3364B186C704731
:1005E00029490B68984208D90B6C984235D3324B95
:1005F000186C7047254B186870472F4B1868704768
:100600002C4B186870472A4B18687047274B18689E
:100610007047254B18687047224B18687047204B6D
:10062000186870471D4B186870471B4B1868704757
:10063000184B18687047164B18687047174AFFF731
:1006400015BF154AFFF712BF124AFFF70FBF104A36
:10065000FFF70CBF0D4AFFF709BF174AFFF706BFA8
:10066000144AFFF703BF124AFFF700BF0F4AFFF714
:10067000FDBE0D4AFFF7FABE0A4AFFF7F7BE084A69
:10068000FFF7F4BEAA9DFF1FDC8AFF1FC88BFF1F68
:10069000848BFF1F488DFF1F7C89FF1F048DFF1F68
:1006A0003489FF1FA08DFF1FC089FF1F048AFF1F11
:1006B000488AFF1FA88CFF1F408CFF1F38B51D4DB7
:1006C0001D482B78013B1B0203F4706318430EF0A6
:1006D000D1FF2878013860F04F00C0B20EF08AF9DF
:1006E0007B200EF087F900200EF084F900242B788F
:1006F000013B1B0203F47063200443F4004343F006
:10070000080300F4FE0018430EF0B4FF2878013807
:1007100060F07F00C0B20EF06DF920460EF06AF96D
:1007200000200EF067F9013402200EF003F8802C4F
:10073000DDD138BD018DFF1F0BB07B0010B5174C0C
:1007400017482378013B1B0203F4706318430EF033
:1007500091FF2078013860F04F00C0B20EF04AF9E6
:1007600007200EF047F964200EF044F923780D4875
:10077000013B1B0203F4706318430EF07BFF2078EB
:10078000013860F04F00C0B20EF034F90B200EF0CB
:1007900031F97F20BDE810400EF02CB9018DFF1F0C
:1007A0000BB007640BB00B7F10B5044641F0E000BE
:1007B0000EF020F904F07F000EF01CF9C4F3C6100F
:1007C000BDE810400EF016B938B5054642F0B0004D
:1007D0000C460EF00FF928460EF00CF9E0B2BDE819
:1007E00038400EF007B900BF38B5054642F090001A
:1007F0000C460EF0FFF828460EF0FCF8E0B2BDE81B
:1008000038400EF0F7B800BF38B5054642F080001A
:100810000C460EF0EFF828460EF0ECF8E0B2BDE81A
:1008200038400EF0E7B800BF38B5284A284B148886
:100830001D68AC4247DA274A274B10781B88421FB5
:10084000191BAB42A8BF2B469142A3EB0403C3BFC5
:10085000043843430131534393FBF1F105310A203E
:100860000DF01EFE1D4A1E4B14881B68A34205DCBA
:1008700000210920BDE838400DF012BE19491A4A7E
:100880000D881078AB42A5EB0401A0F10502A8BFCA
:100890002B4691420CDD1B1B043800FB03F3013196
:1008A000092093FBF1F1BDE8384005310DF0F8BDAA
:1008B0001B1B02FB03F3092093FBF1F1BDE8384059
:1008C00005310DF0EDBD0021C9E700BF169EFF1FE9
:1008D000AC9EFF1FF88DFF1FBC9EFF1FE49DFF1FF6
:1008E0006C9DFF1FA09EFF1F8C8DFF1F5A4A5B4B04
:1008F00010881B685A4A5B49128883422DE9F047E9
:1009000034DB9342A8BF134698420B60C8BF002354
:100910002EDD101AB0F5804FAABF9B03C3EB8333C3
:10092000013093FBF0F0FFF7DBFD4F4FC5093B684B
:1009300005F07F069E4204460AD0DFF83881B8F8F9
:100940000020002A61D1494B1B88002B3FD13E601B
:10095000474D2B689C4207D0464E3288531F032BCD
:100960000DD92C60BDE8F087BDE8F087034608602C
:100970009A42D4BFC0EB0203C0EB0303C9E7DFF820
:10098000FC803D4F98F80030BA5C013B1B0203F439
:100990007063203243F43043120402F4FE0243F049
:1009A0000B032006134300F0FE4018430EF062FED6
:1009B000338898F80020F85C013A2030D2B2C0B2F7
:1009C00004F07F01FFF700FF2C60BDE8F087DFF83F
:1009D000AC8098F800000138000200F470602D042B
:1009E00040F4504005F4FE0540F00D0028430EF0A1
:1009F00041FE98F80000013860F02F00C0B20DF001
:100A0000F9FF30460DF0F6FFA1E7DFF870A0DFF840
:100A100068909AF8003019F80220013B1B0203F499
:100A2000706343F43043120402F4FE02280643F0DC
:100A30000B03134300F0FE4018430EF01BFE9AF820
:100A40000020B8F80030013AD2B219F8030031465C
:100A5000FFF7BAFE77E700BF169EFF1F889EFF1FB5
:100A6000BC9EFF1FAC9EFF1FD89DFF1F129EFF1F45
:100A7000A49DFF1F689EFF1FEC8CFF1F018DFF1FB1
:100A80002DE9F04F172087B00EF046F8DFF8649399
:100A9000C9F8000016200EF03FF8BB4BBB4A1B887C
:100AA00010600C2B00F069820023B94C0F202370DA
:100AB0000EF032F8B74A2378128801921146B64AEE
:100AC000054652F821404BB1204610F09DFB4FF0F7
:100AD0007C5110F0EDFB10F0B1FD0446AF4BDFF898
:100AE00018831B88D8F800A0AD4A013B554552F841
:100AF00023B050DAAB4BAC4E1B88012B00F0EF81DA
:100B0000AA4BAB4A306800931F46049210F07CFB5E
:100B10004FF07C5110F0CCFBA6490290098803915C
:100B2000204610F071FB049A03993F6852F8211097
:100B300010F0BEFB0146002010F0B0FA10F07EFD70
:100B4000CBEB070BAB45CAEB0B015A46B8BF2A46A5
:100B5000CAEB02028842BABF00FB022201314243C3
:100B600092FBF1F0DFF894A210F04EFB4FF07C51B5
:100B700010F09EFB029910F093FA10F05FFD3060C8
:100B80008D4A1288013A032A6AD8DFE812F045013B
:100B9000F10053003901DFF864A2DAF80020954231
:100BA00038DD804B05921B887F4E012B00F0C681FB
:100BB0007E4B00931F4630687D4B049310F024FB5E
:100BC0004FF07C5110F074FB7A4902900988039130
:100BD000204610F019FB0399049B3F6853F821103D
:100BE00010F066FB10F02AFD059ABB44C2EB0B0126
:100BF000AB45A8BFAB468842C2EB0B0B80F2C78166
:100C000000FB0BBB01319BFBF1F010F0FDFA4FF044
:100C10007C51ADE7644E654B306800931F4610F081
:100C2000F3FA4FF07C5110F043FB10F007FD3F68E2
:100C30003060A5E7384610F0E7FA604910F038FB5D
:100C40008346284610F0E0FA5D4910F031FB01467A
:100C5000584610F025FA10F0F1FC009B074618608A
:100C60005849594A08881288D9F80010574DC0EBE6
:100C7000070EC3199142C8F800E0CAF80030B5F871
:100C800000E080F2F6800025C2EB0E0C3F4B64457D
:100C90001F6880F2E280631C974205FB03F50CF1AC
:100CA000010C95FBFCF5C0F28081BE45A8BFBE4695
:100CB000C2EB0E0E03FB0EF494FBFCF4914200F326
:100CC000B780BA42C0F2B480414D286810F09CFA57
:100CD000404910F0EDFA404910F0E2F910F0AEFC96
:100CE000A0F5FF531C3B082B98BF4FF4005033680E
:100CF000184400282860C0F2AE80B0F5804F80F222
:100D0000BF80364B1B781BB1B0F5005F40F0C08050
:100D1000334C2378002B40F0C380324C2B68226880
:100D20002B4D934221D0304E3278A3F50053013A37
:100D300003F30D03120203F5005302F4706218046A
:100D400042F4604242F00E0200F4FE005B0403F045
:100D5000FE43104318430EF08DFC317828680139AA
:100D6000C9B2FFF721FD2B68236007B0BDE8F08F03
:100D7000384610F049FA1D4910F09AFA8346284681
:100D800010F042FA1A4960E7A29EFF1FD09EFF1F93
:100D9000659DFF1FD09DFF1F4C8BFF1FFC8CFF1F0D
:100DA0000C8CFF1FFA9DFF1F889DFF1F949EFF1F45
:100DB000B08AFF1FBC9DFF1FD88AFF1FCDCC4C3FC0
:100DC000CDCC4C3EFE8CFF1F2C9EFF1FB89DFF1FFD
:100DD000988DFF1F9A99193FCDCC4C45B49EFF1FAB
:100DE000119EFF1F7889FF1F018DFF1F6666663FFA
:100DF000CDCCCC3DCC9DFF1FE09DFF1F309EFF1F43
:100E0000384610F001FA6A4910F052FA8346284633
:100E100010F0FAF9674918E7384610F0F5F9664915
:100E200010F046FA8346284610F0EEF963490CE7C5
:100E3000019B002B3FF448AF2B1B002BB8BF5B423C
:100E4000092B34DC33685E4D4FF400501844002801
:100E50002860BFF652AF002214E0974205FB04F56C
:100E6000B8BF002395FBFCF580F2968093FBFCF461
:100E700024E77145D4BFC2EB0105C2EB0E0503E7C1
:100E800043F6FF724F4B2A601B78002B3FF440AFB4
:100E900000210D200DF012FC4B4B01221A703CE793
:100EA00001210D200DF00AFC0023237035E705F524
:100EB00000500130001B10F0A7F93E49404D10F0E2
:100EC000F7F90446286810F09FF9394910F0F0F955
:100ED0000146204610F0E4F810F0B0FB07E73B4B6A
:100EE00000931F4630683A4B049310F08DF94FF091
:100EF0007C5110F0DDF9374A0290128803922046A7
:100F000010F082F9039A049B3F6853F8221010F006
:100F1000CFF910F093FBCBEB070BAB45CAEB0B0201
:100F2000B8BFAB46CAEB0B0B9042BABF00FB0BBB82
:100F3000013200FB0BFB9BFBF2F013E6244B049306
:100F4000224B306800931F4610F05EF94FF07C5141
:100F500010F0AEF91F49029009880391204610F065
:100F600053F9049B03993F6853F8211010F0A0F93E
:100F70000146002010F092F834E601200DF0CCFD7F
:100F8000154B1B689842D4BF002301238DE500FB5D
:100F90000BFB9BFBF1F038E67745D4BFC2EB0703B0
:100FA000C2EB0E0304FB03F360E7964680E600BF46
:100FB0009A99193FCDCCCC3E3333733FCDCC4C3DC9
:100FC000988DFF1FB49EFF1F119EFF1F949EFF1F51
:100FD000B08AFF1FBC9DFF1F988CFF1F30B58DB0DE
:100FE0006D460024E1B234480BF0E0F901340C2CDA
:100FF00045F8040BF6D1314B0A9A1B889A4216DA4F
:10100000009A934213DD029A934210DD049A9342B0
:101010000DDD2B4A2B4B11881B882B4A0B44126881
:101020005B10934238DB294A1268934201DB0DB012
:1010300030BD274B00241C70FFF740FB21460D20DC
:101040000DF03CFB32200DF075FB01210D200DF061
:1010500035FB32200DF06EFB21460D200DF02EFBEE
:1010600032200DF067FB01210D200DF027FB32200F
:101070000DF060FB21460D200DF020FB32200DF01D
:1010800059FB0D2001210DF019FB4FF42F700DB00D
:10109000BDE830400DF04EBB0D4B002101240D206A
:1010A0001C700DF00BFB32200DF044FB0D2021468F
:1010B0000DF004FB3220EAE7109EFF1FC49EFF1FC5
:1010C000B89DFF1F2C9EFF1FCC9DFF1FD09EFF1FB2
:1010D000A89DFF1F2DE9F843B14DB24E286810F0CE
:1010E00093F8B14910F0E4F8044610200DF014FD17
:1010F00010F08AF8AD4910F0DBF821460FF0D0FF70
:1011000010F09CFA34882860002C53D0DFF8BC82A1
:10111000B8F8003098424DDBA5490F78024627B950
:101120000120042C087000F05381012C00F0CE80C7
:10113000022C00F07081032C49D19E4B1B88092B97
:1011400045D02B68B8F800409B4AA3421288C0F2F1
:10115000A2809342D4BFC4EB0303C4EB0203141B6D
:101160007E2CDFF86092D5BFC3EB8313C3EBC313B0
:101170005B00013493FBF4F4D9F800300134A3424E
:1011800014D08E4D8E4A2B78013B1B0203F4706302
:1011900020061A4300F0FE4010430EF06BFA2A7846
:1011A000013AD2B221464A20FFF70EFBC9F80040AF
:1011B000BDE8F8837E4B1A784AB10025012C1D70DA
:1011C00029D0022C47D0032C03D0042C65D0BDE8D5
:1011D000F883784B1B88092BF9D07A4C2368002BB5
:1011E000F5D0764E76483378013B1B0203F47063EA
:1011F00018430EF03FFA3078013860F04F00C0B26B
:101200000DF0F8FB4A200DF0F5FB28460DF0F2FB3F
:101210002560BDE8F8836B4E3368002BD7D0674F4D
:1012200038780138000200F4706040F4D83040F0A3
:101230000B000EF01FFA3878013860F04F00C0B292
:101240000DF0D8FB20460DF0D5FB28460DF0D2FB63
:101250003560BDE8F8835B4C2368002BB7D0574E50
:1012600030780138000200F4706040F4962040F0BD
:101270000B000EF0FFF93078013860F04F00C0B27B
:101280000DF0B8FB04200DF0B5FB28460DF0B2FBC5
:101290002560BDE8F883002361E7484C4A4823787D
:1012A000013B1B0203F4706318430EF0E3F920784E
:1012B000013860F04F00C0B20DF09CFB40200DF0F3
:1012C00099FB2846BDE8F8430DF094BB3A490988DC
:1012D0009142D4BFC3EB0107C3EB0207CB1A7E2BAD
:1012E00040F3A580C7EBC7125F1C92FBF7F70137ED
:1012F000DFF8D090D9F80030BB4216D02F4C2378BD
:10130000013B1B0203F4706343F4D833380643F007
:101310000B0300F0FE4018430EF0ACF92278013ABE
:10132000D2B239460120FFF74FFA3488C9F800706D
:10133000022C7FF400AF2B68B8F800701E4ABB4245
:1013400012886DDA0023D71B7E2FDFF87890D5BF87
:10135000C3EB8313C3EBC3135B00013793FBF7F7B6
:10136000D9F800300137BB4268D0144C2378013BD8
:101370001B0203F4706343F49623380643F00B0317
:1013800000F0FE4018430EF075F92278013AD2B20F
:1013900039460420FFF718FA3488C9F80070CAE605
:1013A000C09DFF1FC89DFF1F9A99193FCDCCCC3E11
:1013B000B09EFF1F689EFF1F429EFF1F018DFF1FF3
:1013C0000BB04A00289EFF1F0BB04000969DFF1FE8
:1013D0001B4C1C482378013B1B0203F47063184329
:1013E0000EF048F92078013860F04F00C0B20DF0DF
:1013F00001FB40200DF0FEFA7F200DF0FBFA34884F
:10140000012C95D12A68B8F800300F499A42098812
:10141000FFF664AF5CE70C4A2B681288B8F80070DE
:101420009A42D4BFC7EB0203C7EB03038BE7C7EBBA
:1014300087177F0097FBF3F7013759E70224ACE7E2
:10144000018DFF1F0BB0407F429EFF1F114B1B8879
:10145000022B03D0104B01221A70704710B50F4CAD
:101460000F482378013B1B0203F4706318430EF00E
:1014700001F92078013860F04F00C0B20DF0BAFADF
:1014800041200DF0B7FA7F200DF0B4FA024B012293
:101490001A7010BD209EFF1FE69DFF1F018DFF1FCC
:1014A0000BB0417F1B4A1C4B70B51B6814881B4A4C
:1014B000A342128826DA0023141B194D7F2CCABFC1
:1014C000DB01C3EBC313013493FBF4F42B68A34299
:1014D00016D0144E3378013B1B0203F4706343F4BF
:1014E000B623200643F00B0300F0FE4018430EF035
:1014F000C1F83278013AD2B221460520FFF764F9EB
:101500002C6070BD9342D4BFC4EB0303C4EB020351
:10151000D2E700BFE49DFF1F6C9DFF1FA09EFF1F31
:10152000B89EFF1F018DFF1F38B5204C236843B9BB
:101530001F4B1B88022B21D01E4A002313702360EF
:1015400038BD1D4D28780138000200F4706040F469
:10155000B62040F00B000EF08DF82878013860F0CE
:101560004F00C0B20DF046FA05200DF043FA0020FE
:101570000DF040FA0E4B1B88022BDDD10E4D0F48AB
:101580002B78013B1B0203F4706318430EF072F8D2
:101590002878013860F04F00C0B20DF02BFA4120DE
:1015A0000DF028FA00200DF025FAC5E7B89EFF1FC0
:1015B000209EFF1FE69DFF1F018DFF1F0BB0410006
:1015C00008B511200DF0A8FA0D4B0E4A1B881060CB
:1015D00053B10D4B1B88984206DB0C4B1B785BB15B
:1015E000BDE80840FFF75EBF084B1B7803B908BD94
:1015F000BDE80840FFF798BFFFF728FFF0E700BFFE
:10160000209EFF1F6C9DFF1FE49DFF1FE69DFF1F97
:101610002DE9F04F8FB002AD0024E1B26E480AF020
:10162000C5FE01340C2C45F8040BF6D16B4B6C4C09
:10163000B3F800E00A9B00227345227014DB089B7C
:101640009E4500F3B480069B664A9E4503DD1378F1
:10165000002B40F0BC80049B9E4540F3AE804FF0D1
:10166000020C84F800C009E0069B5E4A9E45CCBF90
:101670004FF0060C4FF0050C84F800C00C9F039E41
:101680000598079982F800C0BE45D4BF00270127FE
:10169000B645D4BF002601268645099ADFF8708139
:1016A0000B9B0D9DDFF86CA1DFF86C918AF8006050
:1016B000D4BF002001208E45D4BF0021012188F82D
:1016C000001096454849DFF854B1484E89F80000AB
:1016D000D4BF002201229E45D4BF002301230A70FB
:1016E000AE45434A8BF80070D4BF00250125012088
:1016F000137035700DF010FA3E4B3F4A1D6811888B
:101700003E4BA842D4BF002201220B291A7001D9F6
:101710000C2901D0A84246DC00230193384B9AF8EB
:1017200000E01F7899F800C098F800209BF800307E
:101730002D49DFF8ECA091F800902D49367891F80A
:1017400000802478A7EB4E07CCEB070CA2EB8202BB
:10175000C3EB83776244C3EB8703134403EB490372
:10176000BAF80020274FDFF8BCE0B7F800C0264FDA
:10177000434403EB8606033A0C2313FB046602EB97
:10178000420206EB8202019BCEF800606244A8424E
:10179000A2F10C021A44C8BF1C4B3A60C8BF1E70AD
:1017A0000FB0BDE8F08FA1F10C030193B6E74FF045
:1017B000040C84F800C00B4A60E7029B9E45C6BF3C
:1017C0004FF0010C84F800C04FF0000C56E74FF0CA
:1017D000030C84F800C051E7109EFF1FC49EFF1F3A
:1017E000389EFF1F449EFF1FA99EFF1F019FFF1FE2
:1017F000009FFF1F988CFF1FA29EFF1F9C9DFF1F35
:10180000008DFF1F869DFF1FC89EFF1FC69EFF1FE6
:10181000FD9EFF1F989EFF1FFC9EFF1FFE9EFF1F49
:101820008C9EFF1FF49DFF1F10B500EBC000821DB2
:10183000D2B293B284B09C1E981C3D2303918DE8D4
:101840001900392102480BF043F904B010BD00BF64
:10185000D49EFF1F70B50E4C84B0122504220123C4
:1018600006460390029320468DE82400142310219D
:101870000BF02EF9062209230293039601952046C8
:101880000092142310210BF023F904B070BD00BFA7
:10189000D49EFF1F10B50C4C81B220460BF0FAFB12
:1018A000204602210BF0F0FB204621225A210BF0AA
:1018B000E7FB064B204619880EF00EFA2046BDE8DD
:1018C00010400EF0B9B900BFD49EFF1FFC8CFF1F63
:1018D00010B50C4C81B220460BF0DCFB20460221F7
:1018E0000BF0D2FB204621225A210BF0C9FB064BFC
:1018F000204619880EF0F0F92046BDE810400EF0A1
:101900009BB900BFD49EFF1FD88AFF1F10B50C4C97
:1019100081B220460BF0BEFB204602210BF0B4FB47
:101920002046212253210BF0ABFB064B20461988A1
:101930000EF0D2F92046BDE810400EF07DB900BF90
:10194000D49EFF1FFE8CFF1F38B50C460546C9B25A
:101950000CF0E6FB210A681CBDE838400CF0E0BB47
:1019600038B505460CF0C2FB4FF0000460F30704E5
:10197000681C0CF0BBFB60F30F24A0B238BD00BFA5
:1019800008B50CF06BFB042103480BF019FE03486B
:10199000BDE808400AF0A2BCD49EFF1F109EFF1FA6
:1019A00000B5244B1A7883B00121052302B300222D
:1019B00001910093114620480AF09EFF1F4B1A78B0
:1019C00002B3052301220192009300220A211A4842
:1019D0000AF092FF1A4B1A7802BB052301210191EC
:1019E0000093142114480BF009F803B05DF804FBD0
:1019F00001910093114610480BF000F80F4B1A7834
:101A0000002ADED105230121019100930A210A4811
:101A10000AF0F4FF0A4B1A78002ADED005230122CF
:101A2000019200930022142103480AF065FF03B0DD
:101A30005DF804FBA99EFF1FD49EFF1F009FFF1FA0
:101A4000019FFF1F2DE9F04FC54D2B78A3F10A022E
:101A5000022A83B040F22281C24EA3F11402022A6C
:101A60003CD8DFF83083C04AD8F800E01268BF499C
:101A70009645D1F8009080F20E82C2EB090CBCF1C1
:101A80005A0F4FF00004BA4F40F31282D7F800A06B
:101A90005B2052450CF1010100FB04F494FBF1F4CE
:101AA00004F11C0440F3E882002292FBF1F11C31A6
:101AB000A14200F0158209B200232622AD480BF0A6
:101AC00011FD21B201232622AA480BF00BFDA948E3
:101AD0000BF030FFD8F800202B783A60A3F11E02FB
:101AE000022A00F28B80A44FDFF8ACA23968DAF842
:101AF0000030DFF8A8929942D9F8002080F25A818C
:101B0000D01A5A284FF00004DFF8948240F35E8127
:101B1000D8F800104FF05B0E8B420EFB04F400F17E
:101B2000010E94FBFEF404F11C0400F3B98291420F
:101B3000A8BF1146C3EB010C5B2101FB0CF191FB2B
:101B4000FEF11C31A14200F0548109B2002326228B
:101B500088480BF0C7FC21B20123262285480BF0F0
:101B6000C1FCDAF80030DFF83CA2D9F80020DAF83E
:101B7000001099424FF0010CA2EB0300C0F2448127
:101B80009142D4BFC3EB0104C3EB02045A28DFF82F
:101B9000189240F34081D9F800B000F1010E5B4586
:101BA0004FF05B0000FB04F494FBFEF404F11C0412
:101BB00000F378825A45A8BF5A46D21A5B2000FB30
:101BC00002F090FBFEF01C30A04200F0398101B21F
:101BD0000023262267480BF085FC21B20123262230
:101BE00064480BF07FFC63480BF0A4FEDAF80010A9
:101BF0003A682B78C8F80020C9F80010A3F1280231
:101C0000022A42D8DFF8A4815C4AD8F800E01268C2
:101C10005B499645D1F800C080F21A81C2EB0C01F5
:101C20005A294FF00004574F40F31E8138684FF097
:101C30005B09824201F1010109FB04F494FBF1F418
:101C400004F11C0400F316828445A8BF8446C2EB4D
:101C50000C0C5B2000FB0CF090FBF1F11C31A1425D
:101C600000F0158109B20023262242480BF03AFC0D
:101C700021B2012326223F480BF034FC3D480BF0F3
:101C800059FED8F800202B783A603C3B012B40F2FB
:101C90003A810023337003B0BDE8F08F3A4ADFF891
:101CA00010811668D8F800E0384AB645126834DA70
:101CB000911B5A294FF00004354F38DD38684FF03A
:101CC0005B0C864201F101010CFB04F494FBF1F47E
:101CD00004F11C0400F3E8819042A8BF1046861B63
:101CE0005B2000FB06F090FBF1F11C31A14230D0EB
:101CF00009B2002326221F481A4E0BF0F3FB21B233
:101D0000012326221B480BF0EDFB1A480BF012FEB4
:101D1000D8F800202B783A609FE6911B9645D4BFF7
:101D2000C6EB0E04C6EB02045A29194FC6DCD7F8DD
:101D300000C05A20664500FB04F494FBF1F404F162
:101D40001C0440F3BC81002292FBF1F11C31A14242
:101D5000CED1044E3278002A40F0D3807246DAE7C2
:101D60000E9EFF1F749DFF1FAC8AFF1FE48DFF1F97
:101D7000509EFF1FD49EFF1FCC9DFF1FFC8DFF1F99
:101D8000A08AFF1F7C9EFF1FF09DFF1F9C8AFF1FE4
:101D9000A49EFF1F6C9DFF1FE88DFF1F808BFF1F00
:101DA000D49DFF1FD09EFF1F049FFF1FC09DFF1FDC
:101DB000889EFF1FD01A9142D4BFC3EB0104C3EB2E
:101DC00002045A28DFF824833FF7A2AED8F800E0D7
:101DD0005A21734501FB04F494FBF0F404F11C0454
:101DE00040F36481002191FBF0F11C31A1427FF4AA
:101DF000ACAE3478002C77D1DFF8F4A2DAF800101A
:101E00009942A446BFF6BCAE5A284FF00004DFF852
:101E1000E4923FF7C0AED9F800E04FF05A0B73459B
:101E20000BFB04F494FBF0F404F11C0440F319815F
:101E30004FF0000B9BFBF0F01C30A0427FF4C7AECC
:101E40003378002B56D1BCF1000F3FF4D1AECAE677
:101E5000C2EB0C01E645D4BFC2EB0E04C2EB0C048E
:101E60005A299B4F3FF7E2AED7F800905A204A45D7
:101E700000FB04F494FBF1F404F11C0440F307812B
:101E8000002292FBF1F11C31A1427FF4EBAE3278DB
:101E900072BB7246F8E6C2EB090CCE45D4BFC2EB6A
:101EA0000E04C2EB0904BCF15A0F8A4F3FF7EEADA6
:101EB00039685A208A4200FB04F494FBFCF404F1D4
:101EC0001C0400F3E2804945A8BF4946891A5A20FC
:101ED00000FB01F090FBFCF11C31A1427FF4EBAD63
:101EE00032781AB97246F8E509B235E609B2E9E581
:101EF00009B2BEE601B20123262277480BF0F2FABE
:101F000071E609B2FCE6262200248DE8140076234F
:101F10001C217148714D724F0AF020FD1DE0824274
:101F2000D4BFC3EB0201C3EB0001D31A4FF05A0E2A
:101F300073454FF05B00CABF41430EFB01F1013313
:101F400091FBF3F303F11C0101231C44262209B287
:101F500061480BF0C7FA0C2C09D0E1B261480AF0D5
:101F600025FA2B683A688342D9DD0021DDE7DFF8E6
:101F700088815D4C01200CF0CFFDD8F800C02368AB
:101F80003A682968CCEB030E8B1A9E45CCEB000017
:101F90005BDD03FB00000EF1010390FBF3F3134440
:101FA00099424EDC9A42D4BFC1EB0203C1EB03035A
:101FB000521A5A2ACABF5B215A21013201FB03F38C
:101FC00093FBF2F202F11C0109B2012326224248DE
:101FD0000BF088FA00200CF09FFDD8F800E03A687A
:101FE000296824688B1ACEEB04049C42CEEB0000D7
:101FF00031DD03FB0000631C90FBF3F313449942B3
:1020000021DC9A42D4BFC1EB0203C1EB0303521A95
:102010005A2ACABF5B215A21013201FB03F393FB09
:10202000F2F202F11C0109B2012326222A480BF028
:1020300059FA29480BF07EFC0023337003B0BDE849
:10204000F08F0023B4E70023E1E703FB00F393FBE9
:10205000FEF31344A4E703FB00F393FBF4F31344F0
:10206000CDE77245D4BFC3EB0203C3EB0E030BFBFA
:1020700003FBDFE69446EAE5D145D4BFC2EB090293
:10208000C2EB0A0200FB02F20FE511461EE7CC4547
:10209000D4BFC2EB0C02C2EB090200FB02F2F0E675
:1020A000194647E51A4688E5304618E67245D4BF1A
:1020B000C3EB020EC3EB0E0E01FB0EF193E662457D
:1020C000D4BFC6EB0202C6EB0C0200FB02F23BE6F9
:1020D0007C9EFF1F509EFF1FD49EFF1FF48DFF1F8D
:1020E000848CFF1F109EFF1FA08CFF1FD49DFF1F1D
:1020F000D09EFF1F049FFF1FA48AFF1F08B581B257
:1021000017480AF0C7FF022115480AF0BDFF212237
:102110005A2113480AF0B4FF124B114819880DF0E8
:10212000DBFD0F480DF088FD0F4B197891B90C4875
:102130000AF0B0FF01210A480AF0A6FF33227421F9
:1021400007480AF09DFF012208490548BDE80840FC
:102150000DF05EBD012102480AF09CFFEAE700BFD6
:10216000D49EFF1F549EFF1F2F9EFF1FCC200100F7
:1021700070B5194C82B03426002301252046019306
:10218000009640230B223F210AF0B6FB40230B228E
:102190002046009601953F210AF030FC2946204652
:1021A0000AF078FF294620460AF06EFF20460F22EB
:1021B00044210AF065FF0922084920460DF028FD58
:1021C00020460DF039FD064B20461D7002B0BDE8DB
:1021D00070400BF0AFBB00BFD49EFF1FC4200100B6
:1021E000CC9EFF1F70B5194C82B034260023012508
:1021F00020460193009640230B223F210AF07CFBEE
:1022000040230B222046009601953F210AF0F6FB61
:10221000294620460AF03EFF294620460AF034FFB0
:1022200020460F2251210AF02BFF052208492046A3
:102230000DF0EEFC20460DF0FFFC2846FFF766FB94
:10224000204602B0BDE870400BF074BBD49EFF1F67
:10225000D020010070B5194C82B03426002301252E
:1022600020460193009640230B223F210AF044FBB5
:1022700040230B222046009601953F210AF0BEFB29
:10228000294620460AF006FF294620460AF0FCFEB1
:1022900020460F2251210AF0F3FE0522084920466C
:1022A0000DF0B6FC20460DF0C7FC2846FFF7F2FA09
:1022B000204602B0BDE870400BF03CBBD49EFF1F2F
:1022C000D020010070B5194C82B0342600230125BE
:1022D00020460193009640230B223F210AF00CFB7D
:1022E00040230B222046009601953F210AF086FBF1
:1022F000294620460AF0CEFE294620460AF0C4FEB2
:1023000020460F2251210AF0BBFE05220849204633
:102310000DF07EFC20460DF08FFC2846FFF7D8FA22
:10232000204602B0BDE870400BF004BBD49EFF1FF6
:10233000D020010070B5194C82B03426002301254D
:1023400020460193009640230B223F210AF0D4FA45
:1023500040230B222046009601953F210AF04EFBB8
:10236000294620460AF096FE294620460AF08CFEB1
:1023700020460F2244210AF083FE09220849204604
:102380000DF046FC20460DF057FC2846FFF7B6FE40
:10239000204602B0BDE870400BF0CCBAD49EFF1FBF
:1023A000D820010008B581B210480AF073FE02215E
:1023B0000E480AF069FE4F2121220C480AF060FE07
:1023C0000B4B198849B903220A4908480DF020FC33
:1023D0000648BDE808400DF02FBC04480DF07CFC19
:1023E0000248BDE808400DF027BC00BFD49EFF1F87
:1023F0005C9DFF1FE420010070B5194C82B03426AB
:102400000023012520460193009640230B223F2103
:102410000AF072FA40230B222046009601953F21D4
:102420000AF0ECFA294620460AF034FE29462046F6
:102430000AF02AFE20460F2247210AF021FE082238
:10244000084920460DF0E4FB20460DF0F5FB284638
:10245000FFF7A8FF204602B0BDE870400BF06ABA53
:10246000D49EFF1FE820010010B581B2124C134822
:102470000AF010FE022111480AF006FE23882122EC
:102480006BB94F210D480AF0FBFD03220C490B48A4
:102490000DF0BEFB0948BDE810400DF0CDBB5A2140
:1024A00006480AF0EDFD218804480DF015FC0348AC
:1024B000BDE810400DF0C0BB689DFF1FD49EFF1FFC
:1024C000F420010070B5194C82B034260023012598
:1024D00020460193009640230B223F210AF00CFA7C
:1024E00040230B222046009601953F210AF086FAF0
:1024F000294620460AF0CEFD294620460AF0C4FDB2
:1025000020460F2248210AF0BBFD08220849204638
:102510000DF07EFB20460DF08FFB2846FFF7A4FF51
:10252000204602B0BDE870400BF004BAD49EFF1FF5
:10253000F820010010B581B2124C13480AF0AAFD30
:10254000022111480AF0A0FD238821226BB94F21F6
:102550000D480AF095FD03220C490B480DF058FB7D
:102560000948BDE810400DF067BB5A2106480AF043
:1025700087FD218804480DF0AFFB0348BDE81040FB
:102580000DF05ABBBC9DFF1FD49EFF1FF42001001D
:1025900070B5194C82B034260023012520460193E2
:1025A000009640230B223F210AF0A6F940230B227C
:1025B0002046009601953F210AF020FA2946204640
:1025C0000AF068FD294620460AF05EFD20460F22EB
:1025D00051210AF055FD0522084920460DF018FB4F
:1025E00020460DF029FB2846FFF7A4FF204602B045
:1025F000BDE870400BF09EB9D49EFF1FD0200100B3
:1026000010B581B21748184C0AF044FD0221154854
:102610000AF03AFD21224C2112480AF031FD2388AC
:102620004BB9032211490F480DF0F2FA0D48BDE8ED
:1026300010400DF001BB02220D490A480DF0E8FAE6
:1026400008480DF0F9FA2122652106480AF018FD24
:10265000218804480DF040FB0248BDE810400DF011
:10266000EBBA00BFD49EFF1FD09DFF1FF4200100D6
:102670000421010070B5194C82B0342600230125D5
:1026800020460193009640230B223F210AF034F9A3
:1026900040230B222046009601953F210AF0AEF917
:1026A000294620460AF0F6FC294620460AF0ECFCB2
:1026B00020460F2244210AF0E3FC09220849204663
:1026C0000DF0A6FA20460DF0B7FA2846FFF798FF5E
:1026D000204602B0BDE870400BF02CB9D49EFF1F1D
:1026E0000821010010B50C4681B219480AF0D2FC4D
:1026F000022117480AF0C8FC2122502114480AF090
:10270000BFFC002C4FF0010214DB124910480DF001
:102710007FFA0F480DF090FA5D2121220C480AF053
:10272000AFFC21460A480DF0D7FA0948BDE8104031
:102730000DF082BA084906480DF06AFA04480DF017
:102740007BFA5D21212202480AF09AFC6142E9E706
:10275000D49EFF1F142101001821010010B581B281
:102760002048214C0AF096FC02211E480AF08CFCFD
:10277000212250211B480AF083FC2388022B4FF0B2
:10278000010218DC194917480DF042FA15480DF0FE
:1027900053FA21225D2113480AF072FC2188114866
:1027A00003390029B8BF49420DF096FA0D48BDE83B
:1027B00010400DF041BA0E490A480DF029FA0948B7
:1027C0000DF03AFA21225D2106480AF059FC2188D1
:1027D000044803390DF080FA0248BDE810400DF0BE
:1027E0002BBA00BFD49EFF1F8C9EFF1F1821010033
:1027F0001421010070B5194C82B034260023012544
:1028000020460193009640230B223F210AF074F8E2
:1028100040230B222046009601953F210AF0EEF856
:10282000294620460AF036FC294620460AF02CFCB0
:1028300020460F224D210AF023FC0622084920469B
:102840000DF0E6F920460DF0F7F92846FFF786FF70
:10285000204602B0BDE870400BF06CB8D49EFF1F5C
:102860001C21010010B581B22048214C0AF012FC55
:1028700002211E480AF008FC212250211B480AF0C0
:10288000FFFB23880B2B4FF0010218DC1949174876
:102890000DF0BEF915480DF0CFF921225D21134846
:1028A0000AF0EEFB218811480C390029B8BF4942D3
:1028B0000DF012FA0D48BDE810400DF0BDB90E49FB
:1028C0000A480DF0A5F909480DF0B6F921225D215D
:1028D00006480AF0D5FB218804480C390DF0FCF9B4
:1028E0000248BDE810400DF0A7B900BFD49EFF1FFD
:1028F000869DFF1F182101001421010070B5194C9D
:1029000082B03426002301252046019300964023FF
:102910000B223F2109F0F0FF40230B2220460096B6
:1029200001953F210AF06AF8294620460AF0B2FBD9
:10293000294620460AF0A8FB20460F2244210AF02F
:102940009FFB0922084920460DF062F920460DF050
:1029500073F92846FFF786FF204602B0BDE87040B5
:102960000AF0E8BFD49EFF1F2421010000B5324BBE
:102970001B78013B85B0052B0AD8DFE803F00C215A
:10298000364B54032D492E4B5A20012208701A70E1
:1029900005B05DF804FB01232A4A19461846137056
:1029A000FEF742FF28480AF0C5FF284A284B126864
:1029B0000192019A1A60FFF7A1FF05B05DF804FBD0
:1029C0000123244A194602201370FEF72DFF1E48EA
:1029D0000AF0B0FF1D4A1E4B12680292029A1A605A
:1029E000FFF708FF05B05DF804FB01231A4A1946FA
:1029F00003201370FEF718FF13480AF09BFF134AD9
:102A0000134B12680392039A1A60FFF793FC05B008
:102A10005DF804FB09490A4B0A20012208701A706C
:102A200005B05DF804FB0549054B502001220870F4
:102A30001A7005B05DF804FB3289FF1F0E9EFF1F60
:102A40009C8CFF1F809EFF1FD49EFF1F109FFF1FA7
:102A5000349EFF1FB09DFF1FDC9DFF1F08B581B294
:102A60000D480AF017FB02210B480AF00DFB21224A
:102A70004F2109480AF004FB084B1B88032243B18D
:102A8000074905480DF0C4F80348BDE808400DF0BB
:102A9000D3B80449F5E700BFD49EFF1FFA9DFF1F7E
:102AA000342101003021010070B5194C82B0342668
:102AB0000023012520460193009640230B223F214D
:102AC00009F01AFF40230B222046009601953F2172
:102AD00009F094FF294620460AF0DCFA29462046F0
:102AE0000AF0D2FA20460F2244210AF0C9FA09223C
:102AF000084920460DF08CF820460DF09DF8284638
:102B0000FFF7ACFF204602B0BDE870400AF012BFEC
:102B1000D49EFF1F3821010000B53A4B1B78013BC2
:102B200087B0042B16D8DFE803F0182D42570300B6
:102B30000123354A194605201370FEF775FE334808
:102B40000AF0F8FE324A334B12680592059A1A6071
:102B5000FFF7AAFF07B05DF804FB01232E4A1946D0
:102B600018461370FEF760FE28480AF0E3FE284A74
:102B7000284B12680192019A1A60FFF709FD07B00D
:102B80005DF804FB0123254A194602201370FEF765
:102B90004BFE1E480AF0CEFE1D4A1E4B12680292E2
:102BA000029A1A60FFF756FB07B05DF804FB012399
:102BB0001B4A194603201370FEF736FE13480AF02D
:102BC000B9FE134A134B12680392039A1A60FFF777
:102BD00079FB07B05DF804FB0123124A1946042073
:102BE0001370FEF721FE09480AF0A4FE084A094BBB
:102BF00012680492049A1A60FFF7F4FA07B05DF8BD
:102C000004FB00BF8C8AFF1FB59EFF1FD49EFF1FD1
:102C1000109FFF1F349EFF1F2E9EFF1F049EFF1F4D
:102C2000DD9DFF1FB49EFF1F08B581B20D480AF05D
:102C300031FA02210B480AF027FA21224F210948D4
:102C40000AF01EFA084B1B88032243B907490548BE
:102C50000CF0DEFF0348BDE808400CF0EDBF04496E
:102C6000F5E700BFD49EFF1FC69DFF1F482101004E
:102C70004421010070B5194C82B03426002301258F
:102C800020460193009640230B223F2109F034FE99
:102C900040230B222046009601953F2109F0AEFE0D
:102CA000294620460AF0F6F9294620460AF0ECF9B2
:102CB00020460F2244210AF0E3F909220849204660
:102CC0000CF0A6FF20460CF0B7FF2846FFF7ACFF3C
:102CD000204602B0BDE870400AF02CBED49EFF1F13
:102CE0004C21010000B5444B1B78013B87B0052BFC
:102CF00016D8DFE803F0182D42576C0301233F4A32
:102D0000194606201370FEF78FFD3D480AF012FEAB
:102D10003C4A3D4B12680592059A1A60FFF7AAFFDC
:102D200007B05DF804FB0123384A194618461370B2
:102D3000FEF77AFD32480AF0FDFD324A324B126846
:102D40000092009A1A60FFF713FA07B05DF804FBCF
:102D500001232F4A194602201370FEF765FD28480B
:102D60000AF0E8FD274A284B12680192019A1A607E
:102D7000FFF7FEF907B05DF804FB254B02220121A5
:102D800003201A70FEF750FD1D480AF0D3FD1D4ABE
:102D90001D4B12680292029A1A60FFF7E9F907B018
:102DA0005DF804FB1A4B0322012104201A70FEF780
:102DB0003BFD13480AF0BEFD124A134B1268039202
:102DC000039A1A60FFF7D4F907B05DF804FB104BC3
:102DD0000422012105201A70FEF726FD08480AF09A
:102DE000A9FD084A084B12680492049A1A60FFF77A
:102DF000BFF907B05DF804FB948DFF1F4C9EFF1FC9
:102E0000D49EFF1F109FFF1F349EFF1F399EFF1F80
:102E1000B79EFF1F08B581B20D480AF03BF90221A9
:102E20000B480AF031F921224F2109480AF028F90C
:102E3000084B1B884BB90849032205480CF0E8FEF3
:102E40000348BDE808400CF0F7BE02220349F4E74E
:102E5000D49EFF1F129EFF1FF42001005821010085
:102E600070B5194C82B03426002301252046019309
:102E7000009640230B223F2109F03EFD40230B2208
:102E80002046009601953F2109F0B8FD29462046CD
:102E90000AF000F9294620460AF0F6F820460F22EB
:102EA00044210AF0EDF80922084920460CF0B0FE52
:102EB00020460CF0C1FE2846FFF7ACFF204602B0CA
:102EC000BDE870400AF036BDD49EFF1F5C210100B2
:102ED00030B53C4C83B020460AF08AFB20460121E5
:102EE0000AF0D2F8204601210AF0D4F80022204648
:102EF00011460AF0C5F80722334920460CF088FE37
:102F000020460CF099FE09250123204601932A460C
:102F10007F230095002109F021FD20460C2200218D
:102F20000AF0AEF80522294920460CF071FE204631
:102F30000CF082FE2046152200210AF0A1F805229D
:102F4000234920460CF064FE20460CF075FE204616
:102F50001E2200210AF094F806221E4920460CF099
:102F600057FE20460CF068FE2046272200210AF07A
:102F700087F80722184920460CF04AFE20460CF03C
:102F80005BFE2046302200210AF07AF82A461349D7
:102F900020460CF03DFE20460CF04EFE2046392225
:102FA00000210AF06DF800220D4920460CF030FE99
:102FB00020460CF041FE204603B0BDE830400AF048
:102FC000B9BC00BFD49EFF1F682101007021010021
:102FD00078210100802101008821010038210100B1
:102FE0006C22010030B53C4C83B020460AF000FB57
:102FF000204601210AF048F8204601210AF04AF84B
:103000000022204611460AF03BF80C2233492046A4
:103010000CF0FEFD20460CF00FFE09250123204692
:1030200001932A467F230095002109F097FC204652
:103030000C2200210AF024F82A46294920460CF0E7
:10304000E7FD20460CF0F8FD2046152200210AF08D
:1030500017F82A46234920460CF0DAFD20460CF0EA
:10306000EBFD20461E2200210AF00AF808221E4924
:1030700020460CF0CDFD20460CF0DEFD2046272238
:10308000002109F0FDFF0522184920460CF0C0FD83
:1030900020460CF0D1FD20463022002109F0F0FF3F
:1030A0002A46134920460CF0B3FD20460CF0C4FD1F
:1030B00020463922002109F0E3FF08220D4920466D
:1030C0000CF0A6FD20460CF0B7FD204603B0BDE88D
:1030D00030400AF02FBC00BFD49EFF1F902101009A
:1030E000A02101005C210100E8200100AC210100C9
:1030F000B4210100F820010030B53C4C83B02046DB
:103100000AF076FA2046012109F0BEFF204601218F
:1031100009F0C0FF00222046114609F0B1FF0B2242
:10312000334920460CF074FD20460CF085FD09253E
:103130000123204601932A467F230095002109F0B0
:103140000DFC20460C22002109F09AFF0822294993
:1031500020460CF05DFD20460CF06EFD2046152249
:10316000002109F08DFF2A46234920460CF050FD2E
:1031700020460CF061FD20461E22002109F080FF50
:103180002A461E4920460CF043FD20460CF054FD13
:1031900020462722002109F073FF07221849204604
:1031A0000CF036FD20460CF047FD20463022002171
:1031B00009F066FF0822134920460CF029FD20463D
:1031C0000CF03AFD20463922002109F059FF2A4629
:1031D0000D4920460CF01CFD20460CF02DFD20462C
:1031E00003B0BDE830400AF0A5BB00BFD49EFF1F6E
:1031F000C0210100CC21010008210100D8210100DB
:1032000068210100E4210100F021010030B53C4CAF
:1032100083B020460AF0ECF92046012109F034FF82
:103220002046012109F036FF00222046114609F010
:1032300027FF20460D2233490CF0EAFC0125092224
:103240007F2320468DE82400002109F087FB2046DB
:103250000C22002109F014FF08222B4920460CF013
:10326000D7FC20460CF0E8FC20461522002109F08E
:1032700007FF0822254920460CF0CAFC20460CF026
:10328000DBFC20461E22002109F0FAFE082220491C
:1032900020460CF0BDFC20460CF0CEFC2046272238
:1032A000002109F0EDFE08221A4920460CF0B0FC7E
:1032B00020460CF0C1FC20463022002109F0E0FE3F
:1032C0000822154920460CF0A3FC20460CF0B4FC63
:1032D00020463922002109F0D3FE08220F4920465A
:1032E0000CF096FC20460CF0A7FC0D4B29461878F4
:1032F000FEF79AFA204603B0BDE830400AF01ABB48
:10330000D49EFF1FFC2101000C22010018220100A5
:1033100024220100302201003C2201004822010049
:10332000948DFF1F08B581B2154809F0B3FE022144
:10333000134809F0A9FE4F212122114809F0A0FEEF
:10334000104B198849B9104903220D480CF060FC54
:103350000B48BDE808400CF06FBC09480CF0BCFC01
:1033600007480CF069FC28226921054809F088FE0D
:103370000121034809F088FE02220449E5E700BF65
:10338000D49EFF1FB29EFF1FF420010054220100B3
:1033900070B5194C82B034260023012520460193D4
:1033A000009640230B223F2109F0A6FA40230B226E
:1033B0002046009601953F2109F020FB2946204632
:1033C00009F068FE2946204609F05EFE20460F22DD
:1033D000472109F055FE0822084920460CF018FC48
:1033E00020460CF029FC2846FFF79CFF204602B03F
:1033F000BDE870400AF09EBAD49EFF1FE421010090
:1034000008B581B2154809F045FE0221134809F0BC
:103410003BFE4F212122114809F032FE104B198842
:1034200049B9104903220D480CF0F2FB0B48BDE8E6
:1034300008400CF001BC09480CF04EFC07480CF0A9
:10344000FBFB28226921054809F01AFE01210348E7
:1034500009F01AFE02220449E5E700BFD49EFF1FCF
:103460000C9EFF1FF42001005422010070B5194C7E
:1034700082B0342600230125204601930096402384
:103480000B223F2109F038FA40230B2220460096F8
:1034900001953F2109F0B2FA2946204609F0FAFDCC
:1034A0002946204609F0F0FD20460F22452109F06B
:1034B000E7FD0922084920460CF0AAFB20460CF043
:1034C000BBFB2846FFF79CFF204602B0BDE87040DA
:1034D0000AF030BAD49EFF1FB421010030B55A481B
:1034E00083B00AF085F80121574809F0CDFD01218C
:1034F000554809F0CFFD00221146534809F0C0FDA0
:103500000D22524950480CF083FB23200AF00AFD9B
:1035100040F6B833984204464FF0040240F38480EA
:103520004B4949480CF074FB04EB4404494804EB54
:10353000041480FB0430E417C4EB60200DF064FE3B
:1035400045490DF0B5FE0DF009FA012402460B467F
:1035500000943D480CF0C8FB224640493A480CF024
:1035600057FB092401257F2322468DE830000021E6
:10357000354809F0F3F90C220021334809F080FDA9
:103580002246374930480CF043FB2F480CF054FBDF
:10359000152200212C4809F073FD062231492A48E2
:1035A0000CF036FB28480CF047FB1E220021264871
:1035B00009F066FD07222C4923480CF029FB22481C
:1035C0000CF03AFB272200211F4809F059FD062282
:1035D00026491D480CF01CFB1B480CF02DFB30222B
:1035E0000021194809F04CFD0822214916480CF029
:1035F0000FFB15480CF020FB39220021124809F07E
:103600003FFD22461B4910480CF002FB0E480CF00F
:1036100013FB194B29461878FEF706F90A4803B040
:10362000BDE830400AF086B9144907480CF0F0FABA
:1036300040F6F5039C423FF777AF0322104902485A
:103640000CF0E6FA8DE700BFD49EFF1F5822010060
:1036500068220100976A3E2BCDCCCC3D7C22010034
:10366000242101001C210100802201008822010088
:10367000902201009C2201003289FF1F702201006C
:103680007822010030B5544883B009F0B1FF012120
:10369000514809F0F9FC01214F4809F0FBFC0222D6
:1036A00019214D4809F0ECFC0B224C494A480CF01A
:1036B000AFFA49480CF0C0FA14220021464809F03C
:1036C000DFFC0322464944480CF0A2FA4248012498
:1036D0000CF0B2FA11228DE81400782319213E482B
:1036E00009F03CF9132519231946009512223A488E
:1036F000019409F033F978231946009512223648CF
:10370000019409F02BF91D228DE81400782319216A
:10371000314809F023F91C251923194600951B226D
:103720002D48019409F01AF97823194600951B22B7
:103730002948019409F012F923220021264809F0B2
:103740009FFC0322274924480CF062FA22480CF01F
:1037500073FA28251923194624221F48019400953D
:1037600009F0FCF8782319462422019400951A48A0
:1037700009F0F4F81C4A1D4B11681B681C4A5B1ABF
:103780005C2B12881DDC511A5C2202FB01F292FBB9
:10379000F3F31B33174A1048136001241BB21A229B
:1037A00019468DE81400142209F0D8F8124B20466F
:1037B0001C70FEF74FF8084803B0BDE830400AF02F
:1037C000B9B8521A02EB4202C2EB4212234492FBF6
:1037D000F3F31B33DEE700BFD49EFF1FA8220100D6
:1037E000B4220100B8220100F48DFF1F848CFF1F5A
:1037F000C49EFF1F609DFF1F629EFF1FF0B585489E
:10380000854E864D83B009F0F3FE0121814809F011
:103810003BFC01217F4809F03DFC022219217D4833
:1038200009F02EFC10227E497A480CF0F1F9794813
:103830000CF002FA14220021764809F021FC032240
:10384000784974480CF0E4F9724801240CF0F4F95A
:1038500011228DE81400782319216E4809F07EF8B2
:10386000132719231946009712226A48019409F078
:1038700075F878231946009712226648019409F0DA
:103880006DF81D228DE8140078231921614809F094
:1038900065F81C271923194600971B225D480194DF
:1038A00009F05CF87823194600971B2259480194C7
:1038B00009F054F823220021564809F0E1FB0322C5
:1038C000594954480CF0A4F952480CF0B5F928278E
:1038D00019231946009724224E48019409F03EF816
:1038E00078231946009724224A48019409F036F8B3
:1038F00032220021474809F0C3FB03224B494548C7
:103900000CF086F943480CF097F92F228DE814004B
:10391000782319213F4809F021F831271923194646
:10392000009730223B48019409F018F87823194693
:10393000009730223748019409F010F83C228DE8B6
:10394000140078231921334809F008F83B2719237C
:1039500019463A222F480194009708F0FFFF782378
:1039600019463A22019400972A4808F0F7FF316877
:103970002B682F4A5B1A5C2B128839DD521A02EB36
:103980004202C2EB4212234492FBF3F31B33294A57
:103990002048136001241BB21A2219468DE8140036
:1039A000142208F0DBFF31682B682348234A047097
:1039B0005B1A5C2B128823DC511A5C2202FB01F299
:1039C00092FBF3F31B331E4A1248136001241BB20F
:1039D000392219468DE81400322208F0BFFF204634
:1039E000FDF738FF0B4803B0BDE8F04009F0A2BF77
:1039F000511A5C2202FB01F292FBF3F31B33C6E780
:103A0000521A02EB4202C2EB4212234492FBF3F33E
:103A10001B33D8E7D49EFF1FFC8DFF1FA08AFF1F1A
:103A2000BC220100B4220100B8220100D022010012
:103A3000969DFF1F609DFF1F629EFF1F429EFF1FFE
:103A4000849EFF1FF0B58548854E864D83B009F0F2
:103A5000CFFD0121814809F017FB01217F4809F0C2
:103A600019FB022219217D4809F00AFB06227E4932
:103A70007A480CF0CDF879480CF0DEF814220021D9
:103A8000764809F0FDFA0322784974480CF0C0F832
:103A9000724801240CF0D0F811228DE8140078232C
:103AA00019216E4808F05AFF132719231946009769
:103AB00012226A48019408F051FF782319460097B2
:103AC00012226648019408F049FF1D228DE8140077
:103AD00078231921614808F041FF1C271923194652
:103AE00000971B225D48019408F038FF782319469F
:103AF00000971B225948019408F030FF232200212F
:103B0000564809F0BDFA0322594954480CF080F890
:103B100052480CF091F828271923194600972422BF
:103B20004E48019408F01AFF782319460097242282
:103B30004A48019408F012FF32220021474809F058
:103B40009FFA03224B4945480CF062F843480CF0B9
:103B500073F82F228DE81400782319213F4808F0CC
:103B6000FDFE312719231946009730223B48019466
:103B700008F0F4FE78231946009730223748019464
:103B800008F0ECFE3C228DE814007823192133481C
:103B900008F0E4FE3B27192319463A222F480194E6
:103BA000009708F0DBFE782319463A22019400972B
:103BB0002A4808F0D3FE31682B682F4A5B1A5C2B29
:103BC000128839DD521A02EB4202C2EB4212234440
:103BD00092FBF3F31B33294A2048136001241BB2E4
:103BE0001A2219468DE81400142208F0B7FE316835
:103BF0002B682348234A04705B1A5C2B128823DC51
:103C0000511A5C2202FB01F292FBF3F31B331E4AB2
:103C10001248136001241BB2392219468DE81400A2
:103C2000322208F09BFE2046FDF714FE0B4803B03D
:103C3000BDE8F04009F07EBE511A5C2202FB01F2A1
:103C400092FBF3F31B33C6E7521A02EB4202C2EBBC
:103C50004212234492FBF3F31B33D8E7D49EFF1F99
:103C6000F09DFF1F9C8AFF1FD4220100B422010097
:103C7000B8220100D0220100169EFF1F609DFF1F89
:103C8000629EFF1FBC9EFF1F849EFF1FF0B58548EC
:103C9000854E864D83B009F0ABFC0121814809F0C7
:103CA000F3F901217F4809F0F5F9022219217D4835
:103CB00009F0E6F90A227E497A480BF0A9FF794813
:103CC0000BF0BAFF14220021764809F0D9F903223B
:103CD000784974480BF09CFF724801240BF0ACFF4C
:103CE00011228DE81400782319216E4808F036FE61
:103CF000132719231946009712226A48019408F0E5
:103D00002DFE78231946009712226648019408F088
:103D100025FE1D228DE8140078231921614808F042
:103D20001DFE1C271923194600971B225D4801948C
:103D300008F014FE7823194600971B225948019475
:103D400008F00CFE23220021564809F099F90322BD
:103D5000594954480BF05CFF52480BF06DFF28277F
:103D600019231946009724224E48019408F0F6FDC5
:103D700078231946009724224A48019408F0EEFD62
:103D800032220021474809F07BF903224B4945487C
:103D90000BF03EFF43480BF04FFF2F228DE814003D
:103DA000782319213F4808F0D9FD312719231946F6
:103DB000009730223B48019408F0D0FD7823194643
:103DC000009730223748019408F0C8FD3C228DE866
:103DD000140078231921334808F0C0FD3B2719232C
:103DE00019463A222F480194009708F0B7FD78232E
:103DF00019463A22019400972A4808F0AFFD31682D
:103E00002B682F4A5B1A5C2B128839DD521A02EBA1
:103E10004202C2EB4212234492FBF3F31B33294AC2
:103E20002048136001241BB21A2219468DE81400A1
:103E3000142208F093FD31682B682348234A04704C
:103E40005B1A5C2B128823DC511A5C2202FB01F204
:103E500092FBF3F31B331E4A1248136001241BB27A
:103E6000392219468DE81400322208F077FD2046E9
:103E7000FDF7F0FC0B4803B0BDE8F04009F05ABD77
:103E8000511A5C2202FB01F292FBF3F31B33C6E7EB
:103E9000521A02EB4202C2EB4212234492FBF3F3AA
:103EA0001B33D8E7D49EFF1FAC8AFF1FE48DFF1F92
:103EB000DC220100B4220100B8220100D02201005E
:103EC000E49DFF1F609DFF1F629EFF1FA09EFF1FBE
:103ED000849EFF1FF0B58548854E864D83B009F05E
:103EE00087FB0121814809F0CFF801217F4809F0C3
:103EF000D1F8022219217D4809F0C2F80A227E4930
:103F00007A480BF085FE79480BF096FE14220021CA
:103F1000764809F0B5F80322784974480BF078FE2A
:103F2000724801240BF088FE11228DE814007823DA
:103F300019216E4808F012FD13271923194600971E
:103F400012226A48019408F009FD78231946009767
:103F500012226648019408F001FD1D228DE814002C
:103F600078231921614808F0F9FC1C271923194608
:103F700000971B225D48019408F0F0FC7823194655
:103F800000971B225948019408F0E8FC23220021E5
:103F9000564809F075F80322594954480BF038FE89
:103FA00052480BF049FE282719231946009724226E
:103FB0004E48019408F0D2FC782319460097242239
:103FC0004A48019408F0CAFC32220021474809F00F
:103FD00057F803224B4945480BF01AFE43480BF0B3
:103FE0002BFE2F228DE81400782319213F4808F07A
:103FF000B5FC312719231946009730223B4801941C
:1040000008F0ACFC78231946009730223748019419
:1040100008F0A4FC3C228DE81400782319213348D1
:1040200008F09CFC3B27192319463A222F4801949B
:10403000009708F093FC782319463A2201940097E0
:104040002A4808F08BFC31682B682F4A5B1A5C2BDE
:10405000128839DD521A02EB4202C2EB42122344AB
:1040600092FBF3F31B33294A2048136001241BB24F
:104070001A2219468DE81400142208F06FFC3168EA
:104080002B682348234A04705B1A5C2B128823DCBC
:10409000511A5C2202FB01F292FBF3F31B331E4A1E
:1040A0001248136001241BB2392219468DE814000E
:1040B000322208F053FC2046FDF7CCFB0B4803B03E
:1040C000BDE8F04009F036BC511A5C2202FB01F257
:1040D00092FBF3F31B33C6E7521A02EB4202C2EB28
:1040E0004212234492FBF3F31B33D8E7D49EFF1F05
:1040F000E88DFF1F808BFF1FE8220100B422010022
:10410000B8220100D02201002C9EFF1F609DFF1FDE
:10411000629EFF1FB89DFF1F849EFF1F10B581B2D6
:1041200019481A4C08F0B6FF0221174808F0ACFFF6
:104130004F212122144808F0A3FF21880B2910D910
:104140000C2917D0012212490F480BF061FD21887C
:104150000D480C390BF0C0FD0B48BDE810400BF0CA
:104160006BBD0C3908480BF0B7FD0748BDE810409F
:104170000BF062BD0322074903480BF049FD0248DA
:10418000BDE810400BF058BDD49EFF1FA29EFF1F3C
:1041900014210100F422010070B5194C82B03426BC
:1041A0000023012520460193009640230B223F2146
:1041B00008F0A2FB40230B222046009601953F21E8
:1041C00008F01CFC2946204608F064FF29462046DA
:1041D00008F05AFF20460F22442108F051FF09221F
:1041E000084920460BF014FD20460BF025FD28461B
:1041F000FFF794FF204602B0BDE8704009F09ABB7B
:10420000D49EFF1FF021010008B581B20F4808F0CD
:1042100041FF02210D4808F037FF21224F210B48B2
:1042200008F02EFF0A4B1A88012A0CD0022A0EBF72
:1042300008490949032205480BF0EAFC0348BDE898
:1042400008400BF0F9BC02220449F4E7D49EFF1F9A
:10425000209EFF1FF8220100F420010058210100D8
:1042600070B5194C82B034260023012520460193F5
:10427000009640230B223F2108F03EFB40230B22F7
:104280002046009601953F2108F0B8FB29462046BC
:1042900008F000FF2946204608F0F6FE20460F22CF
:1042A000472108F0EDFE0822084920460BF0B0FC3B
:1042B00020460BF0C1FC2846FFF7A6FF204602B0BF
:1042C000BDE8704009F036BBD49EFF1FCC21010031
:1042D00008B581B2224808F0DDFE0221204808F02E
:1042E000D3FE21224F211E4808F0CAFE1D4B1B8819
:1042F000042B33D8DFE803F0121A222A030021220C
:104300005321174808F0BCFE1749022214480BF04D
:104310007FFC1348BDE808400BF08EBC21224F21E2
:104320000F4808F0ADFE03221049EFE72122532188
:104330000B4808F0A5FE02220D49E7E72122532190
:10434000074808F09DFE02220A49DFE72122532197
:10435000034808F095FE02220749D7E708BD00BFD1
:10436000D49EFF1FC89DFF1F08230100F4200100F9
:10437000FC220100002301000423010070B5194C48
:1043800082B0342600230125204601930096402365
:104390000B223F2108F0B0FA40230B222046009662
:1043A00001953F2108F02AFB2946204608F072FEBD
:1043B0002946204608F068FE20460F22442108F0D6
:1043C0005FFE0922084920460BF022FC20460BF034
:1043D00033FC2846FFF77CFF204602B0BDE8704062
:1043E00009F0A8BAD49EFF1FD821010000B53E4BAA
:1043F0001B78013B87B0052B16D8DFE803F0182D9A
:10440000425760030123394A194606201370FDF70D
:104410000BFA374809F08EFA364A374B1268059284
:10442000059A1A60FFF7B8FE07B05DF804FB012398
:10443000324A194618461370FDF7F6F92C4809F070
:1044400079FA2C4A2C4B12680192019A1A60FFF7F4
:1044500007FF07B05DF804FB0123294A1946022033
:104460001370FDF7E1F9224809F064FA214A224B62
:1044700012680292029A1A60FEF7FCF807B05DF823
:1044800004FB01231F4A194603201370FDF7CCF9E2
:10449000174809F04FFA174A174B12680392039A0C
:1044A0001A60FFF76BFF07B05DF804FB1649174B66
:1044B0006E20012208701A7007B05DF804FB01231A
:1044C000134A194605201370FDF7AEF9084809F0A4
:1044D00031FA084A084B12680492049A1A60FEF7EF
:1044E00057FF07B05DF804FB988AFF1F9E9DFF1FD2
:1044F000D49EFF1F109FFF1F349EFF1F409EFF1F73
:10450000589DFF1F649DFF1F0E9EFF1F9C8CFF1F69
:10451000C59DFF1F10B5334C334809F069F8237867
:1045200003BB01213048314C08F0B4FD06212E4870
:1045300008F0AAFD2388092B4ED9632B4FF00A02FD
:1045400094BF1F211146284808F09AFD218826486B
:104550000BF0C2FB24480BF06FFB2348BDE8104072
:1045600009F0E8B9FDF71CFA2378012BD9D9022B01
:104570004FF001011C4817D008F08CFD06211A48A5
:1045800008F082FD0A221146174808F079FD03223F
:10459000174915480BF03CFB13480BF04DFB124834
:1045A000BDE8104009F0C6B908F074FD06210E48B8
:1045B00008F06AFD0A2211460B4808F061FD03224B
:1045C0000C4909480BF024FB07480BF035FB064863
:1045D000BDE8104009F0AEB90A223021024808F0C7
:1045E0004FFDB3E7669DFF1FD49EFF1F609EFF1F18
:1045F000102301000C23010008B581B2394808F0EE
:1046000049FD0221374808F03FFD374B1B884BB16D
:10461000013B092B65D8DFE803F01C242C343C4413
:104620004C545C1421224F212E4808F029FD2F49BB
:1046300003222C480BF0ECFA2A48BDE808400BF0A6
:10464000FBBA21225321274808F01AFD02222849EB
:10465000EFE721225321234808F012FD02222549C9
:10466000E7E7212253211F4808F00AFD02222249D0
:10467000DFE7212253211B4808F002FD02221F49D7
:10468000D7E721225321174808F0FAFC02221C49DF
:10469000CFE721224F21134808F0F2FC03221949E9
:1046A000C7E721224F210F4808F0EAFC03221649F0
:1046B000BFE721224F210B4808F0E2FC03221349F7
:1046C000B7E721224F21074808F0DAFC03221049FE
:1046D000AFE721225321034808F0D2FC02220D4902
:1046E000A7E708BDD49EFF1F689EFF1FF4200100AE
:1046F00030230100FC2201001423010018230100D3
:104700001C23010020230100242301002823010091
:104710002C2301000423010070B5194C82B034260B
:104720000023012520460193009640230B223F21C0
:1047300008F0E2F840230B222046009601953F2125
:1047400008F05CF92946204608F0A4FC29462046DA
:1047500008F09AFC20460F22442108F091FC09221F
:10476000084920460BF054FA20460BF065FA28461B
:10477000FFF742FF204602B0BDE8704009F0DAB80A
:10478000D49EFF1FA021010008B581B2414808F066
:1047900081FC02213F4808F077FC3F4B1B880C2B23
:1047A00077D8DFE803F0161E262E363E464E565EBC
:1047B000666E070021225321364808F061FC374914
:1047C000022234480BF024FA3248BDE808400BF0CE
:1047D00033BA212253212F4808F052FC02223049DB
:1047E000EFE7212253212B4808F04AFC02222D49F1
:1047F000E7E721225321274808F042FC02222A49F8
:10480000DFE721225321234808F03AFC02222749FE
:10481000D7E721224F211F4808F032FC0322244908
:10482000CFE7212253211B4808F02AFC022221490C
:10483000C7E721225321174808F022FC02221E4913
:10484000BFE721225321134808F01AFC02221B491A
:10485000B7E7212253210F4808F012FC0222184921
:10486000AFE7212253210B4808F00AFC0222154928
:10487000A7E721225321074808F002FC022212492F
:104880009FE721225321034808F0FAFB02220F4937
:1048900097E708BDD49EFF1FAA9DFF1F6423010058
:1048A00034230100382301003C2301004023010090
:1048B00044230100482301004C2301005023010040
:1048C00054230100582301005C23010060230100F0
:1048D00070B5194C82B0342600230125204601937F
:1048E000009640230B223F2108F006F840230B22BC
:1048F0002046009601953F2108F080F82946204681
:1049000008F0C8FB2946204608F0BEFB20460F22CF
:10491000502108F0B5FB0522084920460BF078F934
:1049200020460BF089F92846FFF72EFF204602B0FB
:10493000BDE8704008F0FEBFD49EFF1FAC2101000F
:1049400000B5444B1B78013B87B0052B16D8DFE838
:1049500003F0182D42576C0301233F4A19460620E5
:104960001370FCF761FF3D4808F0E4FF3C4A3D4B03
:1049700012680592059A1A60FDF7A4FD07B05DF86C
:1049800004FB0123384A194618461370FCF74CFF04
:10499000324808F0CFFF324A324B12680092009A38
:1049A0001A60FFF7B9FE07B05DF804FB01232F4A38
:1049B000194602201370FCF737FF284808F0BAFFA9
:1049C000274A284B12680192019A1A60FEF748FAAA
:1049D00007B05DF804FB0123254A19460320137034
:1049E000FCF722FF1D4808F0A5FF1D4A1D4B126869
:1049F0000292029A1A60FDF7FFFC07B05DF804FB13
:104A000001231C4A194604201370FCF70DFF1348BC
:104A100008F090FF124A134B12680392039A1A602F
:104A2000FFF756FF07B05DF804FB0123124A194651
:104A300005201370FCF7F8FE084808F07BFF084AD1
:104A4000084B12680492049A1A60FEF70FFD07B033
:104A50005DF804FBA88AFF1FEC9DFF1FD49EFF1F7B
:104A6000109FFF1F349EFF1F5A9DFF1FA89EFF1F10
:104A7000949DFF1FFF9EFF1FBA9DFF1F2DE9F0436E
:104A80000320ADF5257D09F01FFEB0FA80F4042067
:104A900009F01AFE002814BF002102216409052034
:104AA0000C4409F011FE002814BF00210421062047
:104AB0000C4409F009FE9E4D9E4E2B68002814BF41
:104AC0000021082121449942316000F02D819A4C47
:104AD0009A4B22680492049A1A60236805939848B6
:104AE000059B0068944F9B1A834220D9954B1A6806
:104AF000914216D03A680792934ADDF81CE0934839
:104B00001960C2F800E00BF0E7F890480BF094F859
:104B10003B6806938E4A8F4B0698106031680122DD
:104B20001A70012900F0E180042900F0DE808A4F2C
:104B300029603D78002D00F0CD80236882490B93D9
:104B4000864A0B9B096812687B485B1A93423FD9DF
:104B5000834E84488449854A854D864CDFF864C27B
:104B6000DFF864E201233370002303700B701370CD
:104B700081488249824A2B70237003700B70137036
:104B8000804D814C81488249824A2B70237003708A
:104B90000B701370804D814C81488249824A8CF899
:104BA00000303B708EF800302B70237003700B7058
:104BB0001370AE217D48674C08F022FD002333704E
:104BC0002378002B40F004810DF5257DBDE8F083AE
:104BD000022D00F03381012D00F0E681642D00F0FC
:104BE00089810A2D00F02A820B2D01F035800C2DD1
:104BF00001F04181142D01F04E82152D00F0B48397
:104C0000162D01F091841E2D01F074861F2D01F0E8
:104C10006887202D02F07A80282D02F0B381292D9B
:104C200002F083822A2D02F089833C2D02F07784E2
:104C30003D2D02F02785502D02F094865A2D02F06A
:104C4000DB866E2DC0D1464E3378002B43F0768143
:104C50004A4D2A78002A02F075872368DFF86C81B4
:104C60008E93534A8E9BD8F8001012685B1A9342B9
:104C700011D9504B1A78012A0CBF002201221A7058
:104C80001878FDF757FC494808F054FE23688F93C5
:104C90008F9BC8F800302F4A1378002B94D0294BF3
:104CA0001B680021013B1170072B8DD801A252F81F
:104CB00023F000BF9D9200006F920000C94B0000DE
:104CC00039920000C94B0000C94B0000C94B0000DD
:104CD0000B920000224E3378002B7FF46AAF1D4CFC
:104CE0002378002B3FF470AF72E023681848324AF3
:104CF00008930668089B10680F4A9B1B83427FF647
:104D000016AF13682D4809932D4E099B0768366826
:104D1000DB1BB3427FF60BAF13680A930A9A0D4B65
:104D2000026001221A7002E7044B034C1A68D4E6B1
:104D3000249EFF1FC09EFF1F109FFF1F6C9EFF1F22
:104D4000A48CFF1F649EFF1F989DFF1F1094FF1FE0
:104D5000E89DFF1FF89DFF1F0E9EFF1FF08DFF1F98
:104D60009C8CFF1F5A9DFF1FA89EFF1F949DFF1F35
:104D7000409EFF1F589DFF1F649DFF1F2E9EFF1F1B
:104D8000C59DFF1F9E9DFF1FBA9DFF1FEC9DFF1F2E
:104D9000399EFF1FB79EFF1F4C9EFF1F049EFF1FE3
:104DA000DD9DFF1FB49EFF1FB59EFF1FD49EFF1FFA
:104DB000908DFF1F629EFF1F948AFF1F909DFF1F13
:104DC000F88CFF1F809EFF1FDC9DFF1F349EFF1F7E
:104DD00000232370FCF71CFCB94ABA4BBA49BB4804
:104DE00012781B780968007802EB43034A1E03EB34
:104DF00080030E2A3FF6E8AE01A151F822F000BF71
:104E0000D5520000A3520000C94B00006B520000B5
:104E1000C94B0000C94B0000C94B000039520000CB
:104E2000C94B0000C94B0000C94B0000C94B000032
:104E3000C94B0000C94B000035520000A44E337826
:104E4000002B40F0FC86A34D2A6823680D93A249ED
:104E50000D9B09689B1A8B4211D9A048A0490122D9
:104E60000023027026200B703B703270FCF778FD37
:104E70009C4B1988884202D02620FCF765FD9A4B8E
:104E80001A78002A3FF4A0AE00221A70FCF7C0FB8B
:104E90008B4A8C4B8C498D4812781B7809680078B6
:104EA00002EB43034A1E03EB80030E2A3FF68CAE4F
:104EB00001A151F822F000BF455500001555000032
:104EC000C94B0000CF540000C94B0000C94B000083
:104ED000C94B0000A9540000C94B00004954000010
:104EE000C94B0000C94B0000C94B0000C94B000072
:104EF00035520000764E3378002B41F0C6807B4D52
:104F00002B78002B40F05081DFF8F89199F8005091
:104F1000002D01F057812368DFF8EC812493744A57
:104F2000D8F80010249B12685B1A9342714A1178DA
:104F300000D8C1B1704B1878012802F0E18001203F
:104F40001870002941F0BE8618786C4B013D53F86B
:104F50002510FDF7C7FB6A4808F0ECFC2368259391
:104F6000259BC8F80030604A1378002B3FF42CAE24
:104F7000554B1B680021013B1170072B3FF624AEF7
:104F800001A252F823F000BFB3590000735900008A
:104F9000C94B000029590000C94B0000C94B000053
:104FA000C94B0000DB580000494E3378002B40F01D
:104FB0005C87DFF8589199F80000002800F0A8807D
:104FC0002368DFF844811293494A129BD8F80010F5
:104FD00012685B1A934210D9474B1A78012A0CBF0A
:104FE000002001201870FDF73DFC454808F0A2FCA8
:104FF00023681393139BC8F800303B4A1378002BA7
:105000003FF4E2AD304B1B680021013B1170072BD0
:105010003FF6DAAD01A252F823F000BFC9560000F6
:1050200099560000C94B000063560000C94B0000B0
:10503000C94B0000C94B000033560000244E3378A2
:10504000002B40F089812368DFF8BC802E93284A2A
:105050002E9BD8F8001012685B1A934210D9264B89
:105060001A78012A0CBF002001201870FCF7F2FB0F
:10507000234808F05FFC23682F932F9BC8F800306B
:10508000194A1378002B3FF49FAD0F4B1B6800218A
:10509000013B1170072B3FF697AD01A252F823F0A8
:1050A000FD550000F5550000C94B0000BF5500003C
:1050B000C94B0000C94B0000C94B00008B550000D4
:1050C000A99EFF1F009FFF1F649EFF1F019FFF1FE0
:1050D0009C8CFF1FAC9DFF1FEC8DFF1F9D9DFF1F34
:1050E000669DFF1F609EFF1FF89DFF1F399EFF1FDB
:1050F000908DFF1FCC9EFF1F629EFF1F888CFF1F9D
:10510000D49EFF1FB79EFF1F349EFF1F809EFF1F70
:10511000DFF8289399F80030002B40F0E080DFF8AA
:10512000209399F80020002A01F029812268DFF8F5
:1051300014831A92AF491A9AD8F800000968121A13
:105140008A4211D9AC4A117801290BBF18460120B7
:1051500013701070FCF7D2FFA84808F0EBFB23682F
:105160001B931B9BC8F80030A54A1378002B3FF413
:105170002BADA44B1B680021013B1170072B3FF6A0
:1051800023AD01A252F823F0D35B0000975B00002F
:10519000C94B0000095C0000C94B0000C94B00006E
:1051A000C94B0000675B00002368DFF898822093FA
:1051B000904AD8F80010209B12685B1A9342924ADA
:1051C000117800D8B1B18C4B1878012801F07685A0
:1051D00001201870002941F0878318788B4B1968DB
:1051E000FDF780FA854808F0A5FB23682193219BF1
:1051F000C8F80030824A1378002B3FF4E5AC814BAD
:105200001B680021013B1170072B3FF6DDAC01A2AA
:1052100052F823F0D5570000A1570000C94B0000F9
:1052200069570000C94B0000C94B0000C94B000082
:10523000FF56000009F06EFD754B76491C78764BE1
:10524000764A09881B8812680B44002C01F086807E
:10525000B2EB630F81F26C86AF21684808F0D0F999
:10526000642201233A703370AEE4002B01F0838096
:10527000013B6B4A32F813304BB16A4D6A486B49B7
:105280006B4A2B800123002505700B701370AF2132
:105290005A4808F0B5F9012302223A70237033709E
:1052A00092E473B1013B5E4A32F813304BB15D4C6E
:1052B0005D485E495E4A23800123002404700B7020
:1052C0001370AF214D4808F09BF9022201233A7078
:1052D000337079E4002BE5D101232370F1E72368D3
:1052E000DFF860811693434A169BD8F800101268C5
:1052F0005B1A93420FD9404B1A78012A18BF01203C
:105300001870FDF72BFA3D4808F014FB236817933B
:10531000179BC8F800303A4A1378002B3FF454AC7E
:10532000384B1B680021013B1170072B3FF64CAC3A
:1053300001A252F823F000BFA558000075580000E4
:10534000C94B00003F580000C94B0000C94B00008A
:10535000C94B00000F580000FEF774FB354A0121CD
:105360000023117033706EE62368DFF8D8803A931B
:10537000204A3A9BD8F8001012685B1A934219D958
:105380001D4A1E481378012B0CBF00230123137004
:10539000294A0193B2F900301A22194600921422C8
:1053A00007F0DCFA154808F0C5FA23683B933B9BED
:1053B000C8F80030124A1378002B3FF405AC114BAB
:1053C0001B680021013B1170072B3FF6FDAB01A2CA
:1053D00052F823F0E75A0000C15A0000C94B000000
:1053E000415A0000C94B0000C94B0000C94B0000E6
:1053F000FF590000908DFF1F629EFF1FD49EFF1F6C
:10540000F89DFF1F649EFF1FCC9EFF1F488BFF1F50
:105410009C9DFF1F969DFF1F429EFF1FC09DFF1F6B
:10542000789DFF1F609EFF1FED9DFF1F9D9DFF1F2D
:10543000669DFF1F749DFF1F609DFF1FB09DFF1F96
:10544000DC9DFF1F349EFF1FFBF738F9B94808F0B9
:10545000CFF80121B74807F01DFE0221B54807F03B
:1054600013FE0F222321B34807F00AFE0522B2499A
:10547000B0480AF0CDFBAF480AF0DEFB1E22232124
:10548000AC4807F0FDFD0522AC49AA480AF0C0FB74
:10549000A8480AF0D1FBA74808F04CFA23681193FA
:1054A000119B2B60FFF790BBA54C2378012B41F299
:1054B0002B862620FCF754FAA24B1988884202D08A
:1054C0002620FCF741FA00232370FFF77DBB002B59
:1054D00001F00B85013B9C4A32F8136096B1994B61
:1054E0009A489B49964A1E80002701230770262070
:1054F0000B701370FCF734FA864203D03146262035
:10550000FCF722FAFFF706F823681093109B2B6034
:10551000FFF75ABB83B1013B8B4A32F813305BB1C2
:10552000884E8A488A49864A3380012300260670BD
:105530000B701370FEF7EEFF23680F930F9B2B6029
:10554000FFF742BB002B01F0E184013B7E4A32F8B9
:10555000136096B17B4B7D487D49794A1E800027B8
:105560000123077026200B701370FCF7F9F98642AF
:1055700003D031462620FCF7E7F9FEF7CBFF23687E
:105580000E930E9B2B60FFF71FBB012302203B7085
:105590003370FCF7E5F96F4B1988884202D002207E
:1055A000FCF7D2F90420FCF7DBF96B4B1988884231
:1055B0003FF40AAB0420FCF7C7F9FFF705BB012352
:1055C0003C22022033703A70FCF7CAF9614B19880B
:1055D000884202D00220FCF7B7F90420FCF7C0F99A
:1055E0005D4B198888423FF4EFAA0420FCF7ACF920
:1055F000FFF7EABA0B233B70FFF7E6BA0123142248
:10560000022033703A70FCF7ABF9524B198888428C
:1056100002D00220FCF798F90420FCF7A1F94E4BC8
:10562000198888423FF4D0AA0420FCF78DF9FFF7CF
:10563000CBBA0120FDF716F9484B3E4800241C70F8
:1056400008F078F90E2089F80040FCF789F9444BFE
:10565000198888423FF4B8AA0E20FCF775F9FFF7C5
:10566000B3BA3F4D2B88172B3FF6AEAA0020FDF7AB
:10567000F9F82B88012003442B80FDF7F3F8374B12
:105680002C4800221A7008F055F923681593159BD1
:10569000C8F80030FFF798BA0120FDF7E3F82F4B68
:1056A000244800241C7008F045F90E2089F80040B9
:1056B000FCF756F92A4B198888423FF485AA0E2038
:1056C000FCF742F9FFF780BA254D2B88002B3FF4F9
:1056D0007BAA0020FDF7C6F82B880120013B2B8018
:1056E000FDF7C0F81D4B134800221A7008F022F98C
:1056F00023681493149BC8F80030FFF765BA194C5F
:1057000001202168FCF7EEFF144B0A4800261E70AA
:1057100008F010F944202E70FCF722F921681831A6
:1057200088423FF451AA89B24420FCF70DF9FFF7F3
:105730004BBA00BFD49EFF1F6823010070230100F5
:10574000669DFF1F609EFF1F789DFF1FED9DFF1F41
:105750009D9DFF1F169EFF1FBC9EFF1F629EFF1F89
:10576000869DFF1F488BFF1FAE4D296817293FF705
:105770002BAA0020FCF7B6FF2B6801331946012045
:105780002B60FCF7AFFFA84BA84800221A7008F066
:10579000D1F823682393239BC8F80030FFF714BA8D
:1057A000A04C01202168FCF79DFF9F4B9F480026DD
:1057B0001E7008F0BFF844202E70FCF7D1F8216865
:1057C000183188423FF400AA89B24420FCF7BCF8A3
:1057D000FFF7FAB9934D296811F1170FFFF6F4A9F5
:1057E0000020FCF77FFF2B68013B194601202B604E
:1057F000FCF778FF8C4B8D4800221A7008F09AF85D
:1058000023682293229BC8F80030FFF7DDB90120FE
:10581000FCF7A4FF844B854800241C7008F08AF82C
:10582000282089F80040FCF79BF8814B19888842B2
:105830003FF4CAA92820FCF787F8FFF7C5B97C4DCB
:105840002B88052B3FF6C0A90020FCF787FF2B888B
:10585000012003442B80FCF781FF734B7348002227
:105860001A7008F067F823681993199BC8F800307C
:10587000FFF7AAB90120FCF771FF6B4B6B480024BE
:105880001C7008F057F8282089F80040FCF768F8E9
:10589000674B198888423FF497A92820FCF754F8F1
:1058A000FFF792B9624D2B88002B3FF48DA90020A1
:1058B000FCF754FF2B880120013B2B80FCF74EFFA7
:1058C000594B5A4800221A7008F034F8236818938C
:1058D000189BC8F80030FFF777B999F80030554E9B
:1058E000013B012056F82310FCF7FCFE4E4B4F48BD
:1058F00000221A7008F01EF899F8005005F12204F1
:105900006400E4B2013D2046FCF72AF856F8251061
:105910001831884203D089B22046FCF715F80023DD
:1059200089F80030FFF750B999F80030414D424EE8
:10593000013B55F8231017293FF746A90020FCF733
:10594000D1FE3378013B012055F823200244114653
:1059500045F82320FCF7C6FE334B344800221A706A
:1059600007F0E8FF23682793279BC8F80030FFF76C
:105970002BB999F800302F4E013B012056F8231027
:10598000FCF7B0FE284B294800221A7007F0D2FF1E
:1059900099F8005005F122046400E4B22046013D6C
:1059A000FBF7DEFF56F825309842B8D003F1180116
:1059B000B1E799F800301F4D1F4E013B55F82310F9
:1059C00011F1170FFFF600A90020FCF78BFE3378CA
:1059D000013B012055F82320013A114645F82320C8
:1059E000FCF780FE104B114800221A7007F0A2FF4E
:1059F00023682693269BC8F80030FFF7E5B80F4BC5
:105A00000A48B3F90030142401221A2501920095A6
:105A1000194622463C7006F0A1FF044807F08AFFB1
:105A2000FFF7D2B8488BFF1F629EFF1FD49EFF1F57
:105A30008C9EFF1F888CFF1FB79EFF1F609DFF1F5E
:105A4000B24EB34BB34F32881B6839681A448A424E
:105A5000BFF6BAA8B04D3280B5F90030AF484FF06C
:105A6000000E1A2219468DE80440142206F076FF33
:105A7000AB4B3A6819683388521A5C2A42F3598052
:105A8000591A5D23561C03FB01F393FBF6F61B36F4
:105A900033B201211A2201910092194614229F4823
:105AA0002E6006F05BFF9D4807F044FF23683D939E
:105AB0003D9A9C4BC8F8002000221A70FFF784B86A
:105AC000954B9648B3F9003001241A228DE8140052
:105AD0001624194614223C7006F040FF8F4807F048
:105AE00029FFFFF771B8894E894A8D4F33881268B4
:105AF00039689A1A8A427FF767A8874D3280B5F9CC
:105B0000003086484FF0000E1A2219468DE80440F6
:105B1000142206F023FF7F4B39681A683388521A23
:105B20005C2A41F3FD87591A5D23561C03FB01F3E0
:105B300093FBF6F61B3633B201211A220191009233
:105B40001946142275482E6006F008FF734807F0C6
:105B5000F1FE23683C933C9A724BC8F80020002267
:105B60001A70FFF731B80120FCF7C8FA6D4B6B488B
:105B700000241C7007F0DEFE102089F80040FBF7BF
:105B8000EFFE694B198888423FF41EA81020FBF7EE
:105B9000DBFEFFF719B8FBF73BFD644B1C78002CCC
:105BA00041F09C860120FCF7A9FA5E4B5B481C7013
:105BB00007F0C0FE102089F80040FBF7D1FE5A4BD9
:105BC000198888423FF400A81020FBF7BDFEFEF7BD
:105BD000FBBF554D2B88012B7EF6F6AF0020FCF75E
:105BE0008DFA2B880120013B2B80FCF787FA4D4B67
:105BF0004A4800221A7007F09DFE23681C931C9BE4
:105C0000C8F80030FEF7E0BF474D2B880F2B3EF65B
:105C1000DBAF0020FCF772FA2B88012003442B80B5
:105C2000FCF76CFA3F4B3D4800221A7007F082FEE9
:105C300023681D931D9BC8F80030FEF7C5BF039075
:105C4000FEF768FC03983A4D03680C930C9A2A609F
:105C500000233370FFF7F9B80368DFF8E48030936E
:105C6000344A309BD8F8001012685B1A934219D955
:105C70002C4A2A481378012B0CBF002301231370F0
:105C8000254A0193B2F900301A22194600921422D3
:105C900006F064FE214807F04DFE23683193319BE6
:105CA000C8F80030244A1378002B3EF48DAF234B04
:105CB0001B680021013B1170072B3EF685AF01A246
:105CC00052F823F0EB5D0000C55D0000C94B0000F9
:105CD000455D0000C94B0000C94B0000C94B0000E6
:105CE000E55C00000C4B0D48B3F9003001241A228A
:105CF0008DE814000A24194614223C7006F02EFE8A
:105D0000064807F017FEFEF75FBF00BFE49DFF1FC8
:105D1000909EFF1FE48DFF1F609DFF1FD49EFF1FFD
:105D2000AC8AFF1F629EFF1F549EFF1F9C9DFF1F9A
:105D3000AC9DFF1F908DFF1FF89DFF1F649EFF1FEE
:105D4000349EFF1FA24EA34BA34F32881B683968B5
:105D50001A448A42BEF638AFA04D3280B5F9003001
:105D60009F484FF0000E1A2219468DE80440142275
:105D700006F0F4FD9B4B3A6819683388521A5C2A86
:105D800041F34684591A5D23561C03FB01F393FB30
:105D9000F6F61B3633B201211A2201910092194600
:105DA00014228F482E6006F0D9FD8D4807F0C2FD01
:105DB00023683393339A8C4BC8F8002000221A7062
:105DC000FEF702BF854B8648B3F9003001241A2242
:105DD0008DE814000C24194614223C7006F0BEFD18
:105DE0007F4807F0A7FDFEF7EFBE794E794A7D4F59
:105DF0003388126839689A1A8A427EF7E5AE774D81
:105E00003280B5F9003076484FF0000E1A2219465C
:105E10008DE80440142206F0A1FD6F4B39681A6822
:105E20003388521A5C2A41F3FC83591A5D23561CAD
:105E300003FB01F393FBF6F61B3633B201211A2262
:105E4000019100921946142265482E6006F086FDE5
:105E5000634807F06FFD23683293329A624BC8F8AB
:105E6000002000221A70FEF7AFBEFDF737FB0023BB
:105E70003370FFF79EB80368DFF8848134935B4A80
:105E8000349BD8F8001012685B1A934219D9564B0C
:105E900053481A78012A0CBF002201221A70544B71
:105EA0000192B3F90030392219460092322206F0ED
:105EB00055FD4B4807F03EFD23683593359BC8F8E8
:105EC00000304C4A1378002B3EF47EAE4A4B1B68E0
:105ED0000021013B1170072B3EF676AE01A252F86D
:105EE00023F000BF05600000AB5F0000C94B00005D
:105EF0002B5F0000C94B0000C94B0000C94B0000DC
:105F0000055F00003A4B3648B3F9003001243922CE
:105F10008DE814000A24194632223C7006F01EFD5A
:105F20002F4807F007FDFEF74FBE344E294B2A4F8E
:105F300032881B6839681A448A42BEF645AE2C4D39
:105F40003280B5F9003026484FF0000E392219464C
:105F50008DE80440322206F001FD224B3A681968B0
:105F60003388521A5C2A41F3D384591A5D23561C94
:105F700003FB01F393FBF6F61B3633B20121392202
:105F8000019100921946322215482E6006F0E6FC77
:105F9000134807F0CFFC23683793379A124BC8F8A1
:105FA000002000221A70FEF70FBE114B0C48B3F907
:105FB0000030012439228DE814000A2419463222C7
:105FC0003C7006F0CBFC064807F0B4FCFEF7FCBDC5
:105FD000169EFF1F709EFF1F9C8AFF1F609DFF1F64
:105FE000D49EFF1FF09DFF1F629EFF1F908DFF1F1D
:105FF000849EFF1FF89DFF1F649EFF1FBC9EFF1F16
:10600000349EFF1FC34FC44AC448C5493B88126829
:10601000008809689A1A43189A427EF7D5ADC14D97
:106020003A80B5F90030C0483922002619468DE87B
:106030004400322206F092FCBC4ABD4B11681A683B
:106040003B88521A5C2A41F34084591A5D23561C3E
:1060500003FB01F393FBF6F61B3633B20121392221
:106060000191009219463222AF482E6006F076FC6C
:10607000AD4807F05FFC23683693369AAD4BC8F8FD
:10608000002000221A70FEF79FBDFDF7BFF8002325
:106090003370FEF734BFA84E3378002B40F01885DC
:1060A0002368DFF8B0823893A44A389BD8F80010F0
:1060B00012685B1A934210D99E4B1A78012A0CBFC2
:1060C000002001201870FBF7C5FB974807F032FC51
:1060D00023683993399BC8F80030994A1378002B0C
:1060E0003EF472AD974B1B680021013B1170072BEA
:1060F0003EF66AAD01A252F823F000BF8F610000A6
:1061000087610000C94B000051610000C94B0000CD
:10611000C94B0000C94B00001D610000012306208F
:106120003B703370FBF71CFC874B1988884202D008
:106130000620FBF709FC0820FBF712FC834B1988AB
:1061400088423EF441AD0820FBF7FEFBFEF73CBD64
:1061500001230A22062033703A70FBF701FC7A4BC8
:106160001988884202D00620FBF7EEFB0820FBF7D7
:10617000F7FB764B198888423EF426AD0820FBF7E2
:10618000E3FBFEF721BD15233B70FEF71DBD012388
:106190001E22062033703A70FBF7E2FB6A4B198827
:1061A000884202D00620FBF7CFFB0820FBF7D8FB84
:1061B000664B198888423EF407AD0820FBF7C4FB04
:1061C000FEF702BDDFF89091236899F80010DFF820
:1061D0008481002900F0BB822893584A289BD8F874
:1061E000001012685B1A934211D9524B1A78012A97
:1061F00015BF0120284618701D70FCF715FD4A4890
:1062000007F098FB23682993299BC8F800304C4A73
:106210001378002B3EF4D8AC4A4B1B680021013B9D
:106220001170072B3EF6D0AC01A252F823F000BF4C
:10623000E3620000B3620000C94B0000816200000D
:10624000C94B0000C94B0000C94B0000516200005F
:106250000120FCF7E9FC374B334800241C7007F0A1
:1062600069FB4E2089F80040FBF77AFB384B198810
:1062700088423EF4A9AC4E20FBF766FBFEF7A4BCB7
:106280000020FCF7D1FC324A1388B3FA83F35B0990
:1062900001201380FCF7C8FC264B234800221A700B
:1062A00007F048FB23682B932B9BC8F80030FEF7C0
:1062B0008BBC0120FCF7B8FC1E4B1B4800241C7053
:1062C00007F038FB4E2089F80040FBF749FB204BD4
:1062D000198888423EF478AC4E20FBF735FBFEF778
:1062E00073BC0020FCF7A0FC194A1388B3FA83F3AF
:1062F0005B0901201380FCF797FC0E4B0A48002233
:106300001A7007F017FB23682A932A9BC8F80030FD
:10631000FEF75ABCBC9EFF1F709EFF1F169EFF1FFC
:106320009C8DFF1F849EFF1FD49EFF1FF09DFF1FAB
:106330009C8AFF1F629EFF1F9C8CFF1F908DFF1F7A
:10634000F89DFF1F649EFF1FE49DFF1FA09EFF1F7F
:10635000C69DFF1F349EFF1F4C9EFF1FB2EB630FB5
:1063600080F28C83AF21C64807F04AF901233B70C5
:106370003370FEF729BC01232370FEF788BF236822
:10638000DFF840831E93BF481E9BD8F800100068BA
:106390005B1A834215D9BC4B1978012916BF01221B
:1063A0001A701A70B94B08BF154618782946FBF7C2
:1063B0003BFAB34807F0BEFA23681F931F9BC8F847
:1063C0000030B34B1A78002A3EF4FEAB00221A705C
:1063D000FBF71EF9AF4AB04BB049B14812781B78B1
:1063E0000968007802EB43034A1E03EB80030B2A83
:1063F0003EF6EAAB01A151F822F000BFE7640000CD
:10640000DF640000C94B00009D640000C94B000020
:10641000C94B0000C94B000091640000C94B00004B
:106420002D640000C94B00005F640000002B3EF4A7
:10643000CBAB9C4A9C4D128803F11900013B4000F4
:10644000022425F813201146012300F0FE003370CA
:106450003C70FBF779FA954B1C70FEF7B5BB002B2F
:106460003EF4B2AB03F119008F4D013B0022400016
:1064700025F813201146012300F0FE00022433709A
:106480003C70FBF761FA894B03221A70FEF79CBB44
:10649000002201233A703370FEF796BB7B4C2078C4
:1064A00001287EF691AB0021FBF7BEF92378764DEB
:1064B000013BDBB2184601212370FBF7B5F900243C
:1064C00034238DE818006E482C7040230B223F21A6
:1064D00006F012FA6A4807F02DFAFEF775BBFCF7D2
:1064E00045FAFEF771BB694C207805283EF66CAB87
:1064F0000021FBF799F92378634D0133DBB218468D
:1065000001212370FBF790F9002434238DE8180053
:106510005B482C7040230B223F2106F0EDF95848D0
:1065200007F008FAFEF750BB2368DFF898813E9326
:10653000544A3E9BD8F8001012685B1A934219D94E
:10654000514A4F481378012B0CBF002301231370CD
:10655000574A0193B2F9003039221946009232228B
:1065600006F0FCF9464807F0E5F923683F933F9BA6
:10657000C8F80030464A1378002B3EF425AB474B51
:106580001B680021013B1170072B3EF61DAB01A2D9
:1065900052F823F0C96600005B660000C94B00009A
:1065A000DB650000C94B0000C94B0000C94B00006F
:1065B000B56500003E4B3248B3F900300124392262
:1065C0008DE814001424194632223C7006F0C6F9F6
:1065D0002B4807F0AFF9FEF7F7BA364E364B374F78
:1065E00032881B6839681A448A42BEF6EDAA304DDB
:1065F0003280B5F9003022484FF0000E392219469A
:106600008DE80440322206F0A9F92D4B3A6819684A
:106610003388521A5C2A41F33B83591A5D23561C76
:1066200003FB01F393FBF6F61B3633B2012139224B
:10663000019100921946322211482E6006F08EF91F
:106640000F4807F077F923684193419A0E4BC8F839
:10665000002000221A70FEF7B7BA154B0848B3F9AC
:106660000030012439228DE8140014241946322206
:106670003C7006F073F9024807F05CF9FEF7A4BA23
:10668000D49EFF1F908DFF1F629EFF1F3289FF1F48
:10669000F89DFF1FA99EFF1F009FFF1F649EFF1F05
:1066A000019FFF1F609EFF1F789DFF1F669DFF1FBC
:1066B000849EFF1FA09EFF1F909EFF1FE48DFF1F63
:1066C000AC8AFF1F349EFF1FB84EB94AB948BA4979
:1066D00033881268008809689A1A43189A427EF72C
:1066E00073AAB64D3280B5F90030B548392200277B
:1066F00019468DE88400322206F030F9B14AB24BD7
:1067000011681A683388521A5C2A41F35D82591A5B
:106710005D23561C03FB01F393FBF6F61B3633B2E5
:10672000012139220191009219463222A4482E609B
:1067300006F014F9A24807F0FDF823684093409A48
:10674000A24BC8F8002000221A70FEF73DBA2C9325
:106750009F4A2C9BD8F8000012681B1A934211D94B
:106760009A4B1A78012A18BF01211970994B187891
:10677000FBF75AF8924807F0DDF823682D932D9B1C
:10678000C8F80030944B1A78002A3EF41DAA002263
:106790001A70FAF73DFF914A914B9249924812784C
:1067A0001B780968007802EB43034A1E03EB800361
:1067B0000B2A3EF609AA01A151F822F0A7680000B1
:1067C0009F680000C94B00005D680000C94B0000D5
:1067D000C94B0000C94B000051680000C94B0000C4
:1067E000ED670000C94B00001F680000002B3EF45D
:1067F000EBA97E4A7E4D128803F11900013B40004F
:10680000022425F813201146012300F0FE00337006
:106810003C70FBF799F8774B1C70FEF7D5B9002B4D
:106820003EF4D2A903F11900714D013B0022400052
:1068300025F813201146012300F0FE0002243370D6
:106840003C70FBF781F86B4B03221A70FEF7BCB962
:10685000002201233A703370FEF7B6B95D4C207800
:1068600001287EF6B1A90021FAF7DEFF2378574D03
:10687000013BDBB2184601212370FAF7D5FF002453
:1068800034238DE818004E482C7040230B223F2102
:1068900006F032F84A4807F04DF8FEF795B9FCF7D4
:1068A00021FAFEF791B94B4C207805283EF68CA9C9
:1068B0000021FAF7B9FF2378444D0133DBB21846C3
:1068C00001212370FAF7B0FF002434238DE818006B
:1068D0003B482C7040230B223F2106F00DF838482E
:1068E00007F028F8FEF770B9002101201170187028
:1068F000FEF774BC404E3378002B40F00D842368C3
:10690000DFF800814293324A429BD8F800101268A7
:106910005B1A934210D92D4B1A78012A0CBF002024
:1069200001201870FAF796FF254807F003F823684E
:106930004393439BC8F80030274A1378002B3EF45A
:1069400043A9284B1B680021013B1170072B3EF621
:106950003BA901A252F823F0476A00003F6A0000F9
:10696000C94B0000096A0000C94B0000C94B000078
:10697000C94B00007969000001230A203B70337085
:10698000FAF7EEFF1D4B1988884202D00A20FAF769
:10699000DBFF0C20FAF7E4FF194B198888423EF41C
:1069A00013A90C20FAF7D0FFFEF70EB9A09EFF1F27
:1069B000909EFF1FE49DFF1F9C8DFF1F849EFF1F65
:1069C000D49EFF1FAC8AFF1FE48DFF1F629EFF1F36
:1069D000908DFF1F948DFF1FF89DFF1FA99EFF1F25
:1069E000009FFF1F649EFF1F019FFF1F609EFF1FF0
:1069F000789DFF1F669DFF1F9C8CFF1F2C9EFF1F15
:106A0000B89DFF1F349EFF1F012314220A203370FC
:106A10003A70FAF7A5FFAE4B1988884202D00A20D7
:106A2000FAF792FF0C20FAF79BFFAA4B19888842CD
:106A30003EF4CAA80C20FAF787FFFEF7C5B81F235B
:106A40003B70FEF7C1B8012328220A2033703A7048
:106A5000FAF786FF9E4B1988884202D00A20FAF77F
:106A600073FF0C20FAF77CFF9A4B198888423EF49A
:106A7000ABA80C20FAF768FFFEF7A6B8964E974D24
:106A800033782A88B3FA83F382F002025B09114655
:106A9000422033702A80FAF757FF21460D2007F075
:106AA0000DFE962007F046FE01210D2007F006FEA0
:106AB000962007F03FFE21460D2007F0FFFD9620AF
:106AC00007F038FE01210D2007F0F8FDFEF77CB835
:106AD000FDF7DCF8824A0121002311703370FFF7C3
:106AE000DFBA2368DFF8208244937E4A449BD8F8BB
:106AF000001012685B1A934219D97B4A7B481378BD
:106B0000012B0CBF002301231370794A0193B2F9C2
:106B100000301A2219460092142205F01FFF734814
:106B200006F008FF23684593459BC8F80030714A7A
:106B30001378002B3EF448A86F4B1B680021013BE3
:106B40001170072B3EF640A801A252F823F000BFB7
:106B50003D6C0000176C0000C94B0000976B0000F3
:106B6000C94B0000C94B0000C94B0000716B00000D
:106B70005F4B5E48B3F9003001241A228DE81400FF
:106B80001E24194614223C7005F0E8FE574806F012
:106B9000D1FEFEF719B84E4E584B594F32881B683C
:106BA00039681A448A42BEF60FA8514D3280B5F9B1
:106BB00000304E484FF0000E1A2219468DE804406E
:106BC000142205F0CBFE4F4B3A6819683388521AED
:106BD0005C2A41F38581591A5D23561C03FB01F39E
:106BE00093FBF6F61B3633B201211A220191009273
:106BF000194614223D482E6005F0B0FE3B4806F0D1
:106C000099FE23684793479A374BC8F80020002223
:106C10001A70FDF7D9BF364B3448B3F90030012460
:106C20001A228DE814002024194614223C7005F025
:106C300095FE2E4806F07EFEFDF7C6BF244E2F4A75
:106C4000304F3388126839689A1A8A427DF7BCAF90
:106C5000274D3280B5F9003024484FF0000E1A223B
:106C600019468DE80440142205F078FE244B39685B
:106C70001A683388521A5C2A41F32981591A5D2314
:106C8000561C03FB01F393FBF6F61B3633B20121CE
:106C90001A22019100921946142214482E6005F020
:106CA0005DFE124806F046FE23684693469A0E4B58
:106CB000C8F8002000221A70FDF786BF0020187067
:106CC000FEF788BA0021012011701870FEF73DB957
:106CD0002C9EFF1FB89DFF1FBE9DFF1FBE9EFF1F66
:106CE000749DFF1F908DFF1F629EFF1FD49EFF1F8C
:106CF000609DFF1FF89DFF1F649EFF1F749EFF1F76
:106D0000808BFF1FE88DFF1F349EFF1F2368DFF875
:106D100044834893BC4A489BD8F8001012685B1A19
:106D2000934219D9B94ABA481378012B0CBF0023F2
:106D300001231370B74A0193B2F900303922194682
:106D40000092322205F00AFEB14806F0F3FD2368F6
:106D50004993499BC8F80030AF4A1378002B3DF4A3
:106D600033AFAE4B1B680021013B1170072B3DF682
:106D70002BAF01A252F823F0656E00003F6E0000B9
:106D8000C94B0000BF6D0000C94B0000C94B00009B
:106D9000C94B0000996D00009E4B9D48B3F900302F
:106DA000012439228DE814001E24194632223C7039
:106DB00005F0D4FD964806F0BDFDFDF705BF984EE1
:106DC000984B994F32881B6839681A448A42BDF63D
:106DD000FBAE904D3280B5F900308D484FF0000E7B
:106DE000392219468DE80440322205F0B7FD8F4B59
:106DF0003A6819683388521A5C2A41F39180591A0B
:106E00005D23561C03FB01F393FBF6F61B3633B2EE
:106E10000121392201910092194632227C482E60CC
:106E200005F09CFD7A4806F085FD23684B934B9A4C
:106E3000764BC8F8002000221A70FDF7C5BE754BCE
:106E40007348B3F90030012439228DE814001E2460
:106E5000194632223C7005F081FD6D4806F06AFD4E
:106E6000FDF7B2BE6E4E6F4A7148724933881268A0
:106E7000008809689A1A43189A427DF7A5AE654DB5
:106E80003280B5F9003062483922002719468DE872
:106E90008400322205F062FD644A634B11681A686F
:106EA0003388521A5C2A41F30980591A5D23561C13
:106EB00003FB01F393FBF6F61B3633B201213922B3
:106EC000019100921946322251482E6005F046FD8C
:106ED0004F4806F02FFD23684A934A9A4B4BC8F857
:106EE000002000221A70FDF76FBE534A534E1388DC
:106EF00053487F2B94BF013301231380514A002351
:106F00000121337003701170FEF7FCBA4A4A4B4EF0
:106F100013884B48012B8CBF03F1FF338023138070
:106F2000484A00230121337003701170FEF725BB1E
:106F3000454D464C2B782288B3FA83F382F0040245
:106F40005B09114642202B702280FAF7FDFC0021DC
:106F50000D2007F0B3FB962007F0ECFB01210D207C
:106F600007F0ACFB962007F0E5FB00210D2007F0B1
:106F7000A5FB962007F0DEFB01210D2007F09EFB0C
:106F8000FDF722BE324E3378002B40F05383236846
:106F9000DFF8C0804C931C4A4C9BD8F80010126854
:106FA0005B1A934210D9194B1A78012A0CBF0020A2
:106FB00001201870FAF74EFC154806F0BBFC236858
:106FC0004D934D9BC8F80030134A1378002B3DF4C5
:106FD000FBAD124B1B680021013B1170072B3DF6E6
:106FE000F3AD01A252F823F0CB700000C370000093
:106FF000C94B00008D700000C94B0000C94B000058
:10700000C94B000059700000908DFF1F629EFF1F4A
:10701000D49EFF1F849EFF1FF89DFF1F649EFF1FCD
:10702000B89DFF1F749EFF1F808BFF1FE88DFF1F01
:107030002C9EFF1F9C8DFF1F609EFF1FED9DFF1F5D
:10704000669DFF1F9D9DFF1F149EFF1FBE9EFF1F7D
:107050009C8CFF1F349EFF1F012322203B70337046
:10706000FAF77EFCA74B1988884202D02220FAF753
:107070006BFC2420FAF774FCA34B198888423DF47A
:10708000A3AD2420FAF760FCFDF79EBD01231E226C
:10709000222033703A70FAF763FC9A4B19888842C1
:1070A00002D02220FAF750FC2420FAF759FC964B24
:1070B000198888423DF488AD2420FAF745FCFDF795
:1070C00083BD29233B70FDF77FBD01233C22222095
:1070D00033703A70FAF744FC8A4B1988884202D020
:1070E0002220FAF731FC2420FAF73AFC864B198863
:1070F00088423DF469AD2420FAF726FCFDF764BD13
:1071000000201870FDF71DBF8049012300220B707D
:1071100033703A70FEF7CDB9FCF7DCFE7C4A0121F2
:10712000002311703370FFF7EABB2368DFF8088291
:107130004E93784A4E9BD8F8001012685B1A93421F
:107140001AD9754B75491A787548012A0CBF002267
:1071500001221A701A78B1F9003001921A221946E8
:107160000092142205F0FAFB6D4806F0E3FB236859
:107170004F934F9BC8F800306A4A1378002B3DF4B8
:1071800023AD694B1B680021013B1170072B3DF6B5
:107190001BAD01A252F823F0857200005F7200005F
:1071A000C94B0000DF710000C94B0000C94B000053
:1071B000C94B0000B9710000584B5948B3F9003071
:1071C00001241A228DE814002824194614223C7048
:1071D00005F0C4FB524806F0ADFBFDF7F5BC494E87
:1071E000524B534F32881B6839681A448A42BDF6A5
:1071F000EBAC4A4D3280B5F9003049484FF0000EF3
:107200001A2219468DE80440142205F0A7FB494BC9
:107210003A6819683388521A5C2A40F35587591A1C
:107220005D23561C03FB01F393FBF6F61B3633B2CA
:1072300001211A22019100921946142238482E6029
:1072400005F08CFB364806F075FB23685193519A84
:10725000314BC8F8002000221A70FDF7B5BC2F4B47
:107260002F48B3F9003001241A228DE814002A2493
:10727000194614223C7005F071FB294806F05AFBB0
:10728000FDF7A2BC1F4E294A2A4F3388126839687D
:107290009A1A8A427DF798AC204D3280B5F90030B9
:1072A0001F484FF0000E1A2219468DE804401422A0
:1072B00005F054FB1E4B39681A683388521A5C2A51
:1072C00041F32187591A5D23561C03FB01F393FBFD
:1072D000F6F61B3633B201211A22019100921946AB
:1072E00014220F482E6005F039FB0D4806F022FBF2
:1072F00023685093509A084BC8F8002000221A7057
:10730000FDF762BC969DFF1F429EFF1F9D9DFF1FC4
:10731000749DFF1F908DFF1F629EFF1F609DFF1FCA
:10732000D49EFF1FF89DFF1F649EFF1F489EFF1FF6
:10733000A08AFF1FFC8DFF1F349EFF1F2368DFF80C
:1073400040835293BF4A529BD8F8001012685B1AD0
:1073500093421AD9BC4BBD491A78BD48012A0CBFCB
:10736000002201221A701A78B1F9003001923922F4
:1073700019460092322205F0F1FAB54806F0DAFA21
:1073800023685393539BC8F80030B24A1378002BFC
:107390003DF41AACB04B1B680021013B1170072B68
:1073A0003DF612AC01A252F823F000BF9974000020
:1073B00073740000C94B0000F3730000C94B000058
:1073C000C94B0000C94B0000CD7300009F4BA04883
:1073D000B3F90030012439228DE81400282419461D
:1073E00032223C7005F0BAFA994806F0A3FAFDF78C
:1073F000EBBB9A4E9A4B9B4F32881B6839681A44F4
:107400008A42BDF6E1AB914D3280B5F9003090482B
:107410004FF0000E392219468DE80440322205F063
:107420009DFA914B3A6819683388521A5C2A41F3E5
:107430003B80591A5D23561C03FB01F393FBF6F6C0
:107440001B3633B2012139220191009219463222B2
:107450007F482E6005F082FA7D4806F06BFA2368BB
:107460005593559A784BC8F8002000221A70FDF702
:10747000ABBB764B7648B3F90030012439228DE856
:1074800014002824194632223C7005F067FA70482F
:1074900006F050FAFDF798BB704E714A7348744974
:1074A00033881268008809689A1A43189A427DF74F
:1074B0008BAB664D3280B5F9003065483922002724
:1074C00019468DE88400322205F048FA664A654B79
:1074D00011681A683388521A5C2A41F31D86591ABA
:1074E0005D23561C03FB01F393FBF6F61B3633B208
:1074F00001213922019100921946322254482E600E
:1075000005F02CFA524806F015FA23685493549A61
:107510004D4BC8F8002000221A70FDF755BB554EA0
:107520003378002B40F0F4822368DFF854815693BF
:10753000444A569BD8F8001012685B1A934211D93E
:10754000414B1A78012A0CBF002201221A701878C8
:10755000FAF780F93E4806F0EDF923685793579BF8
:10756000C8F800303B4A1378002B3DF42DAB3A4B62
:107570001B680021013B1170072B3DF625AB01A2D2
:1075800052F823F0EF750000E7750000C94B0000CA
:10759000C5750000C94B0000C94B0000C94B000075
:1075A000A575000001232A203B703370FAF7D8F943
:1075B000314B198888423DF407AB2A20FAF7C4F909
:1075C000FDF702BB012328222A2033703A70FAF714
:1075D000C7F9294B198888423DF4F6AA2A20FAF700
:1075E000B3F9FDF7F1BA3D233B70FDF7EDBA012386
:1075F0000A222A2033703A70FAF7B2F91E4B198822
:1076000088423DF4E1AA2A20FAF79EF9FDF7DCBA98
:107610005E1A5C2303FB06F393FBF2F61B36FEF7C0
:10762000B9BB5E1A5C2303FB06F393FBF2F61B3631
:10763000FEF703BCFCF7E2F8104A012100231170A9
:107640003370A4E4908DFF1F629EFF1F849EFF1F76
:10765000D49EFF1FF89DFF1F649EFF1F429EFF1FC9
:10766000489EFF1FA08AFF1FFC8DFF1F969DFF1FD6
:107670009C8DFF1F9C8CFF1FC49EFF1F749DFF1FCE
:10768000349EFF1F2368DFF8D4825893A54A589B85
:10769000D8F8001012685B1A93421AD9A24BA3497A
:1076A0001A78A348012A0CBF002201221A701A7806
:1076B000B1F9003001921A2219460092142205F005
:1076C0004DF99B4806F036F923685993599BC8F841
:1076D0000030984A1378002B3DF476AA964B1B682D
:1076E0000021013B1170072B3DF66EAA01A252F852
:1076F00023F000BF17780000F1770000C94B0000AD
:107700003B770000C94B0000C94B0000C94B00008B
:1077100015770000854B8648B3F9003001241A2202
:107720008DE814003C24194614223C7005F016F92B
:107730007F4806F0FFF8FDF747BA804E804A814F38
:1077400033881268D7F800E01A447245BDF63CAAA7
:107750007D497E4BDFF8089208681D68D9F8001053
:1077600093B2CEEB01012A1A914233806F4DCEEBDA
:107770000303CCBF02FB03335343754AC8BF013137
:1077800093FBF1F3B5F90010034413604FF0000EC2
:107790001A220B468DE804406548142205F0DEF8F5
:1077A000D9F800103A683388521A5C2A40F3A4874B
:1077B000591A5D23561C03FB01F393FBF6F61B36A7
:1077C00033B201211A22019100921946142258481D
:1077D0002E6005F0C3F8564806F0ACF823685B93BA
:1077E0005B9A514BC8F8002000221A70FDF7ECB9E3
:1077F0004E4B4F48B3F9003001241A228DE8140093
:107800003C24194614223C7005F0A8F8484806F0BC
:1078100091F8FDF7D9B9494E494ADFF844913388C8
:107820001268D9F800509A1AAA427DF7CDA9474BA1
:10783000444F4549D7F800E01868096893B2CEEB89
:107840000505421A95423380CEEB030341F354847D
:1078500002FB03336A1C93FBF2F31944334D3C4A99
:10786000B5F9003011604FF0000E1A2219468DE86C
:1078700004402F48142205F071F8D9F800103A6836
:107880003388521A5C2A41F32E84591A5D23561C00
:1078900003FB01F393FBF6F61B3633B201211A22E8
:1078A000019100921946142221482E6005F056F8E5
:1078B0001F4806F03FF823685A935A9A1A4BC8F8A3
:1078C000002000221A70FDF77FB95E1A5C2303FBCB
:1078D00006F393FBF2F61B36FEF7BFBB1D4A137887
:1078E000B3FA83F35B0901201370FAF707FC0E4B20
:1078F0000F4800221A7006F01DF8174A138883F00B
:107900000803194642201380FAF71EF8FDF75CB908
:107910005E1A5C2303FB06F393FBF2F61B36FEF7BD
:107920002CBB00BF908DFF1F629EFF1F609DFF1F3D
:10793000D49EFF1FF89DFF1F649EFF1FC49EFF1F64
:107940008C9DFF1F848CFF1FA48AFF1FA08CFF1F2C
:10795000988CFF1F2F9EFF1FBE9EFF1F349EFF1F90
:10796000F48DFF1F9D4E33781BB1FBF73BFB0023CB
:1079700033709B4D2978002900F086802368DFF85A
:1079800088825C93974A5C9BD8F8001012685B1A57
:10799000934211D9944B1A78012A0CBF002201227C
:1079A0001A701878FCF728FE904805F0C3FF23688A
:1079B0005D935D9BC8F800308D4A1378002B3DF431
:1079C00003A98C4B1B680021013B1170072B3DF66E
:1079D000FBA801A252F823F09F8F00006D8F0000DA
:1079E000C94B0000378F0000C94B0000C94B000095
:1079F000C94B0000058F0000784E3378002B40F013
:107A000098827D4D2A78002A00F000812368DFF8F3
:107A1000F8817893734A789BD8F8001012685B1A43
:107A2000934211D9704B1A78012A0CBF002201220F
:107A30001A701878FCF7E8FB6C4805F07BFF2368A8
:107A40007993799BC8F80030694A1378002B3DF48C
:107A5000BBA8684B1B680021013B1170072B3DF64A
:107A6000B3A801A252F823F0778E0000498E0000DF
:107A7000C94B0000C58E0000C94B0000C94B000077
:107A8000C94B00001B8E00005C4D2A78002A00F0D4
:107A90004B812368DFF870816293524A629BD8F869
:107AA000000012681B1A934211D94F4B1A78012A11
:107AB00016BF012219701A701878FBF7ABF94B4802
:107AC00005F038FF23686393639BC8F80030484A89
:107AD0001378002B3DF478A8464B1B680021013B2E
:107AE0001170072B3DF670A801A252F823F000BFD9
:107AF0006993000037930000C94B00000593000014
:107B0000C94B0000C94B0000C94B0000D3920000D4
:107B1000FBF7B8FD3A4A012100231170337003E5E9
:107B20005E1A5C2303FB06F393FBF2F61B36FEF7AB
:107B300002B85E1A5C2303FB06F393FBF2F61B36D6
:107B4000FDF7A6BF2F4D2978002900F0AA802368F1
:107B5000DFF8B48092932349929BD8F8000009681B
:107B60001B1A8B4210D9204B1978012918BF01220A
:107B70001A701878F9F78EFE1C4805F0DBFE2368B2
:107B80009393939BC8F80030194A1378002B3DF467
:107B90001BA8184B1B680021013B1170072B3DF6F9
:107BA00013A801A252F823F0D59100008F91000094
:107BB000C94B000059910000C94B0000C94B00009F
:107BC000C94B00002B9100005E1A5C2303FB06F3F7
:107BD00093FBF2F61B36FEF7A2BD00BF9C8CFF1F85
:107BE0005A9DFF1F908DFF1F629EFF1FD49EFF1F97
:107BF000F89DFF1F649EFF1F409EFF1FA89EFF1F52
:107C0000749DFF1F049EFF1F349EFF1FB94D2978EE
:107C1000002900F00F812368DFF800837C93B649C8
:107C20007C9BD8F8000009681B1A8B4210D9B34B13
:107C30001978012918BF01221A701878FAF7E0FCA8
:107C4000AF4805F077FE23687D937D9BC8F8003030
:107C5000AC4A1378002B3CF4B7AFAB4B1B68002148
:107C6000013B1170072B3CF6AFAF01A252F823F095
:107C7000B190000083900000C94B00004D900000BF
:107C8000C94B0000C94B0000C94B00001F90000009
:107C90005E1A5C2303FB06F393FBF2F61B36FEF73A
:107CA000C4BC9A4D2A78002A00F066842368DFF865
:107CB0006C829693904A969BD8F8000012681B1A23
:107CC000934211D98D4B1A78012A16BF01221970DF
:107CD0001A701878F9F7FCFD894805F02BFE236827
:107CE0009793979BC8F80030864A1378002B3CF492
:107CF0006BAF854B1B680021013B1170072B3CF6D5
:107D000063AF01A252F823F0218D0000B78C000070
:107D1000C94B0000E58C0000C94B0000C94B0000B6
:107D2000C94B0000198A0000794D297800293DD0FF
:107D30002368DFF8E88166936F49669BD8F80000F6
:107D400009681B1A8B4210D96C4B1978012918BF8E
:107D500001221A701878FAF725FB694805F0EAFD48
:107D600023686793679BC8F80030664A1378002B36
:107D70003CF42AAF644B1B680021013B1170072BB8
:107D80003CF622AF01A252F823F000BFD78A0000D0
:107D9000A98A0000C94B0000758A0000C94B000089
:107DA000C94B0000C94B0000478A0000594D2A7892
:107DB000002A00F0B9822368DFF860816A934E4A96
:107DC0006A9BD8F8000012681B1A934211D94B4BDA
:107DD0001A78012A16BF012219701A701878FCF758
:107DE000D3FC474805F0A6FD23686B936B9BC8F84E
:107DF0000030444A1378002B3CF4E6AE424B1B683B
:107E00000021013B1170072B3CF6DEAE01A252F8B7
:107E100023F000BF858C0000578C0000C94B000088
:107E2000238C0000C94B0000C94B0000C94B000067
:107E3000F58B0000384D2A78002A00F085802368F1
:107E4000DFF8D88080932C4A809BD8F80000126815
:107E50001B1A934211D9294B1A78012A16BF012205
:107E600019701A701878FCF733FA254805F062FD8E
:107E700023688193819BC8F80030224A1378002B35
:107E80003CF4A2AE204B1B680021013B1170072B74
:107E90003CF69AAE01A252F823F000BFE78D000035
:107EA000B98D0000C94B0000858D0000C94B000052
:107EB000C94B0000C94B0000578D00005E1A5C23BF
:107EC00003FB06F393FBF2F61B36FEF7F6BF5E1AD2
:107ED0005C2303FB06F393FBF2F61B36FEF7D6BEDC
:107EE0005E1A5C2303FB06F393FBF2F61B36FEF7E8
:107EF0007ABE00BF589DFF1F908DFF1F629EFF1F1F
:107F0000D49EFF1FF89DFF1F649EFF1FDD9DFF1F76
:107F1000949DFF1FFF9EFF1F649DFF1F349EFF1F48
:107F20005E1A5C2303FB06F393FBF2F61B36FEF7A7
:107F30006EBFFBF7E1F80023337062E5FAF7C8FF84
:107F400000233370FCF784BEBB4D297800293DD057
:107F50002368DFF808838493B849849BD8F800002D
:107F600009681B1A8B4210D9B54B1978012918BF23
:107F700001221A701878FBF7D5F9B24805F0DAFC3F
:107F800023688593859BC8F80030AF4A1378002B8F
:107F90003CF41AAEAD4B1B680021013B1170072B5E
:107FA0003CF612AE01A252F823F000BFF3820000AB
:107FB000C5820000C94B00008F820000C94B000041
:107FC000C94B0000C94B000061820000A04D23682E
:107FD0002A78DFF88882002A3AD08893974A889BCB
:107FE000D8F8000012681B1A934211D9944B1A78E2
:107FF000012A16BF012219701A701878FCF78EF842
:10800000904805F097FC23688993899BC8F8003055
:108010008D4A1378002B3CF4D7AD8C4B1B680021A4
:10802000013B1170072B3CF6CFAD01A252F823F0B3
:1080300003820000D5810000C94B00009F81000031
:10804000C94B0000C94B0000C94B00007181000002
:108050008C937A498C9BD8F8000009681B1A8B42D4
:1080600012D9774B1978012918BF01221A70794A61
:1080700019781078F9F7D8FB724805F05BFC236893
:108080008D938D9BC8F800306F4A1378002B3CF419
:108090009BAD6E4B1B680021013B1170072B3CF61A
:1080A00093AD01A252F823F02F8100002781000038
:1080B000C94B0000E5800000C94B0000C94B00001F
:1080C000C94B0000DB8000005E1A5C2303FB06F353
:1080D00093FBF2F61B36FFF7AAB801233B7033700F
:1080E000FCF772BD5B4C207801287CF66DAD002159
:1080F000F9F79AFB2378524D013BDBB21846012178
:108100002370F9F791FB002434238DE818004D48C3
:108110002C7040230B223F2104F0EEFB494805F070
:1081200009FCFCF751BDFCF761F9FCF74DBD494C6A
:10813000207805283CF648AD0021F9F775FB237837
:108140003F4D0133DBB2184601212370F9F76CFB78
:10815000002434238DE818003A482C7040230B2269
:108160003F2104F0C9FB374805F0E4FBFCF72CBDC8
:108170000120FBF7D3FF324B324800241C7005F07E
:10818000D9FB32202C70F9F7EBFB334B198888426E
:108190003CF41AAD3220F9F7D7FBFCF715BD2E4D94
:1081A0002B88172B3CF610AD0020FBF7B7FF2B8870
:1081B000012003442B80FBF7B1FF214B2148002213
:1081C0001A7005F0B7FB23688B938B9BC8F80030BF
:1081D000FCF7FABC0120FBF7A1FF194B194800245A
:1081E0001C7005F0A7FB32202C70F9F7B9FB1A4B75
:1081F000198888423CF4E8AC3220F9F7A5FBFCF77B
:10820000E3BC154D2B88002B3CF4DEAC0020FBF7C3
:1082100085FF2B880120013B2B80FBF77FFF084B5C
:10822000084800221A7005F085FB23688A938A9B10
:10823000C8F80030FCF7C8BCC59DFF1F908DFF1F1C
:10824000629EFF1FD49EFF1FF89DFF1F649EFF1FAD
:108250009E9DFF1F988AFF1FA29EFF1F349EFF1F37
:108260000120FBF75FF8BA4BBA4800241C7005F0F8
:1082700061FB20202C70F9F773FBB74B19888842FB
:108280003CF4A2AC2020F9F75FFBFCF79DBCB24D9B
:108290002B88452B3CF698AC0020FBF743F82B8845
:1082A000012003442B80FBF73DF8A94BA94800228D
:1082B0001A7005F03FFB23688793879BC8F800304E
:1082C000FCF782BC0120FBF72DF8A14BA14800244C
:1082D0001C7005F02FFB20202C70F9F741FB9E4B02
:1082E000198888423CF470AC2020F9F72DFBFCF78C
:1082F0006BBC994D2B88002B3CF466AC0020FBF73F
:1083000011F82B880120013B2B80FBF70BF8904BD9
:10831000904800221A7005F00DFB23688693869B17
:10832000C8F80030FCF750BC8C4D297800293DD0AE
:108330002368DFF840826E9389496E9BD8F800006D
:1083400009681B1A8B4210D9814B1978012918BF73
:1083500001221A701878FBF753F87E4805F0EAFA04
:1083600023686F936F9BC8F800307E4A1378002B08
:108370003CF42AAC7C4B1B680021013B1170072B9D
:108380003CF622AC01A252F823F000BF678B00003C
:10839000398B0000C94B0000B58B0000C94B0000B1
:1083A000C94B0000C94B00000B8B00006F4D2368C8
:1083B0002A78DFF8C081002A3AD07293684A729B0B
:1083C000D8F8000012681B1A934211D9604B1A7832
:1083D000012A16BF012219701A701878FAF744F8AA
:1083E0005C4805F0A7FA23687393739BC8F80030C4
:1083F0005C4A1378002B3CF4E7AB5B4B1B68002115
:10840000013B1170072B3CF6DFAB01A252F823F0C1
:10841000E5890000B7890000C94B0000838900008E
:10842000C94B0000C94B0000C94B00005589000032
:1084300076934B49769BD8F8000009681B1A8B424B
:1084400012D9434B1978012918BF01221A70484AE2
:1084500019781078F9F7E8F93E4805F06BFA2368C7
:108460007793779BC8F800303E4A1378002B3CF492
:10847000ABAB3D4B1B680021013B1170072B3CF659
:10848000A3AB01A252F823F00F850000078500007E
:10849000C94B0000C5840000C94B0000C94B000057
:1084A000C94B0000BB8400005E1A5C2303FB06F38B
:1084B00093FBF2F61B36FEF7C4BF01233B7033700B
:1084C000FCF782BB2A4C207801287CF67DAB00218A
:1084D000F9F7AAF923781E4D013BDBB218460121BA
:1084E0002370F9F7A1F9002434238DE81800194806
:1084F0002C7040230B223F2104F0FEF9154805F0B3
:1085000019FAFCF761BBFCF71BFAFCF75DBB184CD2
:10851000207805283CF658AB0021F9F785F9237837
:108520000B4D0133DBB2184601212370F9F77CF9BA
:10853000002434238DE8180006482C7040230B22B9
:108540003F2104F0D9F9034805F0F4F9FCF73CBBEE
:10855000629EFF1FD49EFF1FB29EFF1FBA9DFF1F8A
:10856000908DFF1FF89DFF1F649EFF1FEC9DFF1F56
:10857000A88AFF1F349EFF1FBA4D297800293DD0DD
:108580002368DFF804839A93B7499A9BD8F80000D0
:1085900009681B1A8B4210D9B44B1978012918BFEE
:1085A00001221A701878F9F7B1F9B14805F0C2F94B
:1085B00023689B939B9BC8F80030AE4A1378002B2E
:1085C0003CF402ABAC4B1B680021013B1170072B44
:1085D0003CF6FAAA01A252F823F000BF1F8900005E
:1085E000F1880000C94B0000BB880000C94B0000A7
:1085F000C94B0000C94B00008D8800009F4D2368C7
:108600002A78DFF88482002A3AD09E93964A9E9B6D
:10861000D8F8000012681B1A934211D9934B1A78AC
:10862000012A16BF012219701A701878FAF716FA83
:108630008F4805F07FF923689F939F9BC8F800300F
:108640008C4A1378002B3CF4BFAA8B4B1B6800218B
:10865000013B1170072B3CF6B7AA01A252F823F098
:108660003188000003880000C94B0000D18700005A
:10867000C94B0000C94B0000C94B0000A387000094
:10868000A2937949A29BD8F8000009681B1A8B4273
:1086900012D9764B1978012918BF01221A70784A2D
:1086A00019781078F9F7C0F8714805F043F9236894
:1086B000A393A39BC8F800306E4A1378002B3CF4B8
:1086C00083AA6D4B1B680021013B1170072B3CF600
:1086D0007BAA01A252F823F06187000059870000AD
:1086E000C94B000017870000C94B0000C94B0000B0
:1086F000C94B00000B8700005E1A5C2303FB06F3E6
:1087000093FBF2F61B36FFF75BB85A2201233A704F
:108710003370FCF759BA5A4C207801287CF654AAD9
:108720000021F9F781F82378504D013BDBB2184660
:1087300001212370F9F778F8002434238DE818001C
:108740004B482C7040230B223F2104F0D5F84848B9
:1087500005F0F0F8FCF738BAFAF7DEF9FCF734BAAE
:10876000474C207804283CF62FAA0021F9F75CF842
:1087700023783E4D0133DBB2184601212370F9F70F
:1087800053F8002434238DE8180039482C70402316
:108790000B223F2104F0B0F8354805F0CBF8FCF788
:1087A00013BA0120FAF75AF9304B314800241C70F3
:1087B00005F0C0F856202C70F9F7D2F8314B198823
:1087C00088423CF401AA5620F9F7BEF8FCF7FCB940
:1087D0000020FAF743F92B4A1388B3FA83F35B09B5
:1087E00001201380FAF73AF9204B214800221A7031
:1087F00005F0A0F82368A193A19BC8F80030FCF70E
:10880000E3B90120FAF72AF9184B194800241C7023
:1088100005F090F856202C70F9F7A2F8194B19883A
:1088200088423CF4D1A95620F9F78EF8FCF7CCB970
:108830000020FAF713F9134A1388B3FA83F35B099C
:1088400001201380FAF70AF9084B094800221A7030
:1088500005F070F82368A093A09BC8F80030FCF7DF
:10886000B3B900BFB49EFF1F908DFF1F629EFF1F14
:10887000D49EFF1FF89DFF1F649EFF1FB59EFF1F24
:108880008C8AFF1FFA9DFF1F349EFF1F0120F9F7FE
:108890003DF8C14BC14800241C7005F04BF8542032
:1088A0002C70F9F75DF8BE4B198888423CF48CA90E
:1088B0005420F9F749F8FCF787B9B94D2B881D2BDF
:1088C0003CF682A90020F9F721F82B880120034407
:1088D0002B80F9F71BF8B04BB04800221A7005F056
:1088E00029F823689D939D9BC8F80030FCF76CB96C
:1088F0000120F9F70BF8A84BA84800241C7005F0DC
:1089000019F854202C70F9F72BF8A54B19888842D8
:108910003CF45AA95420F9F717F8FCF755B9A04DC3
:108920002B88012B7CF650A90020F8F7EFFF2B884D
:108930000120013B2B80F8F7E9FF974B9748002275
:108940001A7004F0F7FF23689C939C9BC8F80030D2
:10895000FCF73AB90120F9F787FD8F4B8F480024C7
:108960001C7004F0E7FF30202C70F8F7F9FF8D4BF6
:10897000198888423CF428A93020F8F7E5FFFCF775
:1089800023B90020F9F770FD864A1388082B94BF9D
:108990000133002301201380F9F766FD7E4B7F48E9
:1089A00000221A7004F0C6FF23687593759BC8F8FF
:1089B0000030FCF709B90120F9F756FD764B7748EE
:1089C00000241C7004F0B6FF30202C70F8F7C8FFAC
:1089D000744B198888423CF4F7A83020F8F7B4FFAC
:1089E000FCF7F2B80020F9F73FFD6E4A1388002B20
:1089F00000F09381013B13800120F9F735FD664BB0
:108A0000664800221A7004F095FF23687493749BE3
:108A1000C8F80030FCF7D8B80120F8F759FF5E4BD2
:108A20005E4800241C7004F085FF52202C70F8F77B
:108A300097FF5D4B198888423CF4C6A85220F8F78E
:108A400083FFFCF7C1B80120F9F7ACFC524B534847
:108A500000241C7004F06EFF16202C70F8F780FFC5
:108A6000524B198888423CF4AFA81620F8F76CFFE7
:108A7000FCF7AAB80020F9F795FC4C4A13887E2B26
:108A800094BF0133002301201380F9F78BFC424B84
:108A9000424800221A7004F04DFF23686993699BD5
:108AA000C8F80030FCF790B80120F9F77BFC3A4B8E
:108AB0003A4800241C7004F03DFF16202C70F8F793
:108AC0004FFF3A4B198888423CF47EA81620F8F7ED
:108AD0003BFFFCF779B80020F9F764FC334A1388B0
:108AE000002B00F08180013B13800120F9F75AFC34
:108AF000294B2A4800221A7004F01CFF236868934F
:108B0000689BC8F80030FCF75FB80120FAF778FCE2
:108B1000214B224800241C7004F00CFF2E202C70E6
:108B2000F8F71EFF224B198888423CF44DA82E20EE
:108B3000F8F70AFFFCF748B80120FAF761FC164B7A
:108B4000164800241C7004F0F5FE2E202C70F8F757
:108B500007FF174B198888423CF436A82E20F8F7F7
:108B6000F3FEFCF731B80020FAF74AFC104A1388EC
:108B7000002B3CD0013B13800120FAF741FC064B4F
:108B8000064800221A7004F0D5FE23687093709B8B
:108B9000C8F80030FCF718B8629EFF1FD49EFF1F74
:108BA000FE8CFF1F689DFF1FD88AFF1F5C9DFF1F63
:108BB0000C9EFF1F0020FAF723FCBB4A13881D2BD5
:108BC00094BF0133002301201380FAF719FCB74B3F
:108BD000B74800221A7004F0ADFE23687193719BB0
:108BE000C8F80030FBF7F0BF7F2313807DE71E231A
:108BF0001380C1E70120FBF7C7FDAC4BAC48002454
:108C00001C7004F097FE2C202C70F8F7A9FEA94BDD
:108C1000198888423BF4D8AF2C20F8F795FEFBF773
:108C2000D3BF0020FBF7B0FDA24A13880B2B94BFE3
:108C30000133002301201380FBF7A6FD9B4B9C48CA
:108C400000221A7004F076FE23686D936D9BC8F8BD
:108C50000030FBF7B9BF0120FBF796FD934B94481A
:108C600000241C7004F066FE2C202C70F8F778FEAF
:108C7000904B198888423BF4A7AF2C20F8F764FE8C
:108C8000FBF7A2BF0020FBF77FFD8A4A1388002B69
:108C90005ED0013B13800120FBF776FD834B8448B7
:108CA00000221A7004F046FE23686C936C9BC8F88F
:108CB0000030FBF789BF0120F8F70AFE7B4B7C48A8
:108CC00000241C7004F036FE52202C70F8F748FE89
:108CD000794B198888423BF477AF5220F8F734FE7D
:108CE000FBF772BF0020F8F7F3FD734A1388032BDC
:108CF00098BF01334FF0010098BF1380F8F7E8FDEB
:108D00006A4B6B4800221A7004F014FE2368999392
:108D1000999BC8F80030FBF757BF092313806BE617
:108D20000020F8F7D5FD644A13880BB1013B13808E
:108D30000120F8F7CDFD5D4B5D4800221A7004F06C
:108D4000F9FD23689893989BC8F80030FBF73CBF67
:108D50000C2313809FE70120FBF7BAFA534B5448CA
:108D600000241C7004F0E6FD1C202C70F8F7F8FDC0
:108D7000524B198888423BF427AF1C20F8F7E4FDDA
:108D8000FBF722BF0020FBF7A3FA4C4A1388032B02
:108D900094BF0133002301201380FBF799FA434B62
:108DA000434800221A7004F0C5FD23688393839B17
:108DB000C8F80030FBF708BF0120FBF789FA3B4BEE
:108DC0003B4800241C7004F0B5FD1C202C70F8F703
:108DD000C7FD3A4B198888423BF4F6AE1C20F8F7E1
:108DE000B3FDFBF7F1BE0020FBF772FA334A13889C
:108DF000002B00F08180013B13800120FBF768FA13
:108E00002A4B2B4800221A7004F094FD23688293A9
:108E1000829BC8F80030FBF7D7BE0120FBF7F4F9BE
:108E2000224B234800241C7004F084FD18202C7071
:108E3000F8F796FD224B198888423BF4C5AE1820FE
:108E4000F8F782FDFBF7C0BE0120FBF7DDF9174BF9
:108E5000174800241C7004F06DFD18202C70F8F7E2
:108E60007FFD174B198888423BF4AEAE1820F8F707
:108E70006BFDFBF7A9BE0020FBF7C6F9104A13886B
:108E8000002B3CD0013B13800120FBF7BDF9074BC1
:108E9000074800221A7004F04DFD23687A937A9BEC
:108EA000C8F80030FBF790BE0C9EFF1F629EFF1FAC
:108EB000D49EFF1FAA9DFF1FD88AFF1FC89DFF1FBA
:108EC000209EFF1F0020FBF79FF9BC4A1388012B4F
:108ED00094BF0133002301201380FBF795F9B84BB1
:108EE000B84800221A7004F025FD23687B937B9B11
:108EF000C8F80030FBF768BE042313807DE7022327
:108F00001380C1E70120FBF777FBAD4BAD48002490
:108F10001C7004F00FFD12202C70F8F721FDAA4BF5
:108F2000198888423BF450AE1220F8F70DFDF7F790
:108F300005FCFBF749BEA44D2B88092B4FF0000020
:108F400046D8FBF759FB2B88012003442B80FBF705
:108F500053FB9B4B9B4800221A7004F0EBFC2368E8
:108F60006093609BC8F80030FBF72EBE0120FBF732
:108F700043FB934B934800241C7004F0DBFC12204D
:108F80002C70F8F7EDFC904B198888423BF41CAE2E
:108F90001220F8F7D9FCF7F7D1FBFBF715BE8A4D85
:108FA0002E8846B30020FBF727FB2B880120013BCE
:108FB0002B80FBF721FB824B824800221A7004F0C1
:108FC000B9FC23685E935E9BC8F80030FBF7FCBDDC
:108FD000FBF712FB002601202E80FBF70DFB784BE0
:108FE00078481E7004F0A6FC23686193619BC8F862
:108FF0000030FBF7E9BD3046FBF7FEFA0A230120FB
:109000002B80FBF7F9FA6E4B6E481E7004F092FC51
:1090100023685F935F9BC8F80030FBF7D5BD012044
:10902000F9F7EEFA664B674800241C7004F082FCE6
:109030001A202C70F8F794FC644B198888423BF492
:10904000C3AD1A20F8F780FCFBF7BEBD5F4D2B883F
:109050000B2B3BF6B9AD0020F9F7D2FA2B88012093
:1090600003442B80F9F7CCFA554B564800221A706E
:1090700004F060FC23687F937F9BC8F80030FBF707
:10908000A3BD0120F9F7BCFA4D4B4E4800241C70DB
:1090900004F050FC1A202C70F8F762FC4B4B198836
:1090A00088423BF491AD1A20F8F74EFCFBF78CBDDB
:1090B000464D2B88002B3BF487AD0020F9F7A0FA32
:1090C0002B880120013B2B80F9F79AFA3C4B3D4855
:1090D00000221A7004F02EFC23687E937E9BC8F851
:1090E0000030FBF771BD5E1A5C2303FB06F393FBB4
:1090F000F2F61B36FEF7D1BB02FB03F393FBF5F24E
:109100001144FEF7ABBB5E1A5C2303FB06F393FB33
:10911000F2F61B36FEF7DEB85E1A5C2303FB06F39D
:1091200093FBF2F61B36FEF7E2B90120F8F7B2FB2B
:10913000234B244800241C7004F0FCFB50202C70AE
:10914000F8F70EFC224B198888423BF43DAD5020C5
:10915000F8F7FAFBFBF738BD1D4D2B880B2B3BF6C0
:1091600033AD0020F8F796FB2B88012003442B80B9
:10917000F8F790FB124B134800221A7004F0DAFB48
:1091800023689593959BC8F80030FBF71DBD01201F
:10919000F8F780FB0A4B0B4800241C7004F0CAFB54
:1091A00050202C70F8F7DCFB094B198888423BF4FF
:1091B0000BAD5020F8F7C8FBFBF706BD209EFF1F44
:1091C000629EFF1FD49EFF1F689EFF1FD09DFF1F42
:1091D000FC8CFF1F714D2B88012B7BF6F5AC00201A
:1091E000F8F758FB2B880120013B2B80F8F752FB46
:1091F0006B4B6C4800221A7004F09CFB236894931C
:10920000949BC8F80030FBF7DFBC0120F9F792F916
:10921000634B644800241C7004F08CFB1E202C70EF
:10922000F8F79EFB604B198888423BF4CDAC1E20BA
:10923000F8F78AFBFBF7C8BC5B4D2B88082B3BF685
:10924000C3AC0020F9F776F92B88012003442B806A
:10925000F9F770F9524B534800221A7004F06AFB78
:1092600023689193919BC8F80030FBF7ADBC0120B7
:10927000F9F760F94A4B4B4800241C7004F05AFB84
:109280001E202C70F8F76CFB474B198888423BF482
:109290009BAC1E20F8F758FBFBF796BC424D2B8881
:1092A000002B3BF491AC0020F9F744F92B88012006
:1092B000013B2B80F9F73EF9394B3A4800221A70EE
:1092C00004F038FB23689093909BC8F80030FBF7BC
:1092D0007BBC0120F9F79EFD314B324800241C7005
:1092E00004F028FB14202C70F8F73AFB2F4B198858
:1092F00088423BF469AC1420F8F726FBF7F71EFA16
:10930000FBF762BC0020F9F785FD284A1388B3FA01
:1093100083F35B0901201380F9F77CFD204B214882
:1093200000221A7004F006FB23686593659BC8F859
:109330000030FBF749BC0120F9F76CFD184B1948C8
:1093400000241C7004F0F6FA14202C70F8F708FBC7
:10935000164B198888423BF437AC1420F8F7F4FA1E
:10936000F7F7ECF9FBF730BC0020F9F753FD0F4A93
:109370001388B3FA83F35B0901201380F9F74AFDE0
:10938000074B084800221A7004F0D4FA236864934B
:10939000649BC8F80030FBF717BC00BFFC8CFF1FB4
:1093A000629EFF1FD49EFF1FBC9DFF1F129EFF1FCA
:1093B0002DE9F04F924A934D1268934C934E944F7F
:1093C000DFF8D892DFF8D88295B000230CA80121ED
:1093D00004F048FB04E08F4A3B681360FBF74EFB48
:1093E0000E2004F09FFD07F00FFF01460CA804F0CB
:1093F00081FB0CA804F054FB08F020F9864B874A47
:10940000D3F800A080F30C00BAF1010F10605AD01D
:10941000BAF1020F00F0E780BAF1030F00F0728298
:1094200023680893089BD9F800209B1A022B1ED9A9
:109430007B4B1B78002B00F029837A4B794A1B78F1
:10944000002B0CBF01230023137000F01A83744B10
:109450001B78002B40F02783F7F73CFEF7F7E4F981
:10946000F7F7BCFD23680993099BC9F800306E4AE1
:10947000236811680A936D4A0A9B12685B1A93422B
:10948000A9D9F8F7DFFA6A4B1B786BB9694B1B78DF
:1094900053B9694B1B783BB9684B1B7823B9684BB0
:1094A0001B78002B01F01C860D2005F00DF9B0FA99
:1094B00080F149090D2005F001F923680B935A4A00
:1094C0000B9B136087E75F4B2A781B884D49DFF8B9
:1094D00078B19A4218BF0B705B4A5C4B12781B88BC
:1094E0009A4204D05A4A1178002940F0B585594B68
:1094F0001B88834202DB524B1B784BB123680393DA
:109500005549039A554B0A60434A18600223136079
:10951000534B197829BB534B1B7813BB524BD3F8D1
:1095200000B0002004F0FEFCABF21F3B834502DCE0
:109530004E4A00231370002005F0EEFA4C4B4D49C3
:109540001A684D4B904293F800E0D4BF00230123EA
:1095500073450B7002D0904200F34585464A137064
:109560005EE7464B464A1888464B12681B88034400
:109570005B10934280F29680434A1268934280F2D5
:109580009180002900F08E80F8F742F83F4B1A686E
:109590001846531C002B41F39080802B01F38B80E5
:1095A0003B490360B1F800E03A493B48098800684C
:1095B0007144B0EB610FC1F2CE84A2F148030F2BCE
:1095C000ACD8204B473A00210D201A8005F076F8E0
:1095D000962005F0AFF801210D2005F06FF8224B21
:1095E000D3F800B09DE71B4A12888242C0F2B480D3
:1095F000134A1278002A40F0AF8001221A600FE768
:10960000908AFF1F018DFF1F109FFF1FFC9DFF1FF2
:10961000C89EFF1F1C9EFF1F9C9EFF1F889EFF1F52
:109620002F9EFF1FC49DFF1F089EFF1F3C8CFF1F26
:10963000189EFF1F799EFF1FB69EFF1F5B9DFF1F99
:10964000A89DFF1F549EFF1FED9DFF1F609EFF1FE3
:109650009D9DFF1F169EFF1F3C9EFF1F589EFF1FD4
:10966000BE9DFF1F149EFF1F709DFF1FB19EFF1F19
:10967000988CFF1FBB9DFF1F599DFF1FB89DFF1FAB
:10968000CC9DFF1F2C9EFF1FD09EFF1FF49DFF1F30
:10969000969DFF1F429EFF1FC09DFF1F009EFF1F44
:1096A000ABAAAA2A002004F03DFCAF4BD3F800B0CF
:1096B000ABF548739842AD4B198880F2EA81AC4B08
:1096C0001B78002B00F0E581AA4BAB4A1B8812687F
:1096D0000B445B109342A94A126802DA93423FF7A7
:1096E00053AF9342BFF61DAF002004F01BFC9E4B0E
:1096F000D3F800B0ABF548739842BFF612AFA04B59
:109700001A78002A7FF40DAF4FF0010A83F800A009
:10971000F7F77EFF9B4B1B78002B41F041829A4B61
:109720001B78002B41F03284984B1B78002B01F002
:10973000FD84974B1B78002B7FF4F0AE954B1B7884
:10974000002B3FF4EBAE944B944A1B8882F800A0A8
:10975000914A0A331380E1E6914A23681168049321
:10976000904A049B12885B1A934202D8002A7FF425
:1097700057AEF7F74DFF8C4B8C4A19688C4B12880B
:109780001B688C488B42B8BF0B469342008881F21D
:109790006F82894BB3F800E0884B1A60BEF1000F6E
:1097A00041F0628213468342D4BFC2EB0301C2EB95
:1097B0000001801AB0F5804FAABF8903C1EB813147
:1097C000013091FBF0F0F6F78BFEC0F3C61007F006
:1097D0001BFD7B4B8246188807F016FD79498346AE
:1097E000504607F065FD0146584607F061FD5146B9
:1097F00007F056FC4FF07E51824607F0F7FE002836
:1098000041F07D847049504607F00EFF002841F07A
:109810005284504607F038FFC0B23070F7F766F850
:1098200038687F2841F31C827F3888FB0032C317D9
:10983000C3EB620303EB4303A0EB83007330634B82
:1098400038601B88DFF898A1002B41F01C83604B27
:109850001B78002B00F0E8855E4B1B78002B00F096
:10986000E385DFF880B14FF0000A37E003F17300C1
:1098700033782A781B0603F0FE43013A43F4104381
:10988000120202F47062000443F00903134300F46F
:10989000FE00184305F0EEFE3B68DBF800001844BC
:1098A000A0F17F0388FB0321DA17C2EB610202EB10
:1098B00042027F28A3EB820340F3F88003F1730098
:1098C0002A783178013AC0B2D2B2F6F78DFF414B17
:1098D0001B780AF1010A534540F3A6853B685BF803
:1098E000040F1844A0F17F0188FB0123CA17C2EBC3
:1098F000630303EB43037F28A1EB8303B6DCF6F796
:10990000DDFDB5E7294B1B88834240F3DB80324BFA
:109910001B78002B40F0D680304B18787F2841F31D
:1099200012817F3888FB0032C317C3EB620303EB5D
:109930004303A0EB83007330244B284A1B8810702C
:109940009246002B41F02E82214B1B78002B00F019
:10995000DD83204B1B78002B00F0D883DFF884B028
:109960004FF0000A78E000BF709DFF1FB89DFF1FF9
:10997000149EFF1F2C9EFF1FCC9DFF1FD09EFF1F1C
:10998000B19EFF1F389EFF1F989EFF1FFC9EFF1F6A
:10999000FD9EFF1FFE9EFF1F609EFF1F9D9DFF1FE0
:1099A0003C9EFF1F0C9EFF1F889EFF1F169EFF1FE1
:1099B000589EFF1FBC9EFF1F5C9DFF1FAC9EFF1F9C
:1099C000689DFF1FCDCCCC3D0000FE42C69DFF1F11
:1099D000B69EFF1F448BFF1FA89DFF1F789EFF1F91
:1099E000C89EFF1F1C8BFF1F03F1730033782A787A
:1099F0001B0603F0FE43013A43F40043120202F453
:109A00007062000443F00803134300F4FE0018439F
:109A100005F030FE274B1878DBF800301844A0F131
:109A20007F0388FB0321DA17C2EB610202EB4202DB
:109A30007F28A3EB820333DD03F173002A783178AA
:109A4000013AC0B2D2B2F6F7DFFE1B4B1B780AF127
:109A5000010A534540F35A83164B18785BF8043FCC
:109A60001844A0F17F0188FB0123CA17C2EB6303EE
:109A700003EB43037F28A1EB8303B5DCF6F71EFD60
:109A8000B4E7F6F7FDFFF7F79BFDEBE4F6F72EFFE3
:109A9000D3E40A4B0A4A1B8812680B445B1020E689
:109AA000F6F70CFDCAE7F6F721FFD5E4F6F706FD59
:109AB00006E700BF789EFF1F448BFF1F2C9EFF1FF1
:109AC000D09EFF1FF7F7A4FDA74B38681B6898428C
:109AD00001F0358023680593A44B059A1A6023682A
:109AE0000693A349069B09889B1A8B4240F26A821F
:109AF0007F2841F32F807F3888FB0032C317C3EBE8
:109B0000620303EB4303A0EB83007330994B93F89C
:109B100000A0824500F05682974B1B88002B43D152
:109B2000964A1168964A1088964A8142128805DB47
:109B30009142D4BFC0EB0103C0EB0203101AB0F591
:109B4000804FAABF9B03C3EB8333013093FBF0F03C
:109B5000F6F7C6FCC0F3C61007F056FB8A4B8346E7
:109B6000188807F051FB89490190584607F0A0FB7F
:109B7000019B0146184607F09BFB594607F090FAF7
:109B80004FF07E51834607F031FD002841F0E2821C
:109B90007F49584607F048FD002841F0AD825846FD
:109BA00007F072FDC0B23070BAF17F0F41F39880B8
:109BB000AAF17F0A88FB0A234FEAEA72C2EB630329
:109BC00003EB4303AAEB830303F17300714B694A70
:109BD0001B781070002B40F080866F4A1278002AA4
:109BE00040F07B866D4A1278002A40F076866B4BF7
:109BF0001B78002B00F089805E4B1878684B1B683F
:109C000018447F2841F33B827F3888FB0032C3171A
:109C1000C3EB620303EB4303A0EB830073303178A3
:109C20002A78090601F0FE41013A41F4004112028E
:109C3000030441F0080102F4706203F4FE0341EAF8
:109C40000200184305F016FD4A4B1878544B1B6868
:109C500018447F2841F30F827F3888FB0032C317F6
:109C6000C3EB620303EB4303A0EB830073302A785A
:109C70003178013AC0B2D2B2F6F7C6FD3D4A494B3F
:109C800010781B78484A52F8233018447F2841F353
:109C9000EE817F3888FB0032C317C3EB620303EB0E
:109CA0004303A0EB8300733032782978120602F068
:109CB000FE420139090242F4004242F00802030464
:109CC00001F4706003F4FE031043184305F0D2FC66
:109CD000284A344B10781B78334A52F82330184402
:109CE0007F2841F3C0817F3888FB0032C317C3EB64
:109CF000620303EB4303A0EB830073302A783178CF
:109D0000013AC0B2D2B2F6F77FFD224B1B78002B8E
:109D100001F01381254B19889A46002901F06D81C5
:109D200038687F2840F3B6877F3888FB0032C31736
:109D3000C3EB620303EB4303A0EB83007330386093
:109D4000DFF870A0002940F0AD87124B1B78002B84
:109D500000F02085164B1B78002B00F01B85DFF8E8
:109D600058B04FF0000A61E01C9EFF1F5C9EFF1F71
:109D7000B29EFF1F789EFF1F5C9DFF1FAC9EFF1FC2
:109D8000169EFF1FBC9EFF1F689DFF1FCDCCCC3DC4
:109D90000000FE42B69EFF1F5B9DFF1F189EFF1F27
:109DA000488BFF1FFD9DFF1F888CFF1FC69DFF1F57
:109DB000448BFF1FC89EFF1F1C8BFF1F03F1730006
:109DC00033782A781B0603F0FE43013A43F410432C
:109DD000120202F47062000443F00903134300F41A
:109DE000FE00184305F046FC3B68DBF80000184411
:109DF000A0F17F0388FB0321DA17C2EB610202EBBB
:109E000042027F28A3EB820340F3EA8003F1730050
:109E10002A783178013AC0B2D2B2F6F7E5FCA74B06
:109E20001B780AF1010A534540F3B4843B685BF8A0
:109E3000040F1844A0F17F0188FB0123CA17C2EB6D
:109E4000630303EB43037F28A1EB8303B6DCF6F740
:109E500035FBB5E79A4B1B78002B00F08B80994BB4
:109E600038681B6818447F2841F321817F3888FBBC
:109E70000032C317C3EB620303EB4303A0EB830081
:109E8000733032782978120602F0FE420139090255
:109E900042F41042030442F0090201F4706003F43A
:109EA000FE031043184305F0E5FB864B38681B683A
:109EB00018447F2841F3F7807F3888FB0032C317AE
:109EC000C3EB620303EB4303A0EB830073302A78F8
:109ED0003178013AC0B2D2B2F6F786FC7A4B7A4AB0
:109EE0001B78022B9ABF0133DBB200231370774A31
:109EF00052F823003B6818447F2841F3D0807F3814
:109F000088FB0032C317C3EB620303EB4303A0EBF0
:109F10008300733032782978120602F0FE4201394C
:109F2000090242F4104242F00902030401F4706095
:109F300003F4FE031043184305F09CFB624B634996
:109F40001A783B6851F8220018447F2841F3A38017
:109F50007F3888FB0032C317C3EB620303EB430374
:109F6000A0EB830073302A783178013AC0B2D2B2C4
:109F7000F6F73AFC564B1B88002B01F02080554B1E
:109F80001B783BB9544B1B7823B94D4B1B78002BE6
:109F900001F0F381514B1B78002B00F0D885474B23
:109FA00046481B78082B00F2D2854D493A6809686B
:109FB0000133DBB20370013B4A48511A40F82310C9
:109FC000494B1A70494B1A88494B1B689A42BFF695
:109FD00027AA23680793474A079B1360FFF720BA15
:109FE000F6F76CFA14E7F7F713FB434B1A78002ADD
:109FF00000F0D681394B19789E46002940F0CD817A
:10A0000034483E4B01702E481B78017001218EF8B8
:10A010000010002B40F01287394B1B78002B00F00A
:10A020007D832D4B2C4A1B78002B40F075833549DE
:10A030002348097803700123137049B12049012294
:10A040000A70264A00231370224A1370224A1370A2
:10A050002D4B1B78FFF782BA297801920139DBB2C8
:10A060000902581E01F47061000441F4404141F0BE
:10A070000C0100F4FE0008438BF8003005F0FAFAFA
:10A0800028789BF800B001380BF1FF3B60F03F00EF
:10A09000C0B25FFA8BFB04F0ADFC584604F0AAFC9A
:10A0A000134A10680D4A002313700A4A13700A4AB3
:10A0B0001370019A1370FFF71ABA00BF448BFF1F89
:10A0C000189EFF1F488BFF1FFD9DFF1F888CFF1FE1
:10A0D000C69DFF1FB69EFF1F5B9DFF1F799EFF1F42
:10A0E000A09DFF1F208BFF1F789EFF1F169EFF1F46
:10A0F000889EFF1F349EFF1FFE9EFF1FA99EFF1F0D
:10A10000989EFF1F9C9DFF1FBB9DFF1FB64B1B789A
:10A11000002B00F0A380B54B1B78A3F10C007F2827
:10A1200040F39D868B3B88FB0321DA17C2EB61026B
:10A1300002EB4202A3EB820303F1730033782A7827
:10A140001B0603F0FE43013A43F40043120202F4FB
:10A150007062000443F00803134300F4FE00184348
:10A1600005F088FAA14B1B78A3F10C007F2840F37F
:10A1700072868B3B88FB0321DA17C2EB610202EB8C
:10A180004202A3EB820303F173002A783178013A8B
:10A19000C0B2D2B2F6F738FB954B1B78002B5DD0DE
:10A1A000944B1B78002B59D0DFF878B24FF0000A9F
:10A1B00039E002F1730033782A781B0603F0FE437E
:10A1C000013A43F40043120243F0080302F47062C0
:10A1D000000400F4FE0142EA0300084305F04AFAD5
:10A1E000824B1A78DBF800301A44A2F18B0388FB0B
:10A1F0000310D917C1EB6001A2F10C0001EB410182
:10A200007F28A3EB810326DD03F173002A783178E0
:10A21000013AC0B2D2B2F6F7F7FA764B1B780AF1E0
:10A22000010A53451ADD714B18785BF8043F03446B
:10A23000A3F18B0E88FB0E124FEAEE71C1EB6202A6
:10A24000A3F10C0002EB42027F28AEEB8202B0DCED
:10A25000F6F734F9AFE7F6F731F9D7E7664B1B7835
:10A26000002B00F08980614B1878644B1B68184400
:10A270007F2840F304867F3888FB0032C317C3EB86
:10A28000620303EB4303A0EB8300733031782A7839
:10A29000090601F0FE41013A41F4004112020304B3
:10A2A00041F0080102F4706203F4FE0341EA020087
:10A2B000184305F0DFF94D4B1878504B1B681844D4
:10A2C0007F2840F3D8857F3888FB0032C317C3EB63
:10A2D000620303EB4303A0EB830073302A783178E9
:10A2E000013AC0B2D2B2F6F78FFA404A444B107826
:10A2F0001B78444A52F8233018447F2840F3B7852E
:10A300007F3888FB0032C317C3EB620303EB4303C0
:10A31000A0EB8300733032782978120602F0FE42F7
:10A320000139090242F4004242F00802030401F438
:10A33000706003F4FE031043184305F09BF92B4AA9
:10A340002F4B10781B782F4A52F8233018447F285F
:10A3500040F389857F3888FB0032C317C3EB620363
:10A3600003EB4303A0EB830073302A783178013A82
:10A37000C0B2D2B2F6F748FA234B1B88002B00F08C
:10A38000F184224B1B78002B40F0D484204900221A
:10A390000A60204A0123136014E600238EF800307F
:10A3A0001D4B1B783BB1124911480978002900F078
:10A3B0004585002101701949097800297FF431AEE3
:10A3C000002A40F0AB81002B40F0A8810F49144ACD
:10A3D0000B70074912780B7003490B7006490B701C
:10A3E000002A7FF42BAE33E65B9DFF1F789EFF1F94
:10A3F000B69EFF1F448BFF1F189EFF1F488BFF1F39
:10A40000FD9DFF1F888CFF1FC69DFF1F799EFF1FAC
:10A41000AC9EFF1F9C9EFF1FA99EFF1F989EFF1FC3
:10A420009C9DFF1F1C8BFF1FC54B1B78002B40F012
:10A4300048853B68C34A1278002A00F09D80A3F14A
:10A440000C007F2840F38E858B3B88FB0320DA17B6
:10A45000C2EB600000EB4000A3EB800303F173004C
:10A4600033782A781B0603F0FE43013A43F4104385
:10A47000120202F47062000443F00903134300F473
:10A48000FE00184305F0F6F83B68A3F10C007F28A6
:10A4900040F364858B3B88FB0320DA17C2EB600036
:10A4A00000EB4000A3EB800303F173002A783178BE
:10A4B000013AC0B2D2B2F6F797F9A34B1B78002B42
:10A4C00059D0A24B1B78002B55D0DFF8C4B24FF007
:10A4D000000A38E003F1730033782A781B0603F092
:10A4E000FE43013A43F41043120243F0090302F41D
:10A4F0007062010401F4FE0142EA0300084305F022
:10A50000B9F83B68DBF800201A44A2F18B0388FB02
:10A510000310D917C1EB6001A2F10C0001EB41015E
:10A520007F28A3EB810323DD03F173002A783178C0
:10A53000013AC0B2D2B2F6F757F9844B1B780AF150
:10A54000010A534517DD3B685BF8040F1844A0F17E
:10A550008B0188FB0123CA17C2EB63030C3803EBA2
:10A5600043037F28A1EB8303B4DCF5F7A7FFB3E730
:10A57000F5F7A4FFDAE73B68754A1278002A00F085
:10A580008E80744A106818447F2840F3FB84A0F141
:10A590007F0388FB0320DA17C2EB600000EB40006A
:10A5A000A3EB8000733032782978120602F0FE4265
:10A5B000013942F410420902000442F0090201F498
:10A5C000706100F4FE0341EA0200184305F052F8FE
:10A5D000604B38681B6818447F2840F3CF847F386D
:10A5E00088FB0032C317C3EB620303EB4303A0EB0A
:10A5F000830073302A783178013AC0B2D2B2F6F7CC
:10A60000F3F8554B544A1B78022B9ABF0133DBB247
:10A6100000231370514A52F823003B6818447F28E6
:10A6200040F3A8847F3888FB0032C317C3EB620372
:10A6300003EB4303A0EB83007330327829781206D2
:10A6400002F0FE42013942F41042090242F00902CE
:10A6500001F47061000400F4FE0341EA02001843B3
:10A6600005F008F83C4B3D491A783B6851F8220048
:10A6700018447F2840F37A847F3888FB0032C31760
:10A68000C3EB620303EB4303A0EB830073302A7830
:10A690003178013AC0B2D2B2F6F7A6F83B68304A38
:10A6A0001288002A00F02B842E4A13702E4A0323AE
:10A6B0001360FEF7B5BE4FF0800A2C4B2C4A198868
:10A6C0002C4B12681B882C480B44B2EB630FC0F86C
:10A6D00000A0BEF623AF294B1978002940F005836E
:10A6E000274B274A1B8853453EF418AF254BA2F849
:10A6F00000A04FF0010B0D2083F800B003F0DEFF47
:10A70000962004F017F859460D2003F0D7FF1E4B92
:10A71000D3F800B0FEF705BF00231370174B1B786A
:10A72000002B3FF495AC0A4B094A1B78002B3FF4F1
:10A7300085AC164B00211B781170FEF70FBF00BFD0
:10A74000799EFF1F5B9DFF1FB69EFF1F448BFF1F5F
:10A75000189EFF1F488BFF1FFD9DFF1F888CFF1F4A
:10A76000C69DFF1F789EFF1F9C9EFF1F429EFF1FDE
:10A77000C09DFF1F969DFF1FF49DFF1F9C9DFF1F07
:10A78000609EFF1F9D9DFF1F709DFF1FBB9DFF1FB4
:10A790001C8BFF1FB94B1B78002B3FF45BAB3B6856
:10A7A000A3F10C007F2840F372848B3B88FB0321CC
:10A7B000DA17C2EB610202EB4202A3EB820303F160
:10A7C000730033782A781B0603F0FE43013A43F402
:10A7D0001043120202F47062000443F009031343B1
:10A7E00000F4FE00184304F045FF3B68A3F10C00A1
:10A7F0007F2840F348848B3B88FB0321DA17C2EBA8
:10A80000610202EB4202A3EB820303F173002A7898
:10A810003178013AC0B2D2B2F5F7E6FF984B1B7817
:10A82000002B3FF417AB974B1B78002B3FF412AB78
:10A83000DFF85CB24FF0000A37E003F173003378C1
:10A840002A781B0603F0FE43013A43F41043120238
:10A8500002F47062000443F00903134300F4FE00A5
:10A86000184304F007FF3B68DBF800001844A0F130
:10A870008B0388FB0321DA17C2EB61020C3802EB71
:10A8800042027F28A3EB820324DD03F173002A78C0
:10A890003178013AC0B2D2B2F5F7A6FF794B1B78F6
:10A8A0000AF1010A53457FF7D5AA3B685BF8040F0C
:10A8B0001844A0F18B0188FB0123CA17C2EB630384
:10A8C0000C3803EB43037F28A1EB8303B5DCF5F7DA
:10A8D000F5FDB4E7F5F7F2FDD9E76B4A1288002AD7
:10A8E00057D1002B75D0674B1B78002B71D0DFF848
:10A8F000A0B14FF0000A37E003F1730033782A78F3
:10A900001B0603F0FE43013A43F40043120202F433
:10A910007062000443F00803134300F4FE00184380
:10A9200004F0A8FE594B1878DBF800301844A0F169
:10A930007F0388FB0321DA17C2EB610202EB4202BC
:10A940007F28A3EB820340F3F48003F173002A789D
:10A950003178013AC0B2D2B2F5F756FF494B1B78B5
:10A960000AF1010A534534DD484B18785BF8043F7F
:10A970001844A0F17F0188FB0123CA17C2EB6303CF
:10A9800003EB43037F28A1EB8303B5DCF5F796FDCA
:10A99000B4E732782978120602F0FE42013942F417
:10A9A00000420902030401F4706142F008020A4304
:10A9B00003F4FE00104304F05DFE2A78334B317837
:10A9C0001878013AD2B2F5F71FFF2D4B1B78002BF8
:10A9D00089D12A4B1B78002B3FF409A92B4B1B78FC
:10A9E000A3F10C007F2840F33B838B3B88FB0321C2
:10A9F000DA17C2EB610202EB4202A3EB820303F11E
:10AA0000730033782A781B0603F0FE43013A43F4BF
:10AA10000043120202F47062000443F0080313437F
:10AA200000F4FE00184304F025FE184B1B78A3F138
:10AA30000C007F2840F311838B3B88FB0321DA173E
:10AA4000C2EB610202EB4202A3EB820303F173004B
:10AA50002A783178013AC0B2D2B2F5F7D5FE084B68
:10AA60001B78002B00F0EB82064B1B78002B00F0CC
:10AA7000A984DFF81CB04FF0000A44E05B9DFF1F83
:10AA8000B69EFF1F448BFF1FC69DFF1F789EFF1FB2
:10AA90001C8BFF1F03F1730033782A781B0603F029
:10AAA000FE43013A43F40043120202F470620004D0
:10AAB00043F00803134300F4FE00184304F0DAFDEA
:10AAC000C74B1878DBF800301844A0F18B0388FBE3
:10AAD0000321DA17C2EB61020C3802EB42027F2835
:10AAE000A3EB820328DD03F173002A783178013A61
:10AAF000C0B2D2B2F5F788FEBA4B1B780AF1010A50
:10AB000053457FF774A8B64B18785BF8043F184498
:10AB1000A0F18B0188FB0123CA17C2EB63030C3839
:10AB200003EB43037F28A1EB8303B3DCF5F7C6FCFB
:10AB3000B2E7F5F7C3FC0AE7F5F7C0FCD5E7AA4B87
:10AB40001A68FEF7CCBFF5F7B9FCFEF7F5BE3A6818
:10AB5000FFF736BAF5F7B2FCFEF7D8BFA34B1B7868
:10AB6000002B7EF4DBACA24B1B78243B5B007F2BDD
:10AB700040F32F849F4AA0487F2313602B78013B2A
:10AB80001B0203F47063184304F074FD2A78994B98
:10AB9000013A1968D2B25B20F5F716FE974B1B7885
:10ABA000032B7EF4BBAC964A1278002A40F0B483A3
:10ABB000944B1B78002B40F07F838C4B1B78002B31
:10ABC00040F04883904B1B78002B40F013838F4A52
:10ABD00013808F4B1B78002B40F0DC828D4A7F2343
:10ABE0001380874B1B78002B7EF498AC854B1B7829
:10ABF000002B7EF493AC7D4B1A78002A7EF48EAC49
:10AC00002B7885488549013B1B0203F47063184388
:10AC10000A8004F02FFD2878013860F04F00C0B2A0
:10AC200003F0E8FE072003F0E5FE7F2003F0E2FEDC
:10AC30002B787B48013B1B0203F47063184304F03C
:10AC400019FD2878013860F04F00C0B203F0D2FE41
:10AC50000B2003F0CFFE7F2003F0CCFEFEF75EBC9E
:10AC6000F5F72CFCFEF7EBBD86F800E0FEF7D6BD4D
:10AC700068498342B1F800E06A49A8BF03460B6007
:10AC8000BEF1000FF0D19A42C8BF71463EF791ADB8
:10AC9000FEF789BDF5F712FCDFF89CA138600029AA
:10ACA0003FF453A832782978120602F0FE420139A7
:10ACB00042F410420902030401F4706142F00902F7
:10ACC0000A4303F4FE00104304F0D4FC2A789AF8F7
:10ACD00000003178013AD2B2F5F786FDFFF735B8BA
:10ACE0005046F5F7EBFBFEF771BFBAF14B0F40F39F
:10ACF000E5814D4A4C4812880AF11803802BA8BF01
:10AD000080239A423EF40AAC03804FF0010A0021EE
:10AD10000D20464B83F800A003F0D0FC962003F0F2
:10AD200009FD51460D2003F0C9FC414BD3F800B09A
:10AD3000FEF7F7BB2B783F48013B1B0203F470631F
:10AD4000184304F097FC2878013860F04F00C0B237
:10AD500003F050FE402003F04DFE002003F04AFEB9
:10AD6000FFF714BB1E4B28781A78337812041B06A1
:10AD700002F4FE0203F0FE431343013843F40043A0
:10AD8000000243F0080300F47060184304F072FC02
:10AD90002A78134B31781878013AD2B2F5F734FD9E
:10ADA000FFF7EFBA32782978120602F0FE42013935
:10ADB00042F400420902030401F4706142F0080207
:10ADC0000A4303F4FE00104304F054FC2A789AF876
:10ADD00000003178013AD2B2F5F716FDFEF7B4BDA6
:10ADE000789EFF1F448BFF1F5C9EFF1FFE9EFF1F70
:10ADF000C69EFF1FB49DFF1F0BB05B7F389EFF1FD9
:10AE0000989EFF1FFD9EFF1FFC9EFF1F129EFF1FAF
:10AE1000A99EFF1F5C9DFF1F0BB0077F689EFF1F51
:10AE20000BB00B7FAC9EFF1F609EFF1F9D9DFF1F01
:10AE3000709DFF1F0BB04000C89EFF1FC749012037
:10AE40000870C7494FF0000E81F800E0C54981F84D
:10AE500000E0FFF7B0BAF5F731FBFFF796B9F5F769
:10AE60002DFBFFF76BB9F5F729FBFFF77EBAF5F776
:10AE700025FBFFF750BAF5F721FBFFF72FBAF5F7DF
:10AE80001DFBFFF703BA32782978120602F0FE4262
:10AE9000013942F410420902030401F4706142F0E6
:10AEA00009020A4303F4FE00104304F0E3FB2A788E
:10AEB0009AF800003178013AD2B2F5F795FCFEF726
:10AEC000C6BC2B78A848013B1B0203F470631843EF
:10AED00004F0D0FB2878013860F04F00C0B203F0D6
:10AEE00089FD402003F086FD7F2003F083FD9F4A0B
:10AEF0003B689F49136000220A70FFF79BBA3278C3
:10AF00002978120602F0FE42013942F41042090289
:10AF10001B0401F4706142F0090203F4FE000A43CD
:10AF2000104304F0A7FB2A7831783878013AD2B27E
:10AF3000F5F75AFC3B68FFF7B7BB8E4B1B78002B2D
:10AF40007EF4E8AE874B1B78002B7EF4E3AE8A4B91
:10AF50001988FEF7E5BE9A46FFF7BDBBF5F7AEFAD6
:10AF6000FFF7A4BAF5F7AAFAFFF77ABAF5F7A6FA47
:10AF7000FFF78DBBF5F7A2FAFFF75FBBF5F79EFA77
:10AF8000FFF738BBF5F79AFAFFF70DBB7B4B1B7841
:10AF9000002B00F0B7807A4B1B78002B7EF4BEAA02
:10AFA000784B1B78002B3EF4B9AA774B774A1B8865
:10AFB00082F800A0744A0A3B1380FEF7AFBA3B68E0
:10AFC00031782A781B0403F4FE0343F41043090686
:10AFD000013A01F0FE41120243F009030B4302F46F
:10AFE0007060184304F046FB2A7831783878013ACB
:10AFF000D2B2F5F7F9FBFEF7C2BF654B28781A7895
:10B00000337812041B0602F4FE0203F0FE431343DE
:10B01000013843F40043000243F0080300F4706079
:10B02000184304F027FB2A78594B31781878013AF5
:10B03000D2B2F5F7E9FBBAF80010FEF771BE494B42
:10B040001B78002B7EF4D8AD4A4B1B78002B7EF486
:10B0500061AE494B1988FEF763BEF5F72FFAF7E4A6
:10B06000F5F72CFACDE4F5F729FAFEF747BEF5F728
:10B0700025FAFEF719BEF5F721FAFEF7F8BDF5F748
:10B080001DFAFEF7CCBDF5F719FAFFF7C0BBF5F7CF
:10B0900015FAFFF796BBF5F711FAFEF764BFF5F75F
:10B0A0000DFAFEF737BFF5F709FAFEF710BFF5F70F
:10B0B00005FAFEF7E6BE7F20FEF7AFBBAAF1240338
:10B0C000314A002B128840F378819A423EF426AA36
:10B0D0009BB22D4A4FF0010A00210D20138018E683
:10B0E0000D2003F0F1FA00287EF4E7A901210D20DC
:10B0F00003F0E4FAFEF7E1B97F20FEF754BD01202A
:10B10000FEF78BBB1E4B1B78002B7EF407AA1D4B52
:10B110001B78002B3EF402AA1B4B1C4A1B8882F8AA
:10B1200000A0194A013B1380FEF7F8B9144B1B78B5
:10B13000002B7FF413AD134B1B78002B3EF4EEA9CC
:10B14000114B124A1B8882F800A00F4A013313806A
:10B15000FEF7E4B90120FEF726BD00BFB69EFF1F33
:10B16000799EFF1F189EFF1F0BB0407FA09DFF1F01
:10B17000448BFF1F5B9DFF1FC69DFF1FFC9EFF1F93
:10B18000FD9EFF1FFE9EFF1F609EFF1F9D9DFF1FD8
:10B19000789EFF1F2B789748974A013B1B0203F4C8
:10B1A000706318430023138004F064FA2878013890
:10B1B00060F04F00C0B203F01DFC072003F01AFC42
:10B1C0007F2003F017FC2B788C48013B1B0203F413
:10B1D0007063184304F04EFA2878013860F04F008D
:10B1E000C0B203F007FC0B2003F004FC7F2003F047
:10B1F00001FCF6E42B787F48814A013B1B0203F4F3
:10B20000706318430123138004F034FA287801385E
:10B2100060F04F00C0B203F0EDFB072003F0EAFB43
:10B220007F2003F0E7FB2B787448013B1B0203F4FB
:10B230007063184304F01EFA2878013860F04F005C
:10B24000C0B203F0D7FB0B2003F0D4FB7F2003F048
:10B25000D1FBBEE42B7867486A4A013B1B0203F42A
:10B26000706318430423138004F004FA287801382B
:10B2700060F04F00C0B203F0BDFB072003F0BAFB43
:10B280007F2003F0B7FB28780138000200F47060DB
:10B2900040F00B1040F4304004F0ECF9287801380D
:10B2A00060F04F00C0B203F0A5FB0B2003F0A2FB3F
:10B2B000002003F09FFB85E42B784E48514A013B68
:10B2C0001B0203F4706318430223138004F0D2F9C5
:10B2D0002878013860F04F00C0B203F08BFB0720E4
:10B2E00003F088FB7F2003F085FB2B784348013B6C
:10B2F0001B0203F47063184304F0BCF9287801388A
:10B3000060F04F00C0B203F075FB0B2003F072FB3E
:10B310007F2003F06FFB50E428783A4A013800029E
:10B3200000F4706040F4F62040F00B00138004F04D
:10B33000A1F92878013860F04F00C0B203F05AFB41
:10B34000072003F057FB002003F054FB2B782B4819
:10B35000013B1B0203F47063184304F08BF9287857
:10B36000013860F04F00C0B203F044FB0B2003F043
:10B3700041FB7F2003F03EFB1AE4234B28781A7828
:10B38000337812041B0602F4FE0203F0FE4313435B
:10B39000013843F40043000243F0080300F47060F6
:10B3A000184304F067F92A78174B31781878013A76
:10B3B000D2B2F5F729FAFEF7EDBD012A3EF4AEA8A8
:10B3C000012386E6114B1B78002B7EF415ACFEF7AB
:10B3D000A1BC002B05DA0E4A0E4800231360FFF7CC
:10B3E000CDBB0B490B480B601A0602F0FE43184315
:10B3F000FFF7C4BB0BB0077F5C9DFF1F0BB00B7F3B
:10B40000129EFF1F689EFF1F789EFF1F189EFF1F42
:10B41000B49DFF1F0BB05B0008B5FDF7C9FF00BF6F
:10B420002DE9F04F0C2087B002F048FD0C2003F00E
:10B4300035F90221032003F055F90221042003F01D
:10B4400051F90221052003F04DF90221062003F0F5
:10B4500049F901210A2003F045F90121092003F0EF
:10B4600041F901210D2003F03DF90020F6F778FAAB
:10B47000172840F27B82042003F026F9002800F010
:10B480006F820020F6F76CFA1F2800F0A5821F21BA
:10B490000020F6F759FA0C210E20F6F755FA012193
:10B4A0001020F6F751FA02211220F6F74DFA00218A
:10B4B0001420F6F749FA00211620F6F745FA022182
:10B4C0001820F6F741FA01211A20F6F73DFA022179
:10B4D0001C20F6F739FA04211E20F6F735FA14215C
:10B4E0002020F6F731FA01212620F6F72DFA032164
:10B4F0002820F6F729FA04212C20F6F725FA142142
:10B500002E20F6F721FA00213020F6F71DFA0C2143
:10B510003220F6F719FA00213420F6F715FA002147
:10B520003620F6F711FA00213820F6F70DFA00213F
:10B530003A20F6F709FA00213C20F6F705FA002137
:10B540003E20F6F701FA00214020F6F7FDF9002130
:10B550004220F6F7F9F91F214420F6F7F5F91321F7
:10B560004620F6F7F1F90E214820F6F7EDF9112102
:10B570004A20F6F7E9F90A214C20F6F7E5F900210F
:10B580004E20F6F7E1F906215020F6F7DDF9022109
:10B590005220F6F7D9F90F215420F6F7D5F90021FA
:10B5A0005620F6F7D1F90220F6F7DAF9B24BB34E8E
:10B5B00018800420F6F7D4F9B14BDFF89493188083
:10B5C0000620F6F7CDF9AF4BAF4F18800820F6F7FD
:10B5D000C7F9AE4BAE4D18800A20F6F7C1F9AD4B56
:10B5E00018800C20F6F7BCF9AB4B18800E20F6F74C
:10B5F000B7F9AA4B18801020F6F7B2F9A84B1880BB
:10B600001220F6F7ADF9A74B18801420F6F7A8F929
:10B61000A54B18801620F6F7A3F9A44B1880182024
:10B62000F6F79EF9A24B18801A20F6F799F9A14B6C
:10B6300018801C20F6F794F99F4B18801E20F6F70F
:10B640008FF99E4B18802020F6F78AF99C4B1880C2
:10B650002220F6F785F99B4B18802420F6F780F915
:10B66000994B18802620F6F77BF9984A82462820C5
:10B67000A2F800A0F6F774F9954A10802A20F6F790
:10B680006FF9944A04462C201480F6F769F9924A1F
:10B6900010802E20F6F764F9904A10803020F6F7DB
:10B6A0005FF98F4A10803220F6F75AF98D4A1080E0
:10B6B0003420F6F755F930803620F6F751F97080CE
:10B6C0003820F6F74DF9B0803A20F6F749F9F080C6
:10B6D0003C20F6F745F930813E20F6F741F97081BC
:10B6E0004020F6F73DF9B0814220F6F739F97E4A5D
:10B6F0007E4E80464420A2F80080F6F731F97C4A5D
:10B70000A0F1180146201160F6F72AF9A0F11802FD
:10B710004820C9F80020F6F723F9A0F118024A20C2
:10B72000C9F80420F6F71CF9A0F118024C20C9F85A
:10B730000820F6F715F9A0F118024E20C9F80C20E0
:10B74000F6F70EF96B4A10805020F6F709F96A4AAD
:10B7500010805220F6F704F9684A10805420F6F75A
:10B76000FFF838805620F6F7FBF8654A654B6649C6
:10B77000D6F800E01668654AD3F800B00B68D2F836
:10B7800000900593624A634BD2F800C0188062496A
:10B79000059885F800A0CEEB0B0E861BCCEB0900BC
:10B7A00081FB0EA9F1444FEAEE7ECEEBA91EDFF835
:10B7B000A4915A4BC9F800E081FB069EB644F617E7
:10B7C0001A68574BDFF890C11B68DCF800C0C6EB65
:10B7D000AE16DFF888E1CEF8006081FB00E6064493
:10B7E000C017D21AC0EBA6104E4B4F4E1B683060EC
:10B7F00081FB02061644D217CCEB0300C2EBA61263
:10B800004A4E81FB00E132600144494A494EC0176B
:10B810005FFA88F8C0EBA111116008F0020E464AE9
:10B8200086F800E008F00406167044484449454A8A
:10B8300008F0080880F8008012680868C3EB0C0163
:10B84000121A9142A4EB03030FDD02FB0333013113
:10B8500093FBF1F303443C4A3C4813605A2100F047
:10B86000E1FD002840F0C580FEE702FB03F292FBF9
:10B87000F1F30344EFE700BF169EFF1F789DFF1F03
:10B88000BC9EFF1FE49DFF1FFE8CFF1FA09EFF1F9D
:10B89000ED9DFF1F2C9EFF1FB89DFF1F869DFF1F64
:10B8A000549EFF1F689EFF1F129EFF1F5C9DFF1F7F
:10B8B000209EFF1FD09DFF1FC89DFF1FBC9DFF1F27
:10B8C000B29EFF1F969DFF1F429EFF1F609EFF1F9F
:10B8D0008C9EFF1FC49EFF1FAA9DFF1F0C9EFF1F73
:10B8E000689DFF1FA29EFF1FBE9EFF1FF09DFF1FB2
:10B8F000488BFF1FC69DFF1FFC8CFF1FD88AFF1FB0
:10B90000AC8AFF1F9C8AFF1FE48DFF1F808BFF1FE7
:10B91000E88DFF1FFA9DFF1FC94216B2A08AFF1FC4
:10B92000FC8DFF1F848CFF1F749EFF1F489EFF1F0E
:10B930008C9DFF1FBE9DFF1F149EFF1F2F9EFF1F8C
:10B94000A48AFF1FA08CFF1F988CFF1F109EFF1F53
:10B95000888CFF1F709EFF1FF48DFF1F909EFF1F9E
:10B96000062002F0B1FE00287FF48BAD1F210020DD
:10B97000F5F7EAFF4FF4AF610220F5F7E5FF4FF46A
:10B980007A610420F5F7E0FF40F628210620F5F75C
:10B99000DBFF40F6E4410820F5F7D6FF4FF4AF6136
:10B9A0000A20F5F7D1FF40F6FC010C20F5F7CCFF9B
:10B9B0004FF496612220F5F7C7FF4FF4166124205B
:10B9C000F5F7C2FF7D212A20F5F7BEFF0020F5F72D
:10B9D000C7FF1F287FF45BAD042002F075FE00282E
:10B9E0007FF4E1AD062002F06FFE00283FF44FAD7A
:10B9F000D9E501233C220221594801F069FE58484B
:10BA000001F0F6FD4FF0010B002240218023CDF81C
:10BA100008B0019100931146524B514801F0F4F8DF
:10BA20004F4801F087FF0F2003F076F805900E20B5
:10BA300002F078FA594681460D2002F03FFEFA20C6
:10BA400002F078FE0F2003F067F882460E2002F025
:10BA500069FA002180460D2002F030FEFA2002F043
:10BA600069FE0F2003F058F804460E2002F05AFA3F
:10BA7000594606460D2002F021FEFA2002F05AFE39
:10BA800000210D2002F01AFE0F2003F045F8834636
:10BA90000E2002F047FA059A3988334F02EB0A0369
:10BAA000234413EB0B0348BF0333304C9B1009EBCB
:10BAB0000802324423602E4C5E1A1944131848BF02
:10BAC000033321602B493E609B10FA200B6002F08B
:10BAD00031FE01210D2002F0F1FDFA2002F02AFED4
:10BAE00000210D2002F0EAFD01211D4801F0D2FAEB
:10BAF00001211B4801F0C8FA34225521184801F0F1
:10BB0000BFFA02221C49164804F082F805221B499C
:10BB1000134804F07DF8124804F08EF8104801F044
:10BB200009FF40F2DC5002F005FE154A154B0021DA
:10BB30000124042011701C6002F0C6FD10B9124BE4
:10BB400028701C704FF4406002F004FF02F05CFFAC
:10BB500001210D2007B0BDE8F04F02F0AFBD00BFDE
:10BB6000D49EFF1F84230100E09DFF1F949EFF1FB2
:10BB7000309EFF1F709DFF1F782301007C23010072
:10BB80000E9EFF1F9C9EFF1F9D9DFF1F0020704764
:10BB900090F8392090F83800101A704790F8383033
:10BBA00090F839209A4205D95A1C034480F838206D
:10BBB000187E70474FF0FF30704700BF90F8383064
:10BBC00090F839209A4286BF1B18187E4FF0FF303C
:10BBD000704700BF704700BF38B50546B0F85E003B
:10BBE00090B195F85D301446C3F1210294420CD80F
:10BBF00005F13B001844224601F0B4FF95F85D3092
:10BC0000234485F85D30204638BD01201446287154
:10BC1000EEE700BFB0F85E306BB190F85D30202BDE
:10BC200007D8C218013380F85D30012082F83B103C
:10BC30007047012303710020704700BF0023426951
:10BC400080F8383080F8393080F85C3080F85D302A
:10BC500080F85E3080F85F3006CA30B40D68046941
:10BC600043662A4383660A60A370426990F8613094
:10BC70001649146813441D7A5B7B01EBC5051B0252
:10BC80006D6803F4E06343F064032B6090F8623066
:10BC900013449D7CDB7D01EBC5011B02496803F465
:10BCA000E06343F064030B6021685368194205D0D8
:10BCB000036927225A70036904229A7103692022BA
:10BCC0005A71036980229A7030BC70474C2E010073
:10BCD00043690CCB12681A420CD0094B99420AD91D
:10BCE000084B9942036994BF1A220D225A700369C6
:10BCF00004229A717047036927225A70F7E700BF40
:10BD00007F1A06003F420F0010B50269D378DBB2FC
:10BD1000D90604463DD510215806D17038D503F018
:10BD2000040303F0FF02002B51D03D49626E002353
:10BD30000B7084F85D30002A5BD0904794F85D303A
:10BD4000002B56D02369D0229A70236994F83B20A7
:10BD50001A712369012284F85C200222DA7010BD76
:10BD6000304B84F860009C424AD02F4B9C4252D00A
:10BD700094F8391013791F29DBB207D828480078C6
:10BD800020B16018013184F8391003760223D37092
:10BD900010BD5906C3D4917801F0100101F0FF00E5
:10BDA0000029DDD013F001031ED194F85C1094F843
:10BDB0005D00884281BF4B1C091984F85C3091F802
:10BDC0003B3013712369D0229A702269DEE7236920
:10BDD00084F83920C0229A702369114A1979012107
:10BDE00011700222DA7010BDC0239370226913799A
:10BDF000CCE70122002384F85D2084F83B30A1E7E2
:10BE0000626994F86130094913440322187A02F0F8
:10BE100075FA2269ACE7626994F861300449F3E786
:10BE2000089FFF1F008EFF1F6C8EFF1F91BE00003A
:10BE30009DBE00000369DB7803F0200373B190F826
:10BE400060300133DBB2012B80F860301AD94269CF
:10BE500090F861301344187A02F0CCBA70B5426998
:10BE600003F0FF0590F8613013440446187A02F09D
:10BE7000C1FAA36E5BB184F8385094F83900BDE87C
:10BE80007040184790F85F30002BE0D0704770BDCD
:10BE90000148FFF7CFBF00BF008EFF1F0148FFF72B
:10BEA000C9BF00BF6C8EFF1F2DE9F047374FDFF889
:10BEB000E0903B68026982B006460093DDF800809E
:10BEC0000021A025D3789B065BD53B680193019B9D
:10BED000C8EB03030F2BF5D949B1102BF2D000208A
:10BEE0009070336980229A7002B0BDE8F087726961
:10BEF00096F8613013440521187A02F0F3FB726959
:10BF000096F861301344012193F812A0504602F0D4
:10BF1000E9FB09240021504602F0D0FB2B46013BEF
:10BF2000FDD10121504602F0C9FB2B46013BFDD15A
:10BF3000013CEFD1706996F8611001444FF4A07292
:10BF40000C7A4B7B09EBC4011B02496803F4E063E4
:10BF500043F064030B6096F862300344997CDB7D08
:10BF600009EBC1011B02496803F4E06343F0640379
:10BF70000B60013AFDD13269D3789B064FF0010185
:10BF8000A3D4012002B0BDE8F08700BF109FFF1FBF
:10BF90004C2E0100F0B503691222DA700269937821
:10BFA00003F0200385B004460D46002B5ED0B42379
:10BFB00093703C4922690B680093009E05E00B6872
:10BFC0000193019B9B1B042B42D8D37803F02003E1
:10BFD00003F0FF00002BF2D094F85D30002B31D03D
:10BFE0004FF0000E4FF0020C04EB0E0393F83B30C1
:10BFF00013710B680393039F206907E09B060DD51F
:10C000000B680293029BDB1B052B28D8C378DBB29D
:10C0100003F0020202F0FF06002AEFD080F803C00E
:10C020002669F378DBB2DF0632462DD49F062BD586
:10C03000DB0731D40EF1010E94F85D305FFA8EFE0D
:10C040007345D1D800201DBB002384F85E3004E086
:10C050009070236980229A70042005B0F0BD86702C
:10C060002369802204209A7005B0F0BD03F0FF061A
:10C07000FFF71AFF10B9042005B0F0BD236984F85A
:10C080005F60B0229A7094E78023B3700420DAE7EF
:10C0900026698023B370D7E7BEF1000F0CBF0220E2
:10C0A0000320F6E7109FFF1F2DE9F04106690025E8
:10C0B000122780F8385080F83950F770D0F810C047
:10C0C0009CF802E00EF0200E88B004468846154623
:10C0D0001E46BEF1000F49D0B4238CF80230784BD5
:10C0E00021691A680092DDF800E006E01A68019202
:10C0F0000198CEEB0000042830D8C87800F020006A
:10C1000000F0FF070028F1D04FEA480242F0010298
:10C11000D2B20A711A680292DDF808E0206906E0DE
:10C120001A6803920399CEEB010105292AD8C17838
:10C1300001F0020101F0FF070029F1D04FF0020CDD
:10C1400080F803C02269D17811F0110722D12DBBEC
:10C15000002E0CBFA0238023937003E08F7023690F
:10C1600080229A70384608B0BDE8F0810EF0FF07D3
:10C17000FFF79AFE0028F5D0236984F85F70B0229B
:10C180009A70ACE787702369802238469A7008B0AD
:10C19000BDE8F081802393700027E3E7012D75D07F
:10C1A000A021917021690A79BE4667464FF0A80C1C
:10C1B0001A680492049805E01A680592059A121A02
:10C1C000052A4AD8CA7802F0020202F0FF08002AC3
:10C1D000F2D0CF702169CA78D2B212F0100F08469F
:10C1E0005AD1920658D5013DEDB2012D49D0BEF18C
:10C1F0001F0F3BD90A79012DDAD11A680692069DE4
:10C2000005E01A680792079A521B052A46D8C27899
:10C2100002F0020202F0FF01002AF2D00223C370F2
:10C220002269D378DBB2D9063AD49B0634D5B02341
:10C23000BEF11F0F93703FD8226904EB0E031279F1
:10C240001A760EF1010E5FFA8EFE16B12369802276
:10C250009A7084F839E0774684E781F80280236990
:10C2600080229A70774684F839E07BE704EB0E026F
:10C2700091F8048082F818800EF1010E5FFA8EFEAC
:10C28000B9E781F802C021690846B0E7A82191709A
:10C290002069BE460279B0E7774663E78170DEE742
:10C2A0001021A023D170013BFDD12269937803F0C6
:10C2B000F7037746937055E723691B79C5E700BFFD
:10C2C000109FFF1F0148FFF71FBD00BF008EFF1F1B
:10C2D0000148FFF719BD00BF6C8EFF1F704700BFFC
:10C2E00038B5144C037801225B000546204684F8DB
:10C2F0003B3084F85E2084F85D20FFF78BFC2046FD
:10C300000021FFF747FE0B4C2978012320461A46EF
:10C31000FFF7CAFE0128F6D194F8383094F8392096
:10C320009A4205D9E218013384F83830107E38BDBE
:10C33000FF2038BD008EFF1F38B51B4C037801224B
:10C340005B000546204684F83B3084F85E2084F884
:10C350005D20FFF75FFC20460021FFF71BFE124C1B
:10C360002978204601230222FFF79EFE0228F6D1FB
:10C3700094F8382094F839108A420FD2531CDBB25B
:10C38000A018994284F83830007E0AD9234402323A
:10C390001B7E84F8382040EA032038BD4FF6FF703A
:10C3A00038BD40F47F4038BD008EFF1F0C2901D9F5
:10C3B000002070470231490001F0FE01FFF7BCBFC9
:10C3C00070B50C4C0378164601255B00204684F8B6
:10C3D0003B3084F85E5084F85D50FFF71BFC31461B
:10C3E0002046FFF717FC29462046BDE87040FFF7BE
:10C3F000D1BD00BF008EFF1FF8B505460F4616469B
:10C40000412421463A462846FFF7DAFF611C0234F0
:10C41000C9B232462846E4B2FFF7D2FF592CF0D118
:10C42000F8BD00BF38B504460D463548FFF706FC99
:10C430006322802120462570FFF7C2FF012002F011
:10C4400079F9204600225E21FFF7BAFF20465D21E0
:10C45000FFF746FF242801D0002038BD20460622E1
:10C460000C21FFF7C9FF204601222B21FFF7A8FF6F
:10C47000204601222C21FFF7A3FF20460E222D216A
:10C48000FFF79EFF204600222E21FFF799FF20464E
:10C4900001222F21FFF794FF204605223021FFF7CC
:10C4A0008FFF204601223121FFF78AFF204600221C
:10C4B0003221FFF785FF204600223321FFF780FF5E
:10C4C000204600223421FFF77BFF20460022352141
:10C4D000FFF776FF204600225B21FFF771FF204621
:10C4E00010225C21FFF76CFF204620225D21FFF720
:10C4F00067FF20468F225E21FFF762FF012038BDD3
:10C50000008EFF1F10B4047F4160022CC26002D075
:10C5100010BC03F091BA836810BC1847F0B4464BC6
:10C52000464A186BDC6A01791170454922790A7014
:10C530009A6A00790870002A46D05968C9688A4208
:10C540003ED82168CC8B240402F1FF3065D4C0F3BF
:10C550000E00C883C88B80B2C882196B0968C88B6B
:10C56000000452D4C2F30E00C883C88B002480B2EA
:10C5700012F1FF32C88218BF01229C62D96A2E488C
:10C5800009680D6800F12404A54236D00068C4682B
:10C5900014F0804F0C680D6815BF2488247802358C
:10C5A000013544F000440D604463196B254B097953
:10C5B0001970214912B1CA6A12791A70F0BC704719
:10C5C000521A9A620122D9E7586B196805681E4C05
:10C5D0000A63CC62CC682D681C4E24F0804403278B
:10C5E000B542CC6083F825701FD1037F4260022BD7
:10C5F000C2601ED0F0BC03F01FBA016890F824009E
:10C60000CC6840F000404863CFE7CC8BC2F3080011
:10C6100004F47E442043C883A7E7CC8BC0F3080012
:10C6200004F47E442043C88394E72B461146F0BCB3
:10C6300018478368F0BC1847D88EFF1F1F80004042
:10C640001C8000401B80004000000FFF05C500005B
:10C6500090E80C00F0B41C6859682568164F174E16
:10C6600029432160164D17491760D6601561116086
:10C67000417A154A5C180A3194F8244053F8215045
:10C6800002EBC40149680D60017A5C1803EB81017B
:10C69000247ECD6902EBC40149680D60817A581887
:10C6A00003EB810390F83000596B02EBC002F0BC41
:10C6B00053681960704700BF01401F000110003827
:10C6C0000110007800001F804C2E0100704700BF51
:10C6D0002DE9F04F85B09946BDF93870BDF83CA002
:10C6E000BB1AC1EB090B002BB8BF5B42BBF1000FBB
:10C6F000B8BFCBF1000B5B450D4616460093804654
:10C7000048DC4D453A4633464CDC194613460A464A
:10C71000C5EB09019B1A89B2002B0CB2B8BF5B4272
:10C7200004EBD474BE42ACBF4FF0FF3201224D4542
:10C73000039102924FEA640429DC9BB201930DE05D
:10C74000D8F80070BF69B847019BE41AA3B21CB2C5
:10C750000135002C2DB211DBA94518DB009B5B4590
:10C760002A46534631464046EADCD8F80020534674
:10C770009769294632464046B847E5E7029A16448B
:10C78000039AA94502EB030436B224B2E6DA05B0F7
:10C79000BDE8F08F4A462B46B94635464D4517460B
:10C7A0001E46B2DD304629463E464D46074689467E
:10C7B000AEE700BF10B404682469A44610BC60470B
:10C7C00030B40468BDF808500295A46BA44630BC90
:10C7D000604700BF30B40468BDF808500295E46BB0
:10C7E000A44630BC604700BF70B40468BDF90C605B
:10C7F000BDF8105003960495246CA44670BC6047A5
:10C80000704700BF10B582B0B0F90C2001910168EB
:10C81000009200220C6CB0F90A301146A04702B019
:10C8200010BD00BF704700BF01F003010129C175B1
:10C8300006D0032904D0C2880389428183817047CE
:10C840000289C38842818381704700BF2DE9F0418E
:10C850000568134E6F6986B0B7420446BDF8308054
:10C8600010D1013B13441BB20093CDF804800B465A
:10C87000AD6A2046A8472368DB6AB3420AD106B0F6
:10C88000BDE8F081059304920391B84703A9256898
:10C890000EC9E6E7204606B0BDE8F041184700BFE4
:10C8A00001C800002DE9F0410568124E6F6986B09D
:10C8B000B7420446BDF830800FD1013BCDF804806B
:10C8C0000B4400921BB2AD6A2046A8472368DB6A7E
:10C8D000B3420AD106B0BDE8F081059304920391FA
:10C8E000B84703A925680EC9E7E7204606B0BDE8AA
:10C8F000F041184701C800002DE9F04F0568DFF846
:10C9000058B06F6985B05F450646BDF93890BDF8EF
:10C910003CA00C46904615D11F19BC420CDACDF84C
:10C9200000A0214601342D6A4B464246304624B2CF
:10C93000A847BC423568F2DBEB6A5B4507D105B01E
:10C94000BDE8F08F0393B8473568039BE4E73046B2
:10C9500005B0BDE8F04F184701C800002DE9F043CD
:10C9600087B099420546BDF93840BDF83C6025D0F6
:10C97000A24212D00768DFF88080D7F81490C14532
:10C9800032D18DE850002846BC6AA0472B68DB6A8C
:10C99000434524D107B0BDE8F083994202DD084643
:10C9A0001946034628680E96C46B01335B1A1BB206
:10C9B0002846A44607B0BDE8F0436047A24202DD26
:10C9C000134622461C4628680E96631C846B9B1AED
:10C9D0001BB22846A44607B0BDE8F043604728468E
:10C9E00007B0BDE8F0431847059304920391C84788
:10C9F00003A92F680EC9C4E701C800002DE9F04F54
:10CA0000D0F800E0DFF89090DEF814B083B0CB45AA
:10CA10000446BDF93080BDF834A00D4617461E46C9
:10CA200031D1CDF800A0DEF824B0294633463A468D
:10CA30002046D8472368CDF800A008F1FF323A44D9
:10CA4000D3F824B0294612B233462046D84723688B
:10CA5000CDF800A02946D3F820B03A4643462046F8
:10CA6000D8472068CDF800A0711E29444346056AC6
:10CA700009B23A462046A8472368DB6A4B4506D1EF
:10CA800003B0BDE8F08FD847D4F800E0C9E72046EE
:10CA900003B0BDE8F04F184701C80000F0B400240F
:10CAA00001264FF6FF75094F07600471C475C481F4
:10CAB00004824476C4618675067685824582C1808B
:10CAC000028141818281F0BC704700BF682801006B
:10CAD0002DE9F04F85B00668BDF84450BDF93880A7
:10CAE000CDF8008004460195D6F848B00392BDF910
:10CAF0003C60BDF9407089469A46D8472368019545
:10CB0000009742465146D3F8488020463346C047F6
:10CB10002068039B0E930F95856C4B463A46314631
:10CB20002046AC4605B0BDE8F04F60472DE9F04F18
:10CB300087B01746BDF9404000912546E91D059391
:10CB400044BF2B4603F10E010268BDF848605369EB
:10CB50000294C91003912B49BDF9444001968B42C0
:10CB6000824645D1002C3CDD029B3C445E1EB6B2A1
:10CB70004FF0000923B2049301364D46029B002B6F
:10CB800028DD059B002403EB090806E0EDB22B0627
:10CB900004F1010411D4A6421CD0A1B211F0070F78
:10CBA00023B24FEA4505F1D1002BB8BF0733DB10A4
:10CBB000013418F803502B06EDD5009BD2F818B0BD
:10CBC00019443A4609B2019B5046D847A642DAF8C2
:10CBD0000020E2D1039B01379944049B3FB2BB4242
:10CBE000CCD1D36A074A934206D107B0BDE8F08F93
:10CBF0009847DAF80020B5E7504607B0BDE8F04F97
:10CC0000184700BF01C8000070B4BDF90C60BDF941
:10CC10001050BDF8144003960495059470BCFFF7BE
:10CC200085BF00BF2DE9F04F93B090460591C169D3
:10CC30001090BDF870000790BDF874909DF878A032
:10CC40000493002900F0CD800A7A0AC98946049924
:10CC50008A1AD2B203EBC203BAF1010FDA780B924F
:10CC600093F905201E8893F802B00F9293F90640BD
:10CC700079D913B2099323B20C93109B1A68A94B6C
:10CC80001193194653698B4240F0A6800B9B002BF1
:10CC900055D01FFA88F300210D93C8462344DDF8D0
:10CCA000409006910E930F460C46BBF1000F3FD00B
:10CCB000BDF818100C9B03971FFA8AF0CB1813FBD2
:10CCC00000F304900E9801440D98034409B21BB27E
:10CCD0000A910893002505E00135EBB264009B45FD
:10CCE000E4B222D9039B2B44590703D1731C18F8D3
:10CCF00006409EB22306EFD5099BBDF81000E91847
:10CD000011FB00F10598BAF1010F0FFA8AF3014403
:10CD10001CD0079801900093D26909B21746484683
:10CD2000089AB847D9F80020D6E7039F5F44FFB2BE
:10CD3000069B0B9901330693DBB29942B5D8D36AAF
:10CD4000119A934243D113B0BDE8F08F0F9B19188D
:10CD500093690A9A29441F4609B2079B4846B84777
:10CD6000D9F80020B8E700230C93099385E70A9AC5
:10CD70000D9B0132013B52B213F0FF030A920D9357
:10CD80006FD1DDF81890079BDDF83C80DDF820A01E
:10CD90004B4517D0BAF1010F00F0C8800B9A109DD7
:10CDA000CDF804900BEB8B014FEACB030A440093C0
:10CDB0001146DEF81C405346424609B22846A047B9
:10CDC000D5F800E0DEF82C30119A9342BBD01098D1
:10CDD00013B0BDE8F04F1847109D284698472A68C1
:10CDE00054E7109A0598B2F90A308342ABDDB2F9E4
:10CDF0000C304345A7DD062313FB0A03002BA2DDFD
:10CE000008EBCA03002B9EDD537E2BB9049BAF2B8E
:10CE100002D90133DBB20493109BD3F800E0414BFD
:10CE200011931A46DEF81430934240F08E801FFAB8
:10CE300088F30E9308339BB2BDF8142005930523A5
:10CE40000D9300230A93CDF83C800FFA8AF3DDF8A6
:10CE50004080CDF818900B921FFA8AFBCDF820A0E5
:10CE600099460A9ABDF810000B9C0E9D05231946A1
:10CE700011FB00232C481146C75C039702FB0B42B1
:10CE800014FA81F312B21BB209920C932C462E466F
:10CE90001CE0089B0999012B2AB24B4640462DD035
:10CEA000079F0197CDF80090DEF81CA0D047D8F876
:10CEB00000E0039B5B0801340393059BA4B25D442F
:10CEC0005E44A342ADB2B6B23FF451AF039BD80764
:10CED000DFD4079B069A9342EBD0089B012B16D018
:10CEE000069B0193CDF80090DEF81CA009994B46F3
:10CEF00032B24046D047D8F800E0DAE7DEF818A0B2
:10CF0000079B0C9922B2D047D8F800E0D1E7DEF8B1
:10CF100018A00C991346404622B2D047D8F800E03A
:10CF2000C7E700BF01C80000B82801000B99109D99
:10CF3000CDF800900531DEF8204009B242460823C2
:10CF40002846A047D5F800E03CE7109C20469847CB
:10CF5000D4F800E06BE700BFF0B5C36985B00446C4
:10CF60002BB30A2968D00D294AD01A7A914247D3A7
:10CF7000587A884244D35D688A1A05EBC205AA78BC
:10CF8000002A50D0E87800284DD0207E00283AD0E2
:10CF900095F905E0B4F90E00A67DB4F90A70724463
:10CFA00006FB0202BA4262DCB4F9102030E00A2922
:10CFB00056D00D2924D0027E002A4BD0B0F90E00A5
:10CFC000A57DB4F90A60062212FB0502B2423EDDDD
:10CFD000228AE38102EBC50212B218462282A78A96
:10CFE000668A02950B468DE8C00001462046FFF791
:10CFF00019FEA37DE28903EB430302EB4303E381C4
:10D00000012005B0F0BDA67DB4F90E00B4F91020E2
:10D01000B4F814E0678A02960B468DE8804001461A
:10D020002046FFF7FFFD2979E389A27D012001FB5E
:10D030000233E38105B0F0BD0022C2819A7A817D7E
:10D04000038A01FB02330382012005B0F0BDB4F96D
:10D050001020C4E7857DB4F91020B0F90E00BEE7BA
:10D06000028A817DC38102EBC1030382C8E70020ED
:10D07000E0819B7A228A03FB062212B22282C7E752
:10D08000C1810282704700BF002908BF012181755C
:10D09000704700BF81824182704700BFC07D7047EA
:10D0A000B0F90A00704700BFB0F90C00704700BF2C
:10D0B000F0B5C47DBDF81450022C75D0032C6ED091
:10D0C000012C32D0002A79DBB0F90840944265DDAA
:10D0D000002978DBB0F906605818B042C4BF731A53
:10D0E0001BB2002B5ADD002A1046B8BFD01D012408
:10D0F00040F3CF0002F00702704E01EBC01104FABA
:10D1000002F2A5423144D2B200F0A480C0F0958072
:10D11000022D43D1013B11FA83F04B1E13F8011F7E
:10D12000514083421970F9D1F0BDC488013CA21A64
:10D1300012B2002A7BDBB0F9064094422EDD0029B2
:10D140003DDBB0F908605818B042C4BF731A1BB277
:10D15000002B23DDC9B2C808584C02EBC01211F0F5
:10D160000701DBB204EB020039D0C1F10801C9B2FA
:10D17000534E8B42765C2AD2C3EB010EFF2747FA4F
:10D180000EF7012D06EA070674D06ED3022D40F08B
:10D190009480A75C7E40A6548B421DD2F0BD0489CA
:10D1A000E41A611A09B2C4E70689C488013EB21ABA
:10D1B000E41A12B2611A002A09B285DAF0BD0B44F2
:10D1C0001BB20021BDE70B441BB2002182E7012DF9
:10D1D00050D04AD3022DDCD05B1ADBB28030072B53
:10D1E00018D9022D4ED0A3F10806C6F3C406B11C0F
:10D1F00000EBC111012D0CBFFF24002400F18002BF
:10D2000002F8804C80328A42FAD1013600EBC61017
:10D2100003F00703002BC1D02A4A012DD35C2DD087
:10D2200006D3022DBAD1027853400370F0BDF0BD91
:10D23000027822EA03030370F0BD013BD24311FAE6
:10D2400083F0D2B24B1E13F8011F114083421970B4
:10D25000F9D1F0BD013B11FA83F04B1E13F8011F09
:10D26000114383421970F9D1F0BDA75C27EA060685
:10D27000A65491E7A75C3E43A6548DE7027813437A
:10D280000370F0BDA3F10805C5F3C405AC1C00EBA9
:10D29000C41400F1800212F8801CC94302F8801CFB
:10D2A0008032A242F7D1013513F0070300EBC5101D
:10D2B0003FF474AF034AD35CB5E7F0BD208FFF1F86
:10D2C000188FFF1F108FFF1FF0B5C47DBDF81450DD
:10D2D000022C76D0032C6FD0012C37D000297ADBBA
:10D2E000B0F906408C4230DD002A79DBB0F90860E5
:10D2F0009818B042C4BFB31A1BB2002B25DDD2B2BE
:10D30000D008754C01EBC01112F00702DBB204EB40
:10D31000010071D0C2F10802D2B2704E9342B65CE5
:10D3200062D2C3EB020EFF2747FA0EF7012D06EA81
:10D33000070600F0AC80C0F0A580022D40F0CA8046
:10D34000675C7E406654934253D2F0BDC488E41AB1
:10D35000A21A12B2002977DBB0F908408C42F4DD42
:10D36000002A39DBB0F906609818B042C4BFB31A7E
:10D370001BB2002BE9DD00290846B8BFC81D0124F7
:10D3800040F3CF0001F00701534E02EBC01004FA46
:10D3900001F1A54206EB0002C9B268D05AD3022DB2
:10D3A000D3D1013B12FA83F0531E13F8012F4A40E8
:10D3B00083421A70F9D1F0BD0489013C611A09B2A7
:10D3C000C8E7C6880489013E711AE41A09B2A21A94
:10D3D000002912B284DAF0BD13441BB20022C1E767
:10D3E00013441BB2002281E7012D50D04AD3022DF5
:10D3F000A6D09B1ADBB28030072B18D9022D4ED055
:10D40000A3F10806C6F3C406B11C00EBC111012D3F
:10D410000CBFFF24002400F1800202F8804C80320F
:10D420008A42FAD1013600EBC61003F00703002B45
:10D430008BD02B4A012DD35C2DD006D3022D84D165
:10D44000027853400370F0BDF0BD027822EA030376
:10D450000370F0BD013BC94312FA83F0C9B2531EF9
:10D4600013F8012F0A4083421A70F9D1F0BD013B35
:10D4700012FA83F0531E13F8012F0A4383421A70E5
:10D48000F9D1F0BD675C27EA060666545BE7675C86
:10D490003E43665457E7027813430370F0BDA3F18F
:10D4A0000805C5F3C405AC1C00EBC41400F18001F1
:10D4B00011F8802CD24301F8802C8031A142F7D1A1
:10D4C000013513F0070300EBC5103FF43EAF044AEB
:10D4D000D35CB5E7F0BD00BF208FFF1F188FFF1F83
:10D4E000108FFF1FF8B50D1E06DB14461F460646BB
:10D4F000FFF7D6FD854200DBF8BD002CFCDB304693
:10D50000FFF7D2FD8442F7DA3046FFF7C7FD022865
:10D510004BD0032843D0012804D1F388013B1B1BC7
:10D520002C461DB2012F03D026D3022F12D0F8BDF6
:10D53000002C2346B8BFE31D43F3CF0305EBC3150F
:10D540001E4804F00704435D012101FA04F41C4362
:10D550004455F8BD002C2346B8BFE31D43F3CF0369
:10D5600005EBC315154804F00704435D012101FADA
:10D5700004F45C404455F8BD002C2346B8BFE31DBD
:10D5800043F3CF0305EBC3150C4804F00704435DD8
:10D59000012101FA04F423EA04044455F8BD338957
:10D5A000013B5B1B25461CB2BCE7F188328901397F
:10D5B000013A4D1B141B2DB224B2B3E7208FFF1F7D
:10D5C00038B5402204460D468021FFF767FAFF2355
:10D5D000064A84F8255084F8223084F8263084F8EE
:10D5E000243084F823302260204638BDC02D01004D
:10D5F0004FF480620021014804F054BB208FFF1FCC
:10D60000F8B590F92230013304460F4642D001218B
:10D6100090F8260001F052F8002194F8240001F05F
:10D620004DF8002194F8260001F048F894F82730CE
:10D6300083B1254B1A684FF00043D3625763D36A16
:10D64000002BFCDA936B94F826000121BDE8F8402A
:10D6500001F034B808268025002194F8230001F059
:10D660002DF817EA05034FF0010194F8220008BFD6
:10D67000194601F023F8012194F82300CD4001F070
:10D680001DF8013EE8D194F826000121BDE8F840DC
:10D6900001F014B80D4C90F8203001255B002046B5
:10D6A000002184F83B3084F85E5084F85D50FEF72A
:10D6B000B1FA39462046FEF7ADFA29462046BDE8C4
:10D6C000F840FEF767BC00BFD88EFF1F008EFF1F1B
:10D6D000F8B50D4690F9221080F82020013104465B
:10D6E00080F821501F4600F0AD80012190F8240001
:10D6F00000F0F8FF012194F8260000F0F3FF94F801
:10D700002730002B00F0D380804E3046FEF7A0FF7C
:10D71000F37A002B40F0DB8033687D4AD968914270
:10D7200006D07C4E7C487D491E60DA601861196025
:10D73000E7B194F92500002818DBC0B2012100F000
:10D74000D1FF012194F8250000F0B8FF012000F07E
:10D75000F1FF002194F8250000F0B0FF0A2000F04E
:10D76000E9FF012194F8250000F0A8FFAE21204632
:10D77000FFF746FFD5212046FFF742FF80212046D4
:10D78000FFF73EFFA8212046FFF73AFF3F21204642
:10D79000FFF736FFD3212046FFF732FF0021204656
:10D7A000FFF72EFF40212046FFF72AFF8D2120465C
:10D7B000FFF726FF012D4DD014212046FFF720FF53
:10D7C00020212046FFF71CFF00212046FFF718FF0D
:10D7D000A1212046FFF714FFC8212046FFF710FFC4
:10D7E000DA212046FFF70CFF12212046FFF708FF41
:10D7F00081212046FFF704FFCF212046FFF700FFDD
:10D80000D9212046FFF7FCFEF1212046FFF7F8FE64
:10D810002046DB21FFF7F4FE20464021FFF7F0FE13
:10D820002046A421FFF7ECFE2046A621FFF7E8FEE4
:10D8300020462E21FFF7E4FE2046AF21BDE8F84048
:10D84000FFF7DEBE3648FEF7F9F936493448FEF7F1
:10D850003FFA6DE720461021FFF7D2FE2046202137
:10D86000FFF7CEFE20460021FFF7CAFE2046A12189
:10D87000FFF7C6FE2046C821FFF7C2FE2046DA2188
:10D88000FFF7BEFE20461221FFF7BAFE2046812197
:10D89000FFF7B6FE20469F21FFF7B2FE2046D921B2
:10D8A000FFF7AEFE22212046FFF7AAFEB0E70121D6
:10D8B00094F8220000F016FF012194F8230000F0F4
:10D8C00011FF94F82730002B3FF432AF1CE772B6FB
:10D8D000F37AD8071A4606D51349F2680868024059
:10D8E000B2610A601A46990706D51049336908687B
:10D8F000F27A0340F3610B60530705D50C4A736954
:10D9000011680B403362136062B605E7D88EFF1FC3
:10D910000000013801403F000000017800003F8016
:10D92000008EFF1F801A060080E100E084E100E025
:10D9300088E100E02DE9F84F21210546FFF760FE60
:10D9400028460021FFF75CFE28467F21FFF758FE9E
:10D9500028462221FFF754FE28460021FFF750FEFB
:10D9600028460721FFF74CFE95F92230013349D0B4
:10D97000012195F82600DFF8E480DFF8E4B000F03C
:10D980009DFE012195F8240000F098FE002195F8F5
:10D99000260000F093FE08F580694FF0004A95F8E4
:10D9A000273018F8017F0BBB08268024002195F84A
:10D9B000230000F083FE17EA04034FF0010195F8FD
:10D9C000220008BF194600F079FE012195F82300D6
:10D9D000CC4000F073FE013EE8D1C845DFD195F898
:10D9E00026000121BDE8F84F00F068BEDBF80020FA
:10D9F000C2F82CA05763D36A002BFCDAC845936B9E
:10DA0000CDD1ECE7DFF85080124F00244FF0010930
:10DA100095F82030104888F85E905B00402188F827
:10DA20003B3088F85D90FEF7F5F804F11006B6B2C9
:10DA3000395D09480134A4B2FEF7ECF8B442F7D1DD
:10DA400001210548FEF7A6FAB4F5806FE0D1BDE8E4
:10DA5000F88F00BF208FFF1F008EFF1F1F8FFF1F3B
:10DA6000D88EFF1F38B50446104621700A491D465E
:10DA700003F01EFC01464FF07E5003F0CDFC074939
:10DA800003F016FCE56060602561656100F030FE22
:10DA9000E061204638BD00BFDB0FC9400024744957
:10DAA00038B503780446032B20D8DFE803F01A18B2
:10DAB0001002C168406903F0F1FA0D49054660683B
:10DAC00003F0AAFC0146284603F0A6FC38BD08492D
:10DAD000406803F0A1FCE16803F0EAFB38BDC068D0
:10DAE00038BDC168406903F0D9FA38BD002038BD9F
:10DAF0000024744970B504460E4600F0F9FD054651
:10DB0000E069281A03F080FBE3682361E561666140
:10DB1000A0610146606803F07FFC0146A0601048E8
:10DB200003F07AFC02F01AFF02F0BAFB03F062FA8B
:10DB3000054601464FF07E5003F0B0FA616903F0EC
:10DB4000B7FB21690646284603F0B2FB0146304682
:10DB500003F0A6FAE0602046BDE87040FFF7A0BFE2
:10DB6000000080BF844641EA000313F003036DD137
:10DB7000403A41D351F8043B40F8043B51F8043B90
:10DB800040F8043B51F8043B40F8043B51F8043B97
:10DB900040F8043B51F8043B40F8043B51F8043B87
:10DBA00040F8043B51F8043B40F8043B51F8043B77
:10DBB00040F8043B51F8043B40F8043B51F8043B67
:10DBC00040F8043B51F8043B40F8043B51F8043B57
:10DBD00040F8043B51F8043B40F8043B51F8043B47
:10DBE00040F8043B51F8043B40F8043B51F8043B37
:10DBF00040F8043B403ABDD2303211D351F8043BD7
:10DC000040F8043B51F8043B40F8043B51F8043B16
:10DC100040F8043B51F8043B40F8043B103AEDD285
:10DC20000C3205D351F8043B40F8043B043AF9D2D6
:10DC3000043208D0D2071CBF11F8013B00F8013BA9
:10DC400001D30B8803806046704700BF082A13D3B6
:10DC50008B078DD010F003038AD0C3F10403D21ACE
:10DC6000DB071CBF11F8013B00F8013B80D331F802
:10DC7000023B20F8023B7BE7043AD9D3013A11F882
:10DC8000013B00F8013BF9D20B7803704B784370ED
:10DC90008B78837060467047374A384913681B0693
:10DCA000FCD40B6813F08003F8D172B634490A78BB
:10DCB000002A5FD0334A3448F0B4344C1768066801
:10DCC0002568D4680C303E44143200681268304F26
:10DCD00035442C4420440244C2F34E022D4E2E48BB
:10DCE0002E4D2F4C42F400423A60376806682D688A
:10DCF0002C4A24680C303E44006812682A4F354490
:10DD00002C4420440244C2F34E02284E2848294D98
:10DD1000294C42F400423A60376806682D68274A69
:10DD200024680C303E4400681268254F35442C446A
:10DD300020440244C2F34E02224E2348234D244C79
:10DD400042F400423A60376806682D68214A246828
:10DD50000C303E440068126835442C442044024490
:10DD6000C2F34E021C4842F4004202600B7062B6DD
:10DD7000F0BC704762B6704724B0034024B00B403B
:10DD80000A9FFF1F38B003403CB0034040B003403F
:10DD90002CB0034058B003405CB0034060B0034077
:10DDA00064B003406CB0034030B0034038B00B4067
:10DDB0003CB00B4040B00B4044B00B404CB00B406B
:10DDC0002CB00B4058B00B405CB00B4060B00B4027
:10DDD00064B00B406CB00B4030B00B4030B42948FD
:10DDE000294A2A4B2A4D6024E121047011701B78C6
:10DDF000284C082B30D00A2B2748284937D00C2B29
:10DE00000CBF35223D2212232A60236002600B6082
:10DE1000234B24491B78244ABBB101230B601360B8
:10DE2000224B23491B78234A012B26D9042B0FD9D7
:10DE3000082B1ED9102B94BF862387230B601360F9
:10DE40001D4B01221A7030BC70470B601360E7E76E
:10DE500084230B601360F3E700F58E200F49083030
:10DE6000012213232A60236002600B60D0E739226D
:10DE7000F7E785230B601360E2E780230B601360F4
:10DE8000DEE700BF00400740014007402093FF1F2E
:10DE900008B003400CB0034008B00B400CB00B407E
:10DEA0000D9FFF1F20B0034020B00B402193FF1FA8
:10DEB00024B0034024B00B400A9FFF1F0C2830B44D
:10DEC00017D91023984228BF18461C46104A114DF6
:10DED0001178181A8C42287018D00F4913700B78DB
:10DEE00023B10E490E4A00230B60136030BCFFF7CC
:10DEF00075BF0A2802D90C231C46E7E7082802D977
:10DF00000A231C46E2E708231C46DFE730BC7047C3
:10DF10002093FF1F099FFF1F0A9FFF1F24B003408C
:10DF200024B00B4028282FD8334B2DE9F0411E5C3C
:10DF3000FF2E2BD0314B1B78002B2AD132062CD44C
:10DF400072B62F4D2F4C2F46012326602B7062B6E0
:10DF500072B623681B060CD43B781BB9F4E72B7808
:10DF6000002BF1D062B601F0B3FF72B62368180639
:10DF7000F5D5254B1B6800222A7062B6234A10781B
:10DF800043FA00F0BDE8F081002070470020BDE8B2
:10DF9000F081FFF781FE3206D2D572B61C4DDFF854
:10DFA0007C801C4C06F04007FFB206F03F06D8F814
:10DFB0000030DFB123F01003C8F8003001232660E1
:10DFC000134A2B7062B672B6236819060CD4137804
:10DFD0001BB9ECE72B78002BE9D062B601F078FF93
:10DFE00072B623681B06F5D50B4BC3E743F010034D
:10DFF000C8F80030E2E700BF102E01000A9FFF1FA3
:10E000000C9FFF1F00B0034010B00340099FFF1F8B
:10E010000B9FFF1F00B00B4010B00B400CB00B402B
:10E020000A4A0B49136843F4805313600B7843B9D1
:10E03000084BC0221A70084B80F30C0000B2188005
:10E040007047044B80221A70F5E700BF2C80044013
:10E050000D9FFF1F21C00C4000C00C40F0B51B4BB2
:10E060001B4E596818689A68DB6885B06C460FC407
:10E07000337899071DD5174A174C1378174913F0B1
:10E08000700318BF1370164A164B802717700026AE
:10E090003320032226706D4608701A7072B6043C55
:10E0A00045F001052046A84762B6237813F07003B7
:10E0B00009D10D4B064901E0013B02D00A78D20795
:10E0C000FAD505B0F0BD237005B0F0BD3C2E0100BF
:10E0D0000100024000000240040002400B00024028
:10E0E000070002400A000240410D0300B0F5006F36
:10E0F0000AD210B5094B1B78DB07044606D504F19C
:10E10000A0500078C0B210BD00207047FFF7A6FFF6
:10E1100004F1A0500078C0B210BD00BF0100024061
:10E12000B0F5006F17D238B50F4B1B78DA070D46E4
:10E13000044611D504F1A0500378AB420AD00B4A33
:10E14000137813F0700318BF1370074A0570137823
:10E15000DB07FCD538BD7047FFF780FF04F1A05006
:10E160000378AB42EBD1F5E701000240000002402A
:10E1700008B5104C08E0236859050DD423681A052A
:10E180000FD42368DB0411D423685803F3D500F0BF
:10E19000C3FD23685905F1D501F01EFF23681A0558
:10E1A000EFD501F0AFFF2368DB04EDD500F048FCAC
:10E1B000EAE700BF3480044008B5FFF7D9FF00BF8D
:10E1C000014B10221A80704700200540704700BFA5
:10E1D000094908B50B6830B16A461844A2F5805267
:10E1E000904202D20860184608BD03F06DFA0C2375
:10E1F00003604FF0FF3008BD2493FF1FFEE700BF10
:10E20000EFF3138070B9EFF310836BB9EFF305826E
:10E210005AB94FF48070EFF311832BB1984228BFA5
:10E22000184670474FF0FF3070470F2A01D8184644
:10E23000F1E7014BD05CEEE7F0E300E0704700BF90
:10E2400010B40F4B53F8302092F880422CB10123C8
:10E2500069B182F8803010BC704703EBC0035B6883
:10E260001A6841B922F002021A6010BC704782F8A5
:10E27000003110BC704742F003021A6010BC7047B6
:10E280004C2E01001C4A02EBC00301295B6811D02F
:10E2900004291BD052F83000002280F8802229B1D6
:10E2A000022920D0032922D01A6070474FF48072CF
:10E2B0001A60704752F830004FF4A27280F8801252
:10E2C0001A601A6822F020021A60704752F8301063
:10E2D0004FF4A272012081F880021A601A6842F09D
:10E2E00020021A60704740F203121A6070474FF420
:10E2F00081721A60704700BF4C2E0100212817D888
:10E30000F8B5042A13D8DFE802F0494C4F14460050
:10E310002C4872B6236823F4702343F08072C4F350
:10E3200084011643236040F82150266062B6F8BD90
:10E3300070474FF41026244B03EBC0030D465C6876
:10E34000216811F4E06134D0204B214A2149C3F8FF
:10E350009C2104F140422048C3F8A411A2F5922167
:10E360001E4FC3F8A0017C291D48C3F8A871C3F84B
:10E37000AC01CDD9A2F594237C2B18D9A2F5962314
:10E380007C2B19D9A2F598237C2B17D9A2F59A22B8
:10E390007C2A15D9F8BD4FF43026CCE74FF400267F
:10E3A000C9E74FF44026C6E74FF42026C3E70D48DF
:10E3B000AFE7FFF767FFC7E70B48AAE70B48A8E7F7
:10E3C0000B48A6E72893FF1F4C2E01000082FF1F79
:10E3D000F188FF1F9988FF1FC588FF1F6D88FF1FE9
:10E3E0004188FF1F6093FF1FB093FF1FE093FF1F43
:10E3F0000094FF1F1A4B03EBC00010B4426802F1F7
:10E400004043A3F592217C2905D9A3F594217C29C9
:10E4100013D8144900E0144972B61368134C23F062
:10E420008773C2F3840023F4803343F08073136056
:10E4300041F8204062B610BC7047A3F596217C29B4
:10E4400009D9A3F598217C2907D9A3F59A237C2B18
:10E45000F1D80749E0E70749DEE70749DCE700BFF5
:10E460004C2E01006093FF1F2893FF1F3DE2000028
:10E470000094FF1FB093FF1FE093FF1F30B4054BC4
:10E48000054D064C002210211A602A602060196098
:10E4900030BC704714D0034004D0034000D0034088
:10E4A000282838B52ED0002904464FDD5F4B1B7855
:10E4B000012505FA03F28A4202D8212837D938BD4E
:10E4C0000338C2B2012A3AD9202C4AD0192C48D09C
:10E4D000574A126802FB011222FA03F31D2800F2C8
:10E4E0009B80DFE800F0928B847D9999766F9999F3
:10E4F0009999999999999968615A53994C999999C7
:10E5000099999945494B1B780B2B08D90C2B1CBFAB
:10E510000C3B19410846BDE83840FFF781BDC3F107
:10E520000C0399400846BDE83840FFF779BD2946FD
:10E53000FFF786FE2946BDE83840FFF7A3BE3D4AF7
:10E54000126802FB011222FA03F3C7E72128B6D8AA
:10E550000021FFF775FE20460121BDE83840FFF796
:10E5600091BE354A126802FB011222FA03F3B5E7A5
:10E570003249334A0B604FF45173136038BD31494F
:10E58000314A0B604FF45173136038BD2F49304A44
:10E590000B6040F24443136038BD2E492E4A0B6095
:10E5A00040F24443136038BD2C492D4A0B6040F2C1
:10E5B0004443136038BD2B492B4A0B6040F244435F
:10E5C000136038BD29492A4A0B6040F24443136066
:10E5D00038BD2849284A0B6040F24443136038BDD7
:10E5E0002649274A0B6040F24443136038BD254951
:10E5F000254A0B6040F24443136038BD2349244A46
:10E600000B604FF45173136038BD2249224A0B60EE
:10E610004FF45173136038BD212C3FF650AF7F2962
:10E62000D4BF00210121204693E700BF0894FF1FBB
:10E63000088003400890034008800B4010800B4086
:10E6400048A0044018800B404CA0044018800340B0
:10E6500008B004401080034004B0044040800340F0
:10E6600018C004403880034014C004402880034090
:10E6700010B00440208003400CB0044030800340C0
:10E6800010C00440488003401CC004401890034060
:10E6900034900440109003403090044038B110286A
:10E6A00028BF1020044AC3B2107813707047024A82
:10E6B00001231078137070470894FF1F212801D898
:10E6C000FFF7BEBD704700BF212806D8044B53F8A2
:10E6D000303093F80002C0B270470020704700BF8E
:10E6E0004C2E0100212801D8FFF7CCBD704700BF98
:10E6F00072B60C490C4B0D4A1B680868126862B66A
:10E70000520102D5322B88BF01300949C3F5BB3312
:10E710004FF47A72FF33A1FB031302FB00F000EB0E
:10E7200093107047109FFF1F18E000E004ED00E019
:10E73000ABAAAAAA2DE9F843054672B6204F214B91
:10E74000214A1B683C68126862B6520102D5322B1E
:10E7500088BF013495B3C3F5BB331C4EDFF864901A
:10E76000DFF86480FF334FF47A72A6FB031302FBD9
:10E7700004F404EB931472B6D9F800103A68D8F890
:10E7800000E062B6C1F5BB33FF33A6FB03031EF006
:10E79000806FC4EB93134FF47A7002D0322988BF94
:10E7A000013200FB0233B3F57A7F04D3013D05D07B
:10E7B00004F57A74DFE701F08BFBDCE7BDE8F88352
:10E7C000109FFF1F18E000E004ED00E0ABAAAAAA2A
:10E7D000F8B52D4B2D49DFF8D0E0DFF8D0C02C4E36
:10E7E0002C4D2D4C2D4A2E4F4FF4000018604FF049
:10E7F000807018604FF0007018604FF080601860F3
:10E800004FF0006018600020086028234BF6FF716D
:10E81000CCF80010CEF80030336013602B6023601A
:10E820003B60B3629362092245F8242CC4F8D80FE8
:10E8300005F57F65C7F8D41F07F5FF2707F5FA67C9
:10E84000C6F8F83F2B6006F5FF26C4F8D42F05F56F
:10E85000FD2504F5FF24386006F2F4761148316096
:10E8600005F5FF6504F5FD642B6023600260FFF78A
:10E87000B5FA1920FFF75EFF00F05AFE40F21310C0
:10E88000BDE8F840FFF756BF08E100E00480034010
:10E8900014800340248003402C8003401C800340EC
:10E8A0003480034000800B400C800340088003400C
:10E8B0002DE9F84F214B1B6807460BB101221A7056
:10E8C000DFF888901E4D99F80040DFF884801D4ED7
:10E8D0000134272C8ABF4FF0000A5FFA84FA5446AD
:10E8E000AB462B78A34216D1FFF78AFC40281FDCE9
:10E8F00033791B06F5D59BF800300133272B86BFF3
:10E9000000221346DAB218F80330DBB2F3712A7032
:10E910002B78A342E8D00C490A4BFFB208F80470E8
:10E920000120AC22087089F800A0DA70BDE8F88FE9
:10E93000FF28D6DD01F0CCFAD3E700BF889FFF1F88
:10E94000859FFF1F00C00640849FFF1F8C9FFF1FF5
:10E950001C9FFF1F1C4BDFF894C01A681B49F0B5C1
:10E9600042F480521A4D1A60DFF884E0194F1A4EB3
:10E970001A4C00238CF800304FF451722B701F2872
:10E9800040F213358EF800303B70337025600A601A
:10E9900012D819460124124A124D117012485470AF
:10E9A00000212C27402693724FF40034917011748B
:10E9B000D7702E700460F0BDC0F34431C0F347142B
:10E9C00000F01F03E7E700BF348004400CC00440A0
:10E9D000199FFF1F859FFF1F849FFF1F08C00440D2
:10E9E00000C0064031E400E004E100E0189FFF1F92
:10E9F0008C9FFF1F034B1B68DB0401D5FFF758BF3B
:10EA0000704700BF3480044010B5044C237823B114
:10EA100001F05EFA2378002BFAD110BD849FFF1F0E
:10EA2000054A064B10781B78C0B2DBB2984238BF5B
:10EA30004030C01A704700BF189FFF1F199FFF1F6B
:10EA400030B42B4B1A7994061FD52A48DA7903780B
:10EA5000294901333F2B0978C8BF00238B42D2B22A
:10EA600003D0264CD9B2E2540170254A116861B135
:10EA7000244A1278D2B2934236BFC2F140029B1AA6
:10EA80009B18272BC4BF01230B70194AD378DBB224
:10EA9000180611D45A060DD5154B1B795B0609D5FE
:10EAA000194B1A491B6800220A7003B11A70104BE7
:10EAB0002C22DA7030BC704711790906EAD5144966
:10EAC00010480C780178C9B28C420DD04A1C272A14
:10EAD00084BF00210A460F4D054C98BFD1B2AA5CF5
:10EAE000D2B2E2710170D5E76C21D170D2E700BFDC
:10EAF00000C00640189FFF1F199FFF1F449FFF1F64
:10EB0000149FFF1F859FFF1F889FFF1F849FFF1F6C
:10EB10008C9FFF1F1C9FFF1F21282FD8184B195CAB
:10EB2000FF292BD0174B184ADFF870C003EBC00049
:10EB3000F0B54368DFF868E0144F154D154E00241A
:10EB40001C60DEF80030012043F020038840CEF83E
:10EB5000003014604FF4A07338602E60C2F800C01B
:10EB6000013BFDD113689B05FCD42023013BFDD163
:10EB7000094B09B233F8110080B2F0BD0020704794
:10EB80005C2F01004C2E010000500440085004404E
:10EB900004500440000002030051044080014A0078
:10EBA00038800440431E032B14D872B60A4951F82A
:10EBB000230068B170B4094C058834F81320466806
:10EBC00041F82360521B24F8132062B670BC7047D2
:10EBD00062B6704700207047E89FFF1FF8A1FF1F33
:10EBE000013803280BD872B6074B53F8203043B1D5
:10EBF00000205B680130002BFBD162B6704700201B
:10EC000070471846F9E700BF3CA0FF1FF0B472B68A
:10EC10001A491B4E012311F8014B194F9A00240782
:10EC200042F0010505D556F8324064B156F835205A
:10EC3000BAB10133052BEED162B6124B00221A7025
:10EC4000F0BC00F0F1BC0F4C0F4D217847F832506A
:10EC500007EB431308304A1E5860227062B6F0BCBE
:10EC600070470849094B0A7847F8353007EBC50368
:10EC70000830013A58600A7062B6F0E7B42F01001C
:10EC80000080FF1F65A0FF1F88004000C8004000F3
:10EC9000431E032B1DD81B4A400140F0100030B426
:10ECA000104472B6184CE25C032A1BD8DFE802F06D
:10ECB0000212151703220D88E25410F0080F14BF3A
:10ECC000C823882343EA054308310360416062B6E4
:10ECD00030BC704708300222EDE70522EBE7083030
:10ECE0000422E8E7094A52F8230038B1084A52F8EA
:10ECF0002300416042F8231062B6E9E742F823108E
:10ED0000034AF7E70080FF1F74A0FF1F3CA0FF1F0E
:10ED10004CA0FF1F00BE70472DE9F04FDFF814A391
:10ED2000DFF814B387B044E0AC4F4FEA930807EB29
:10ED3000C809013ED9F8042003F00803F6B2A2F195
:10ED4000080003F0FF04002B40F0FE8057F8383035
:10ED50001B0C99B222F8081C002B00F0EC80A04B91
:10ED600022F8064C42F8044C53F82620002A00F002
:10ED7000CD819C4D55F8263058609B4C45F82600B7
:10ED800034F81630194424F8161000F02DFC002831
:10ED900000F0C081954A964B19F0080F00F1080069
:10EDA00018BF1346C9F8040047F8383008238AF81A
:10EDB00000309AF80040E4B261071CD58D4B1B78F7
:10EDC000B3B18D490A7802F0FF0322B1013BDBB2F7
:10EDD0000B7003B900BE89490A7802F0FF032AB11B
:10EDE000013BDBB20B70002B00F0668100F092FC5F
:10EDF00004238AF8003004F0080303F0FF02002B1C
:10EE000000F0C6809BF80030DBB21E098CD19A0856
:10EE1000724F57F8321007EBC200C1F3830101397A
:10EE200040680C2900F28380DFE801F07878818166
:10EE3000818181814281818107000168704D714B20
:10EE400040680193694B47F832306F4E686040F27A
:10EE5000816288B26B4B29600024012190421C60C2
:10EE60003C61BC61317000F2E980B0F5D06F80F098
:10EE70000F82B0F5817F00F0DA8100F26B8180288B
:10EE800000F00182822840F0D881A8885F4B00F012
:10EE90007F00042800F2D2815D4A80000344147090
:10EEA00054701878840740F102831170022174E1D4
:10EEB000544B01931A6832B3564B534E5648198837
:10EEC0003478057840298E4645F0020828BF4FF077
:10EED000400E002C84F001043470CEEB01010CBF15
:10EEE0008824C82407EBC80689B285F0010544EAE6
:10EEF0000E447260198047F838407244057000294A
:10EF000066D0019B1A603E4B1A88B2F5A06F0ED1F5
:10EF100000219A785970414B1A7008E03849404CEA
:10EF20000D68A54200F09980304947F832103D4AFB
:10EF3000012313703AE72D4A2D4B19F0080F18BF23
:10EF4000134647F8383031E700F06EFB364A374950
:10EF500052F82630002B00F0E48058688C5D42F8AF
:10EF6000260003F10802C9F80420032C05D8DFE8C5
:10EF700004F02C02292602228A551A8819F0080F5B
:10EF80000CBF8823C82343EA024347F838300DE713
:10EF9000E00700F19480210600F1D280A20706D597
:10EFA000234A244913780220DBB213700870E30669
:10EFB00002D5204B10221A7007B0BDE8F08F042252
:10EFC0008A55DAE705228A55D7E703228A55D4E71E
:10EFD000BEF1400F18BF002293E700BF0080FF1F63
:10EFE000E89FFF1F949FFF1FF8A1FF1FC80040006C
:10EFF0008800400070A0FF1FF99FFF1F90A0FF1F17
:10F000005CA0FF1F909FFF1FF89FFF1FC0200740BD
:10F0100068A0FF1FA49FFF1F64A0FF1F9820074048
:10F0200021090003942007403CA0FF1F74A0FF1F8C
:10F03000882007408020074090200740B0F5106FDF
:10F0400000F03E8140F2A28040F62112904240F052
:10F050001C82A44A0123137069E74C68A2498C42C0
:10F060007FF462AF0178A9297FF45EAF417845292A
:10F070007FF45AAF8178C2297FF456AFC1786B29EB
:10F080007FF452AF99489A4E0178347881F00105A7
:10F09000002C41F0020105700CBF8820C82084F0CC
:10F0A000010447F8310007EBC10192483470002594
:10F0B00005244D60047037E700F09EFC96E68E4B09
:10F0C00088488A491A614FF0020E80F800E08B4FA1
:10F0D0000A708B49196099608A4E8B4D8B4C9A61EE
:10F0E0000D213970FF213170DFF848E2297022705C
:10F0F000874D884A8EF800109F27012406F8047C6B
:10F100005D600470DA6007B0BDE8F08F43F8260058
:10F11000814D32E6814A47F8380013780133137085
:10F1200044E68B5D032B00F2A78001A252F823F086
:10F13000ADED0000ADED000087F1000081F10000B1
:10F140006E49714B80220D2008701A70A2077FF55E
:10F150002EAF25E740F20232904240F08E81AA881D
:10F1600002F07F02042A68D86D88002D65D16348BB
:10F17000029192001044027842F00202027048E1CB
:10F1800001238B5512E600238B550FE6B0F5086F6F
:10F1900053D16348634A00781070ED888D4280F047
:10F1A0009B815248047844F0020C07EBCC01402DBF
:10F1B000AE464FF0010328BF4FF0400E4A6002EB0D
:10F1C0000E09CEEB05014FEA0E4802930025C82236
:10F1D00042EA080384F0010247F83C3035700270BF
:10F1E000DFF814C1424BDFF8048151BBBEF1400F80
:10F1F0007FF42FAF42F0020207EBC203DFF8F8E022
:10F20000C3F8049095BB0D0445F088059DF80830BF
:10F2100033704029047009EB01034EF832507FF43B
:10F2200018AF0021404A01981180036011E7AA88B5
:10F2300002F07F02042A40F22D81304B0F221A7017
:10F2400007E74029D6D942F002020CEBC200C0F811
:10F2500004907DB135489DF808501D70403988F8FC
:10F26000004009F140034CF83200DBE70D0445F0A3
:10F27000C805CBE72248EEE719F0080F0CBF0223C0
:10F2800003238B5592E5274A02211470547084E7BA
:10F2900027494A68002AD0D06C88B5F804E003E01A
:10F2A0000C314A68002AC8D00B88A342F8D14B8899
:10F2B0007345F5D1240A032C0CBF117809896CE73A
:10F2C000174A0D4CA978117004F1800502E008344A
:10F2D000AC4231D0236A1A06F9D5606A083800F0CA
:10F2E000A3F9F4E7942007400100040064A0FF1F85
:10F2F000F89FFF1FF99FFF1F0080FF1FC0200740DE
:10F300008800400088200740802007409820074060
:10F31000A89FFF1FFC9FFF1F949FFF1F65A0FF1F5B
:10F3200070A0FF1F68A0FF1FA49FFF1FC800400020
:10F33000B82F01008C2007406F49704B704A029132
:10F340007049714D714C059603954FF00009884640
:10F3500016461D460494286828B1446800F064F9F4
:10F360002046002CF9D100232B60039B30681A46FD
:10F37000002342F8293028B1446800F055F92046AE
:10F38000002CF9D100223260029A98F80030114620
:10F39000002241F8042B049A0291023B4FF0000135
:10F3A00022F81910032B07D8DFE803F047024702C1
:10F3B0004FF0010388F8003009F10109B9F1040F99
:10F3C00005F1040506F1040608F10108C3D1504B0C
:10F3D000059EDFF85491DFF8548100211970012552
:10F3E00018F8013B09F8043B1B072BD4AC0044F090
:10F3F000020244F00304002347F8323047F8343067
:10F40000444B994505F10105EAD13378029383F025
:10F4100001050021894688468E460A463E48047802
:10F4200044F0020C07EBCC030393029B002B039BDD
:10F430005A600CBF8822C822CAE64FF0000388F841
:10F440000030B9E700F0D0F8AC0007EB451300F14D
:10F450000802002837D05A60304B47F8343000F0AB
:10F46000C3F844F0010307EBC30200F1080100B345
:10F4700051602B4A47F83320B9E7B0F5A06F7FF40D
:10F48000DCAE012300250293C3E740F6212290421F
:10F49000F7D0D2E66D88002D7FF4CFAE21480291DF
:10F4A00092001044027822F002020270B1E70221B9
:10F4B00073E6174B44F001021B7847F83200144AF8
:10F4C0000133137093E7124B114A1B78AC000133E0
:10F4D00047F834001370C2E740298E464FF001030D
:10F4E00028BF4FF0400ECEEB01014FEA0E4802EB71
:10F4F0000E090025029391E74CA0FF1FE89FFF1F14
:10F500003CA0FF1F74A0FF1F949FFF1FF8A1FF1FC7
:10F5100065A0FF1FD420074064A0FF1F88004000A3
:10F52000C8004000C0200740C4200740B42F01009D
:10F530002DE9F843204C00F06BFE002204F1880016
:10F5400023461A605A60083383424FF00001F8D115
:10F550001A4A1B4F13681B4D1B481C4EDFF878805E
:10F56000DFF878C0DFF87890DFF878E043F48023A4
:10F570001360C4F307233B70C4F307432B70240EBE
:10F58000FF2302F528320470114D88F8003011482D
:10F590008CF80030D4323370012389F800307026A3
:10F5A0008EF800104FF40074102107F8183C2E70EC
:10F5B00004601170BDE8F8830080FF1F34800440B0
:10F5C0009C200740B0200740B4200740102007408F
:10F5D00049E400E008E100E080200740882007407F
:10F5E000942007400021074072B60D480268B2FA25
:10F5F00082F30F2B10DC4FF00041D94022EA0102C8
:10F60000026062B6074803EBC303DB00C2180021A7
:10F61000C15010465160704762B60020704700BF6D
:10F620000C94FF1FBC83FF1F0D4B0E4AC31AA2FB95
:10F6300003231B090F2B0CD80B4A127852B972B650
:10F640000A484FF00041026821FA03F31A430260AE
:10F6500062B67047064A1278002AF0D0FFF7D6BA91
:10F66000BC83FF1F398EE33865A0FF1F0C94FF1F7A
:10F6700070A0FF1F2DE9F843224E234F316801236C
:10F6800080463B70C1B1214D4B8801EB83000133B3
:10F6900000220F2BC0F808802A7004D84B8000236A
:10F6A0003B70BDE8F88340230B800320FFF7F0FA9E
:10F6B000FFF79AFF3060F2E7DFF8549099F80030D6
:10F6C000002BEED0114D45F6215408E0013C12D03C
:10F6D0002B7883B900F0FCFB99F800307BB1032054
:10F6E000FFF77EFA0528F1D8FFF77EFF014630606C
:10F6F0000028EBD0C8E701232B70BDE8F883BDE8F4
:10F70000F88300BF7CA0FF1F78A0FF1F80A0FF1F11
:10F7100070A0FF1F094B1B787BB910B5084C2168FE
:10F7200009B14B8803B910BD9B000B800320FFF784
:10F73000AFFAFFF759FF206010BD704778A0FF1F98
:10F740007CA0FF1F70B5124E33788BB1114D286825
:10F7500040B14388C218147A6CB9FFF765FF33785B
:10F760002C602BB10220FFF71DFA28600028F0D191
:10F770004FF0FF3070BD02880133934202D24380C4
:10F78000204670BDFFF750FF002320462B6070BD60
:10F7900070A0FF1F8CA0FF1F70B50D4E33788BB18A
:10F7A0000C4D286840B1438803441C7A6CB9FFF7BC
:10F7B0003BFF33782C602BB10220FFF7F3F9286070
:10F7C0000028F0D14FF0FF3070BD204670BD00BF63
:10F7D00070A0FF1F8CA0FF1F38B5164D2868E0B140
:10F7E00001884488A14213DD03191B7A83B104F117
:10F7F0000803C2180C1B002302E012F8011F21B1FC
:10F800000133A342F9D1204638BD1C46204638BDFD
:10F81000FFF70AFF0020286038BD074B1B780BB9A3
:10F82000002038BD0220FFF7BDF928600028D7D19D
:10F83000F6E700BF8CA0FF1F70A0FF1F2DE9F04F5F
:10F840003D4D012283B02A7071B3DFF8F8A0DFF8D4
:10F85000F880DFF8E89083460E46DAF800000028CA
:10F8600035D0364B01934488019BC4F14001B1422D
:10F8700028BF314667180022BFB21A70761A478037
:10F8800000F1080249B1013C224459441BF8014BE4
:10F8900002F8014F5945F9D147883F2F09D8284B25
:10F8A00005221A70002ED8D10020287003B0BDE8C0
:10F8B000F08F4022224B02800146002401201C7060
:10F8C000FFF7E6F9CAF80040002EC6D1ECE798F839
:10F8D00000204AB3194B019344F2D95401270BE09D
:10F8E000013C17D099F80020A2B92A7000F0F0FA74
:10F8F0002F7098F80020BAB10120FFF771F90528A0
:10F90000EED82F70FFF770FECAF800000028AAD1C9
:10F91000013CE7D10199012200234FF0FF300A702A
:10F920002B7003B0BDE8F08F00234FF0FF302B7039
:10F9300003B0BDE8F08F00BF81A0FF1F88A0FF1FAC
:10F9400090A0FF1F84A0FF1F70A0FF1F00B583B011
:10F9500002AB012103F8010D1846FFF76FFF03B05A
:10F960005DF804FB38B50E4D0E4C2B68012020705D
:10F970002BB1588800232370C0F1400038BD0A4BDA
:10F980001B7813B90020207038BDFFF729F905282E
:10F99000F8D8FFF729FE034628600028E9D1F1E7EF
:10F9A00084A0FF1F81A0FF1F70A0FF1F0F4B1B78BB
:10F9B000DBB110B50E4C2168B1B14B88A3B10D4835
:10F9C00000223F2B027007DC07330B4401F1470094
:10F9D00003F8012F8342FBD140230B800120FFF766
:10F9E00057F90023236010BD10BD704770A0FF1FA2
:10F9F00084A0FF1F90A0FF1F0D4B1B78BBB910B553
:10FA00000C4C216803F0FF024B883F2B07DC0733C7
:10FA10000B4401F1470003F8012F8342FBD140233F
:10FA20000B800120FFF734F90023236010BD7047DD
:10FA300081A0FF1F84A0FF1F10B4EFF3108272B6E5
:10FA4000437F33B9017F012907D003290FD0012358
:10FA5000437702B962B610BC7047124C2168A1B15D
:10FA6000114943610B68836108605861EFE70F4CEF
:10FA7000216881B10E4943610B6883610860586158
:10FA80000C4B4FF080511960E1E7074B41618161F8
:10FA900020601860DBE7064B4161816120601860DF
:10FAA000EEE700BFA4A0FF1FA0A0FF1F94A0FF1FB0
:10FAB00098A0FF1F04ED00E070B5EFF3108272B65E
:10FAC0000C4C206880B10C4E00254369236073B153
:10FAD0009D6102B962B6457783689847EFF310825B
:10FAE00072B620680028F0D102B962B670BD3360EA
:10FAF000EFE700BF94A0FF1F98A0FF1FFFF7DCBF38
:10FB0000184A30B41468002C27D0036821688B424F
:10FB10000ED2CB1A00218460C1602360E0601060C7
:10FB20000223037530BC704711688B42144608D31A
:10FB3000A2685B1A0360002AF6D18260C460A060EC
:10FB4000EEE7D268C2608460E060C568CB1A02222A
:10FB5000A8602360027530BC70478460C460106088
:10FB6000DEE700BF9CA0FF1FF8B5224E34682CB31F
:10FB70002368002B3AD1204F1D4604E03468ECB1D5
:10FB80002368002B32D1A36803B1DD6020693360A4
:10FB9000036825751B68BB4221D1037F4560022B9A
:10FBA000C46020D0FFF748FF6368002BE6D02360D5
:10FBB0002046FFF7A5FF3468002CE1D1EFF3108356
:10FBC00072B60E4A00211068116003B962B628B1FE
:10FBD0008468FFF795FF20460028F9D1F8BD22463A
:10FBE00000219847E0E783689847DDE7013B236001
:10FBF000E4E700BF9CA0FF1F05C50000ACA0FF1FED
:10FC0000024A136801331360FFF7AEBF109FFF1F56
:10FC1000F8B572B106460F4614460025336817F84A
:10FC2000011B1B6830469847013C0544F6D1284625
:10FC3000F8BD1546FBE700BF00B5064A0368128809
:10FC40005B6883B001A9ADF804200222984703B095
:10FC50005DF804FB802F0100F0B507468BB0002A49
:10FC600033D0012A08BF0A2251B3212400E0F4B2A4
:10FC7000B1FBF2F502FB1511C8B2092900F1300100
:10FC800098BFC8B20AA988BF3730214488BFC0B224
:10FC900001F8240C661E2946002DE8D133B1013C41
:10FCA000E4B20AAB23442D2203F8242C3B6801AABA
:10FCB00011195B683846C4F1220298470BB0F0BDB9
:10FCC00030228DF825202124E8E70368C9B21B689B
:10FCD00098470BB0F0BD00BF0029BABF49422D23A1
:10FCE00000230A22FFF7B8BF2DE9F04385B0804614
:10FCF0001946104616461F469DF8305001F01CF973
:10FD0000002840F0B18027F00044304621464FF0F3
:10FD1000FF32594B01F010F998B9304621464FF0A7
:10FD2000FF32554B01F0EAF858B9D8F80030534982
:10FD30005B684046032298478146484605B0BDE8C7
:10FD4000F083304639464FF060424D4B01F0EAF8FF
:10FD5000002870D1304639464FF06042494B01F0DF
:10FD6000C3F8002867D1304639460022002301F04D
:10FD7000BBF8002863D18146002D65D0424B00249A
:10FD80000022104619463AA3D3E9002300F03AFEB8
:10FD900001340B46E1B28D420246F2D83046394674
:10FDA00000F07EFC0F46064601F004F9044600F020
:10FDB000B3FD02460B463046394600F06FFC4B4619
:10FDC00006460F460A2221464046FFF745FF0F2D03
:10FDD00028BF0F2501352E238146EDB28DF8003066
:10FDE00001240022294B3046394600F00BFE0F4615
:10FDF000064601F0DFF804AB2344C0B200F1300244
:10FE000003F8102C00F098FD02460B4630463946A8
:10FE100000F044FC0134E4B2AC4206460F46E0D1A7
:10FE2000D8F8003022465B68404669469847484605
:10FE300005B0BDE8F083D8F80030154978E707F140
:10FE400000474FF0010997E700220F4B3046394633
:10FE500000F026FC01F0AEF84B4601460A2240466F
:10FE6000FFF7FAFE814668E7D8F8003009495FE7F6
:10FE7000000000A09999B93FFFFFEF7F8C2F010090
:10FE8000FFFFEF41FFFFEFC10000E03F0000244013
:10FE9000882F0100842F010008B5FBF7C1FAFBF79A
:10FEA000BBFA00F015F8FAE7FFF776BCFFF74ABC9B
:10FEB000FFF792BCFFF77ABDFFF754BD0846114625
:10FEC000FFF7BCBC0846FFF741BD00BF704700BF4D
:10FED00038B5224C237803B138BD01232370FFF7D6
:10FEE0007BFC70BB00F068F840BB00F0FBF810BB77
:10FEF000FEF796FDE0B900232370EFF30583002B96
:10FF0000EAD1EFF3108172B6154B1868E0B1154CC9
:10FF10002278CAB945691D6001232370C5B1AA6161
:10FF200001B962B600254577836898472570D3E705
:10FF300000F0B4F9DFE700F0AFF9D9E700F0AAF973
:10FF4000D3E7FFF7C3FFCDE70029C5D162B638BDBF
:10FF5000054B1D600029E5D1E3E700BFB0A0FF1FFE
:10FF6000A4A0FF1FA8A0FF1FA0A0FF1FF0B44D1E5C
:10FF70002E46002400E00134B0FBF2F302FB130034
:10FF8000092800F130078ABF3730F8B2C0B206F84E
:10FF9000010F1846002BEED10A1953704CB110789E
:10FFA00015F8016F28700133E01A834202F80169E5
:10FFB000F5DB0846F0BC7047054A064B10781B7805
:10FFC000C0B2DBB2984238BF4030C01A704700BFA1
:10FFD000B8A0FF1FB9A0FF1FF0B4384B1A7912F078
:10FFE000300F2CD072B6997D01F0FF0200293DD070
:10FFF00062B6334F334938780D78334E1C46C0B261
:020000021000EC
:10000000EDB2431C402BE17928BF0023AB4202F143
:10001000FF32C9B21CBFF154184612F0FF02F0D1F2
:100020002A4B1B68C2B23A704BB1A84236BFC5F129
:100030004005401B40192728C4BF01221A701F49E0
:10004000CA78D2B2150616D452060DD51B4B1B79B1
:100050005B0609D51E4B1F491B6800220A7003B1BD
:100060001A70164B3C22DA70F0BC70474022D979E6
:100070005A7462B6E3E70B791C06E5D5164B174EAA
:100080001C783378E4B2DBB29C420ED0144D01E010
:10009000A3420AD00133402B28BF00230879E85C33
:1000A000C0B2C871087D0728F2D9DBB203493370AA
:1000B0000B79180644BF7C23CB70C5E700A006402F
:1000C000B8A0FF1FB9A0FF1FFCA0FF1FB4A0FF1F17
:1000D00040A1FF1F3CA1FF1F44A1FF1F3DA1FF1F27
:1000E000BCA0FF1F054A064B10781B78C0B2DBB2DC
:1000F000984238BF4030C01A704700BFB8A1FF1FF8
:100100004DA1FF1FF0B4384B1A7912F0300F2CD0EC
:1001100072B6997D01F0FF0200293DD062B6334FDF
:10012000334938780D78334E1C46C0B2EDB2431CCB
:10013000402BE17928BF0023AB4202F1FF32C9B264
:100140001CBFF154184612F0FF02F0D12A4B1B6875
:10015000C2B23A704BB1A84236BFC5F14005401B50
:1001600040192728C4BF01221A701F49CA78D2B289
:10017000150616D452060DD51B4B1B795B0609D507
:100180001E4B1F491B6800220A7003B11A70164BE0
:100190003C22DA70F0BC70474022D9795A7462B6BA
:1001A000E3E70B791C06E5D5164B174E1C78337820
:1001B000E4B2DBB29C420ED0144D01E0A3420AD05F
:1001C0000133282B28BF00230879E85CC0B2C8712E
:1001D000087D0728F2D9DBB2034933700B79180682
:1001E00044BF7C23CB70C5E700B00640B8A1FF1F19
:1001F0004DA1FF1F78A1FF1F48A1FF1FBCA1FF1F3A
:100200004CA1FF1FC0A1FF1FB9A1FF1F50A1FF1FDD
:1002100070B584B072B6194B194D1A487022412638
:100220000F2480211A702E701A46047019701378EA
:100230001B06FCD5144B186862B6144B144C98423C
:1002400098BF00EB800001A998BF40000A22FFF789
:100250008DFE01A92046002311F8012B01333AB18C
:100260000A2B20F8022FF7D11623237004B070BD9B
:100270005B00DBB2237004B070BD00BF0000024021
:100280000700024006000240080002407F969800E6
:10029000E894FF1F704700BF704700BF704700BF62
:1002A0002DE9F043DFF8EC808BB006460F4600F0F6
:1002B00073F898F90030013304460D4637D03046C4
:1002C000394600F0DFF9002831D02BA3D3E9002311
:1002D0003046394600F026FE814668BB28A3D3E9A4
:1002E00000233046394600F0FFFD00B398F9003096
:1002F000254ACDF82090042400200021022BCDE9CE
:100300000467CDE9026700940192CDE906012CD083
:10031000684600F0BDF940B3089B1BB101F0D4F969
:10032000089B0360DDE906010BB0BDE8F0832046C1
:1003300029460BB0BDE8F083134A98F900300192CA
:1003400003210022CDE90467CDE9026700910892FC
:100350002BB90E4B4FF06042CDE90623D8E70C498C
:100360000020022BCDE90601D2D101F0ADF9222304
:100370000360D1E7AFF30080EF39FAFE422E8640EA
:1003800051302DD5104987C024300100FFFFEF47C1
:100390000000F07FFE94FF1F2DE9F04FB04F21F0D9
:1003A0000042BA4283B00C464FEAD17605460DD9D9
:1003B000AC4FBA4225D9C1F31303034340F0EF8099
:1003C0000EB10020014603B0BDE8F08FA64B9A4263
:1003D00000F2CC80A54B9A4200F2DE808AA3D3E9DA
:1003E000002300F05DF90022A14B00F09BFD0028E6
:1003F00000F005812846214600229D4B00F050F96F
:10040000E1E783A3D3E9002300F08CFD002840F04E
:10041000CB802846214680A3D3E9002300F064FD69
:100420000028CED1934B284603EBC60821467CA377
:10043000D3E9002300F0E6FAD8E9002300F030F910
:1004400000F090FD804600F077FA77A3D3E900230F
:1004500006460F4600F0D6FA02460B4628462146CD
:1004600000F01CF972A3D3E90023CDE90001304666
:10047000394600F0C7FA82468B4652465B46DDE9B4
:10048000000100F00BF905460C462A462346284693
:10049000214600F0B7FA68A3D3E9002306460F46C9
:1004A00000F0B0FA66A3D3E9002300F0F7F8324673
:1004B0003B4600F0A7FA64A3D3E9002300F0F0F86C
:1004C00032463B4600F09EFA61A3D3E9002300F0D8
:1004D000E5F832463B4600F095FA5FA3D3E90023E6
:1004E00000F0DEF832463B4600F08CFA02460B463E
:1004F0002846214600F0D2F806460F4628462146F7
:1005000032463B46B8F1000F56D000F07BFA324637
:1005100004460D463B4600204FF0804100F0BEF8F7
:1005200002460B462046294600F096FB02460B4643
:100530005046594600F0B2F8DDE9002300F0AEF86D
:100540000B4602464A49002000F0A8F86FF47F737A
:1005500098454FDA08F57A7801EB085100224FF000
:10056000B87300F04FFA03B0BDE8F08F424B9A42E7
:100570003FF658AF414BF4002344D3E9002300F089
:100580008DF83F4BC6F101081C44CDE90001D4E9C8
:1005900000ABC6EB080870E74FF0000875E70246AD
:1005A0000B4600F07DF80EE717A3D3E900231046B1
:1005B000194600F027FA06E700F024FA00228046E8
:1005C00089464FF080433046394600F067F80246CE
:1005D0000B464046494600F03FFB2A46234600F0C2
:1005E0005DF802460B460020214900F057F803B0A1
:1005F000BDE8F08F01EB085103B0BDE8F08F8046F5
:1006000043E700BFAFF300809C7500883CE4377E71
:10061000EF39FAFE422E864051302DD5104987C061
:10062000FE822B654715F73F0000E0FE422EE63FB5
:10063000763C7935EF39EA3DD0A4BE726937663E23
:10064000F16BD2C541BDBB3E2CDE25AF6A56113FD2
:1006500093BDBE166CC1663F3E5555555555C53FB9
:10066000412E8640FFFFEF7F422ED63FFFFF2F3EF9
:100670000000F03F28300100B1A2F03F48300100F7
:100680003830010041F0004101F58010C00F704783
:100690000020704781F0004102E000BF83F000437A
:1006A00030B54FEA41044FEA430594EA050F08BF0D
:1006B00090EA020F1FBF54EA000C55EA020C7FEAD1
:1006C000645C7FEA655C00F0E2804FEA5454D4EB4E
:1006D0005555B8BF6D420CDD2C4480EA020281EA18
:1006E000030382EA000083EA010180EA020281EA50
:1006F0000303362D88BF30BD11F0004F4FEA0131A2
:100700004FF4801C4CEA113102D0404261EB4101B0
:1007100013F0004F4FEA03334CEA133302D0524236
:1007200063EB430394EA050F00F0A780A4F10104F2
:10073000D5F1200E0DDB02FA0EFC22FA05F280182C
:1007400041F1000103FA0EF2801843FA05F3594112
:100750000EE0A5F120050EF1200E012A03FA0EFC91
:1007600028BF4CF0020C43FA05F3C01851EBE371BB
:1007700001F0004507D54FF0000EDCF1000C7EEBD8
:1007800000006EEB0101B1F5801F1BD3B1F5001F16
:100790000CD349085FEA30004FEA3C0C04F1010435
:1007A0004FEA445212F5800F80F09A80BCF1004F5E
:1007B00008BF5FEA500C50F1000041EB045141EAE0
:1007C000050130BD5FEA4C0C404141EB010111F4E1
:1007D000801FA4F10104E9D191F0000F04BF01468C
:1007E0000020B1FA81F308BF2033A3F10B03B3F16A
:1007F00020020CDA0C3208DD02F1140CC2F10C02FA
:1008000001FA0CF021FA02F10CE002F11402D8BF57
:10081000C2F1200C01FA02F120FA0CFCDCBF41EA23
:100820000C019040E41AA2BF01EB0451294330BDF2
:100830006FEA04041F3C1CDA0C340EDC04F11404CF
:10084000C4F1200220FA04F001FA02F340EA0300A6
:1008500021FA04F345EA030130BDC4F10C04C4F1EC
:10086000200220FA02F001FA04F340EA03002946CC
:1008700030BD21FA04F0294630BD94F0000F83F416
:10088000801306BF81F480110134013D4EE77FEAF9
:10089000645C18BF7FEA655C29D094EA050F08BF45
:1008A00090EA020F05D054EA000C04BF1946104626
:1008B00030BD91EA030F1EBF0021002030BD5FEA6A
:1008C000545C05D14000494128BF41F0004130BD92
:1008D00014F580043CBF01F5801130BD01F00045E6
:1008E00045F0FE4141F470014FF0000030BD7FEA59
:1008F000645C1ABF194610467FEA655C1CBF0B4654
:10090000024650EA013406BF52EA033591EA030F6A
:1009100041F4002130BD00BF90F0000F04BF002162
:10092000704730B54FF4806404F132044FF0000595
:100930004FF0000150E700BF90F0000F04BF00210E
:10094000704730B54FF4806404F1320410F0004574
:1009500048BF40424FF000013EE700BF42004FEA6F
:10096000E2014FEA31014FEA02701FBF12F07F43EC
:1009700093F07F4F81F06051704792F0000F14BFE9
:1009800093F07F4F704730B54FF4607401F000452D
:1009900021F0004120E700BF50EA010208BF704784
:1009A00030B54FF000050AE050EA010208BF704779
:1009B00030B511F0004502D5404261EB41014FF4E2
:1009C000806404F132045FEA915C3FF4DCAE4FF0E6
:1009D00003025FEADC0C18BF03325FEADC0C18BFCD
:1009E000033202EBDC02C2F1200300FA03FC20FA1E
:1009F00002F001FA03FE40EA0E0021FA02F114446B
:100A0000C1E600BF70B54FF0FF0C4CF4E06C1CEA7F
:100A100011541DBF1CEA135594EA0C0F95EA0C0FF4
:100A200000F0DEF82C4481EA030621EA4C5123EA67
:100A30004C5350EA013518BF52EA033541F4801196
:100A400043F4801338D0A0FB02CE4FF00005E1FB49
:100A500002E506F00042E0FB03E54FF00006E1FB93
:100A600003569CF0000F18BF4EF0010EA4F1FF04D6
:100A7000B6F5007F64F5407404D25FEA4E0E6D4116
:100A800046EB060642EAC62141EA55514FEAC52027
:100A900040EA5E504FEACE2EB4F1FD0C88BFBCF5A3
:100AA000E06F1ED8BEF1004F08BF5FEA500E50F154
:100AB000000041EB045170BD06F0004646EA01011A
:100AC00040EA020081EA0301B4EB5C04C2BFD4EB4C
:100AD0000C0541EA045170BD41F480114FF0000E45
:100AE000013C00F3AB8014F1360FDEBF002001F0B3
:100AF000004170BDC4F10004203C35DA0C341BDC2D
:100B000004F11404C4F1200500FA05F320FA04F0FE
:100B100001FA05F240EA020001F0004221F0004132
:100B200010EBD37021FA04F642EB06015EEA430EA5
:100B300008BF20EAD37070BDC4F10C04C4F12005D5
:100B400000FA04F320FA05F001FA04F240EA020088
:100B500001F0004110EBD37041F100015EEA430E59
:100B600008BF20EAD37070BDC4F1200500FA05F279
:100B70004EEA020E20FA04F301FA05F243EA0203F8
:100B800021FA04F001F0004121FA04F220EA020007
:100B900000EBD3705EEA430E08BF20EAD37070BD4D
:100BA00094F0000F0FD101F00046400041EB01012D
:100BB00011F4801F08BF013CF7D041EA060195F00F
:100BC000000F18BF704703F00046520043EB0303C9
:100BD00013F4801F08BF013DF7D043EA06037047B6
:100BE00094EA0C0F0CEA135518BF95EA0C0F0CD0C1
:100BF00050EA410618BF52EA4306D1D181EA030107
:100C000001F000414FF0000070BD50EA410606BF00
:100C10001046194652EA430619D094EA0C0F02D145
:100C200050EA013613D195EA0C0F05D152EA03368A
:100C30001CBF104619460AD181EA030101F00041A8
:100C400041F0FE4141F470014FF0000070BD41F0F1
:100C5000FE4141F4780170BD70B54FF0FF0C4CF4CB
:100C6000E06C1CEA11541DBF1CEA135594EA0C0FEA
:100C700095EA0C0F00F0A7F8A4EB050481EA030E37
:100C800052EA03354FEA013100F088804FEA03331E
:100C90004FF0805545EA131343EA12634FEA0222EC
:100CA00045EA111545EA10654FEA00260EF00041AD
:100CB0009D4208BF964244F1FD0404F5407402D2FF
:100CC0005B084FEA3202B61A65EB03055B084FEA90
:100CD00032024FF480104FF4002CB6EB020E75EB8D
:100CE000030E22BFB61A754640EA0C005B084FEAB5
:100CF0003202B6EB020E75EB030E22BFB61A754632
:100D000040EA5C005B084FEA3202B6EB020E75EB7C
:100D1000030E22BFB61A754640EA9C005B084FEAF4
:100D20003202B6EB020E75EB030E22BFB61A754601
:100D300040EADC0055EA060E18D04FEA051545EAF0
:100D400016754FEA06164FEAC30343EA52734FEA99
:100D5000C2025FEA1C1CC0D111F4801F0BD141EA12
:100D600000014FF000004FF0004CB6E711F4801F77
:100D700004BF01430020B4F1FD0C88BFBCF5E06F57
:100D80003FF6AFAEB5EB030C04BFB6EB020C5FEA67
:100D9000500C50F1000041EB045170BD0EF0004EBC
:100DA0004EEA113114EB5C04C2BFD4EB0C0541EAEE
:100DB000045170BD41F480114FF0000E013C90E6EB
:100DC00045EA060E8DE60CEA135594EA0C0F08BFAF
:100DD00095EA0C0F3FF43BAF94EA0C0F0AD150EAAE
:100DE00001347FF434AF95EA0C0F7FF425AF104641
:100DF00019462CE795EA0C0F06D152EA03353FF469
:100E0000FDAE1046194622E750EA410618BF52EAE5
:100E100043067FF4C5AE50EA41047FF40DAF52EAB9
:100E200043057FF4EBAE12E74FF0FF3C06E000BF56
:100E30004FF0010C02E000BF4FF0010C4DF804CD63
:100E40004FEA410C7FEA6C5C4FEA430C18BF7FEA23
:100E50006C5C1BD001B050EA410C0CBF52EA430C51
:100E600091EA030F02BF90EA020F0020704710F1D1
:100E7000000F91EA030F58BF994208BF90422CBF60
:100E8000D8176FEAE37040F0010070474FEA410C59
:100E90007FEA6C5C02D150EA013C07D14FEA430C77
:100EA0007FEA6C5CD6D152EA033CD3D05DF8040BE8
:100EB000704700BF8446104662468C46194663461A
:100EC00000E000BF01B5FFF7B7FF002848BF10F1F1
:100ED000000F01BD4DF808EDFFF7F4FF0CBF012036
:100EE00000205DF808FB00BF4DF808EDFFF7EAFFB2
:100EF00034BF012000205DF808FB00BF4DF808ED6D
:100F0000FFF7E0FF94BF012000205DF808FB00BF61
:100F10004DF808EDFFF7CEFF94BF012000205DF8EB
:100F200008FB00BF4DF808EDFFF7C4FF34BF0120F8
:100F300000205DF808FB00BF4FEA410C7FEA6C5CC3
:100F400002D150EA013C0AD14FEA430C7FEA6C5CC3
:100F500002D152EA033C02D14FF0000070474FF03B
:100F6000010070474FEA410212F5001215D211D567
:100F70006FF47873B3EB625212D94FEAC12343F096
:100F8000004343EA505311F0004F23FA02F018BF18
:100F9000404270474FF00000704750EA013005D1E1
:100FA00011F0004008BF6FF0004070474FF00000A4
:100FB000704700BF4A0011D212F5001211D20DD5B0
:100FC0006FF47873B3EB62520ED44FEAC12343F04F
:100FD000004343EA505323FA02F070474FF00000F9
:100FE000704750EA013002D14FF0FF3070474FF0A8
:100FF000000070474FEA4102B2F1E04324BFB3F56D
:10100000001CDCF1FE5C0DD901F0004C4FEAC0027F
:101010004CEA5070B2F1004F40EB830008BF20F063
:101020000100704711F0804F21D113F13872BCBF1D
:1010300001F00040704741F480114FEA5252C2F172
:101040001802C2F1200C10FA0CF320FA02F018BFBB
:1010500040F001004FEAC1234FEAD32303FA0CFC0E
:1010600040EA0C0023FA02F34FEA4303CCE77FEA9D
:10107000625307D150EA01331EBF4FF0FE4040F4E7
:101080004000704701F0004040F0FE4040F4000096
:10109000704700BF80F0004002E000BF81F00041D7
:1010A00042001FBF5FEA410392EA030F7FEA226C0E
:1010B0007FEA236C6AD04FEA1262D2EB1363C1BF9E
:1010C000D218414048404140B8BF5B42192B88BF0D
:1010D000704710F0004F40F4000020F07F4018BF30
:1010E000404211F0004F41F4000121F07F4118BF50
:1010F000494292EA030F3FD0A2F1010241FA03FCF8
:1011000010EB0C00C3F1200301FA03F100F00043DF
:1011100002D5494260EB4000B0F5000F13D3B0F1A7
:10112000807F06D340084FEA310102F10102FE2A16
:1011300051D2B1F1004F40EBC25008BF20F0010086
:1011400040EA03007047490040EB000010F4000F34
:10115000A2F10102EDD1B0FA80FCACF1080CB2EBC7
:101160000C0200FA0CF0AABF00EBC2505242184326
:10117000BCBFD0401843704792F0000F81F40001CB
:1011800006BF80F400000132013BB5E74FEA41039E
:101190007FEA226C18BF7FEA236C21D092EA030F0A
:1011A00004D092F0000F08BF0846704790EA010F84
:1011B0001CBF0020704712F07F4F04D1400028BFB1
:1011C00040F00040704712F100723CBF00F5000093
:1011D000704700F0004343F0FE4040F400007047C9
:1011E0007FEA226216BF08467FEA23630146420275
:1011F00006BF5FEA412390EA010F40F48000704788
:101200004FF0000304E000BF10F0004348BF40422D
:101210005FEA000C08BF704743F0964301464FF069
:1012200000001CE050EA010208BF70474FF00003C5
:101230000AE000BF50EA010208BF704711F0004306
:1012400002D5404261EB41015FEA010C02BF8446D6
:101250000146002043F0B64308BFA3F18053A3F535
:101260000003BCFA8CF2083AA3EBC25310DB01FA7C
:1012700002FC634400FA02FCC2F12002BCF1004F00
:1012800020FA02F243EB020008BF20F00100704791
:1012900002F1200201FA02FCC2F1200250EA4C00E5
:1012A00021FA02F243EB020008BF20EADC7070472B
:1012B0004FF0FF0C1CEAD0521EBF1CEAD15392EA39
:1012C0000C0F93EA0C0F6FD01A4480EA010C400215
:1012D00018BF5FEA41211ED04FF0006343EA50106F
:1012E00043EA5111A0FB01310CF00040B1F5000FB1
:1012F0003EBF490041EAD3715B0040EA010062F160
:101300007F02FD2A1DD8B3F1004F40EBC25008BF49
:1013100020F00100704790F0000F0CF0004C08BF67
:1013200049024CEA502040EA51207F3AC2BFD2F134
:10133000FF0340EAC250704740F400004FF0000342
:10134000013A5DDC12F1190FDCBF00F0004070477C
:10135000C2F10002410021FA02F1C2F1200200FABA
:1013600002FC5FEA310040F1000053EA4C0308BF81
:1013700020EADC70704792F0000F00F0004C02BFD2
:10138000400010F4000F013AF9D040EA0C0093F04D
:10139000000F01F0004C02BF490011F4000F013BA7
:1013A000F9D041EA0C018FE70CEAD15392EA0C0F15
:1013B00018BF93EA0C0F0AD030F0004C18BF31F080
:1013C000004CD8D180EA010000F00040704790F056
:1013D000000F17BF90F0004F084691F0000F91F0FA
:1013E000004F14D092EA0C0F01D142020FD193EAC0
:1013F0000C0F03D14B0218BF084608D180EA010048
:1014000000F0004040F0FE4040F40000704740F023
:10141000FE4040F4400070474FF0FF0C1CEAD052F1
:101420001EBF1CEAD15392EA0C0F93EA0C0F69D04D
:10143000A2EB030280EA010C49024FEA402037D0B8
:101440004FF0805343EA111143EA10130CF00040AF
:101450008B4238BF5B0042F17D024FF4000C8B429F
:1014600024BF5B1A40EA0C00B3EB510F24BFA3EB7F
:10147000510340EA5C00B3EB910F24BFA3EB91034F
:1014800040EA9C00B3EBD10F24BFA3EBD10340EAA9
:10149000DC001B0118BF5FEA1C1CE0D1FD2A3FF6EF
:1014A00050AF8B4240EBC25008BF20F001007047A4
:1014B0000CF0004C4CEA50207F32C2BFD2F1FF0347
:1014C00040EAC250704740F400004FF00003013A78
:1014D00037E792F0000F00F0004C02BF400010F41C
:1014E000000F013AF9D040EA0C0093F0000F01F030
:1014F000004C02BF490011F4000F013BF9D041EA52
:101500000C0195E70CEAD15392EA0C0F08D1420284
:101510007FF47DAF93EA0C0F7FF470AF084676E757
:1015200093EA0C0F04D14B023FF44CAF08466EE730
:1015300030F0004C18BF31F0004CCAD130F00042FE
:101540007FF45CAF31F000437FF43CAF5FE700BF56
:101550004FF0FF3C06E000BF4FF0010C02E000BF7F
:101560004FF0010C4DF804CD4FEA40024FEA410321
:101570007FEA226C18BF7FEA236C11D001B052EAD7
:10158000530C18BF90EA010F58BFB2EB030088BF9D
:10159000C81738BF6FEAE17018BF40F0010070470C
:1015A0007FEA226C02D15FEA402C05D17FEA236CEE
:1015B000E4D15FEA412CE1D05DF8040B704700BF35
:1015C000844608466146FFE70FB5FFF7C9FF0028CC
:1015D00048BF10F1000F0FBD4DF808EDFFF7F4FF05
:1015E0000CBF012000205DF808FB00BF4DF808ED9E
:1015F000FFF7EAFF34BF012000205DF808FB00BFC1
:101600004DF808EDFFF7E0FF94BF012000205DF8E2
:1016100008FB00BF4DF808EDFFF7D2FF94BF012093
:1016200000205DF808FB00BF4DF808EDFFF7C8FF8C
:1016300034BF012000205DF808FB00BF4FEA4002E4
:10164000B2F1FE4F0FD34FF09E03B3EB12620DD9F0
:101650004FEA002343F0004310F0004F23FA02F05A
:1016600018BF404270474FF00000704712F1610F01
:1016700001D1420205D110F0004008BF6FF00040D8
:1016800070474FF00000704742000ED2B2F1FE4F9B
:101690000BD34FF09E03B3EB126209D44FEA002341
:1016A00043F0004323FA02F070474FF00000704708
:1016B00012F1610F01D1420202D14FF0FF307047A9
:1016C0004FF00000704700BF014B1868704700BF23
:1016D0002899FF1F70B50F4E0F4D761BB61018BF1F
:1016E000002405D0013455F8043B9847A642F9D1AF
:1016F0000A4E0B4D761B01F0B1FCB61018BF00244A
:1017000006D0013455F8043B9847A642F9D170BD84
:1017100070BD00BF68300100683001007430010006
:1017200068300100024B0146186800F003B800BFA2
:101730002899FF1F2DE9F04F01F10B05162D83B0FD
:10174000064640F29F8035F0070500F1BF80A942B0
:1017500000F2BC8000F0F4FAB5F5FC7FC0F09C828A
:101760006B0A00F0BA80042B00F28381A80900F113
:10177000390E4FEA4E033830C44F07EB8303A3F111
:1017800008015C68A14207D1ACE0002A80F2AC807D
:10179000E468A14200F0A680636823F003035A1BAB
:1017A0000F2AF2DDB9493C6901F1080E744500F0D9
:1017B000B381636823F003035A1B0F2A00F3998156
:1017C000002AC1F814E0C1F810E080F29E80B3F561
:1017D000007F80F06781DB0803F1010C01229B1080
:1017E00002FA03F34A6851F83C80C4F8088001EB20
:1017F000CC091A43A9F10803E3604A6041F83C4070
:10180000C8F80C40831001249C40944200F28A8066
:10181000144206D120F003006400144200F10400D9
:10182000FAD007EBC009CC468046DCF80C108C459A
:1018300007D173E1002A80F28181C9688C4500F0EC
:101840006D814B6823F003035A1B0F2AF2DD0C460F
:10185000D1F80CC054F8088F4B1945F001054D60C4
:1018600042F00101C8F80CC03046CCF808807B611A
:101870003B61C3F80CE0C3F808E059609A5000F0EF
:1018800061FA1FE0102921D800F05AFA102506232A
:1018900002207E4F07EB8303A3F108025C689442A9
:1018A00000F045816368E168A56823F003032344E1
:1018B00030465A68E96042F001028D605A6000F0DB
:1018C00041FA0834204603B0BDE8F08F00240C2311
:1018D0002046336003B0BDE8F08F80234FF0400E08
:1018E0003F2049E770465DE72344E1685A68A568F0
:1018F00042F00102E96030468D605A6000F022FA41
:101900000834204603B0BDE8F08F234430465A68BF
:1019100042F001025A6000F015FA0834204603B084
:10192000BDE8F08FBC68636823F00308A84504D3C2
:10193000C5EB08030F2B00F38C80554BDFF860914B
:101940001A68D9F8003001332A4404EB080A00F081
:10195000608102F580520F3222F47F6222F00F0282
:1019600011463046019200F0EFF9B0F1FF3F834697
:10197000019A00F05881824500F2FC80454B1968BD
:10198000DA451144196000F05381D9F80000DFF8FE
:1019900010E101301BBFCAEB0B0A5144CEF800B076
:1019A00019601BF0070100F01781C1F10800C1F5B3
:1019B0008051834408315A44C2F30B02C2EB01093F
:1019C00049463046019300F0BFF9431C019B00F0EB
:1019D0003F81CBEB00024A4442F001021968C7F88C
:1019E00008B04944BC42CBF804201960DFF8A49049
:1019F00016D0B8F10F0F40F2FD806268A8F10C0319
:101A000023F00703E01802F001024FF0050E1A431D
:101A10000F2B6260C0F804E0C0F808E000F21C81FF
:101A20001D4BBC681A68914288BF19601B4B1A682D
:101A30009142626888BF196022F003029542A2EBCE
:101A4000050301D80F2B04DC304600F07BF900249D
:101A500038E7621943F0010345F00105656030463F
:101A6000BA60536000F06EF90834204603B0BDE858
:101A7000F08F142B71D9542B00F2A480280B00F1A5
:101A80006F0E4FEA4E036E3076E600BF2C99FF1FB3
:101A9000CCA1FF1FD0A1FF1FC8A1FF1FC4A1FF1F22
:101AA000389DFF1F5A0A042A5ED9142A00F2B38017
:101AB00002F15C0149005B3207EB810C57F8211001
:101AC000DFF8DC81ACF1080C8C4500F088804A68B6
:101AD00022F00302934202D289688C45F7D1D1F8F3
:101AE0000CC07A68C4F80CC0A160CCF80840CC6087
:101AF00088E6631942F0010745F00105656030464C
:101B00004B610B61C3F80CE0C3F808E05F609A50CA
:101B1000083400F017F9D5E64A6873E608F10108C1
:101B200018F0030F0CF1080C7FF47FAE30E0DC6896
:101B3000A34208BF02303FF435AEB3E60B440C4677
:101B40005A68C96854F8085F42F001025A6030468A
:101B5000E9608D6000F0F6F8B4E603F15C0E03F185
:101B60005B004FEA4E0307E69A0902F1390149008A
:101B70003832A1E7BC424A4B3FF400AF9C68626830
:101B800022F003025AE759F80839994540F082805B
:101B900010F0030F00F1FF30F5D17B6823EA040356
:101BA0007B6064009C423FF6BDAE002C3FF4BAAEB1
:101BB0001C4240467FF435AE64001C4200F1040034
:101BC000FAD02EE6B3F5AA7F18D8E80B00F1780E0C
:101BD0004FEA4E037730CFE54FF48051EBE6012119
:101BE000D8F80430921001FA02F21A43C8F804201F
:101BF000614677E70123CBF8043025E740F25452E1
:101C0000934220D8A80C00F17D0E4FEA4E037C30A1
